:0600000024EF06F01200DF
:0600080004EF08F01200F5
:100018000CEF08F012001DEE00F02DEE00F0F86A6B
:0600280040EF06F012009B
:1000300001000E0E0000E6000000020000003E0E6F
:10004000006E016AFC0E026E036A046A07680868A3
:100050000968066A1200D9CFE6FFE1CFD9FFE65260
:1000600004501EE1040108BF1AD0400EE66E600E77
:10007000E66E000EE66E34EC05F0E552E552E55210
:10008000010E046EDF6A400EDF5C09E2DF50EA6AAF
:10009000A00FE96E000EEA22EF6ADF2AF4D717D12B
:1000A00000016051080A01E10DD10F0A01E1D3D02E
:1000B000010A01E1CAD0030A67E0010A58E0070A11
:1000C00044E0010A01E003D10001020EA06F00012B
:1000D0003A0EA16F0001010EA26F0001010EA36F85
:1000E0000001A46B100EA56FA66BA76B01C0A8F052
:1000F00002C0A9F003C0AAF0100E0001A95F000E13
:100100000001AA5B0001AB6B0001030EAC6F0001A4
:10011000F80EAD6FAE69AF6BB06B0001080EB16F3A
:10012000B26BB36BB46B0001B56904010CBF0CD0AA
:10013000400EE66EA00EE66E000EE66E04EC05F0D4
:10014000E552E552E552046AC2D00001615107E16F
:100150003F0E006EF80E016E0268036A06D03E0E76
:10016000006E016AFC0E026E036A046AB0D0040ECF
:10017000056E0028055C06E20400AED88EEC05F0A2
:10018000052AF7D7046AA3D0E868071805E1E868EC
:10019000081802E1E868091806E161C007F062C0CA
:1001A00008F063C009F007500001611908E1085028
:1001B0000001621904E109500001631900E143E103
:1001C000DF6A00016551DF5C3EE2000E075C100E45
:1001D0000858000E09582CE30028596E5A6A0A0E76
:1001E000D89059365A36E806FBE15B6A5ABE5B681E
:1001F0005950075C5A5008585B50095819E23A0E9A
:100200000001D8806555DF24EA6A660FE96E000EAA
:10021000EA22EF50E66E0650E96EEA6AE9BEEA6845
:100220000A0EE926000EEA22E552E750EF6E062A92
:10023000072A000E0822000E09223A0E065C01E190
:100240005ED8DF2ABED7046A42D059D8076808684A
:100250000968046A3CD00001070EA06F61C0A1F0DC
:1002600062C0A2F063C0A3F064C0A4F065C0A5F0B2
:1002700061C0F6FF62C0F7FF63C0F8FFDF6A0001EC
:100280006551DF5C0FE209003A0E0001D880655528
:10029000DF24EA6AA60FE96E000EEA22F5CFEFFF2F
:1002A000DF2AEDD704010CBF0CD0400EE66EA00E85
:1002B000E66E000EE66E04EC05F0E552E552E552FE
:1002C000046A05D06592656A68D8FF0000D0E552DF
:1002D000E552E7CFD9FF1200F66A0550F76EF86ACB
:1002E000D890F736F836F736F836140EA66EF29E2A
:1002F000550EA76EAA0EA76EA682A6941200D9CF9D
:10030000E6FFE1CFD9FFE652DF6A000EE76E06187E
:10031000E8AE02D0063403D0E750D880065436E267
:100320000650596E5A6A5B6A59AE02D05A685B68C9
:100330005950075CF66E5A500858F76E5B500958D2
:10034000F86EDF50EA6A0A0FE96E000EEA22EF50FB
:10035000F56E0D00DF2A0606065009E0DF50EA6A56
:100360000A0FE96E000EEA22EF50F56E01D0F56833
:100370000C00DF2A240EA66EF29E550EA76EAA0E62
:10038000A76EA682065001E00606BFD7A694066AAD
:10039000E552E552E7CFD9FF1200D9CFE6FFE1CF12
:1003A000D9FFE652DF6AFF0EDF5C0AE2E868E85038
:1003B00005E0E80600D000D000D0F9D7DF2AF3D757
:1003C000E552E552E7CFD9FF12005FD9E6526450FB
:1003D00032E16296040100513C0BE842E8420D080C
:1003E00028E1180E021923E1040E031920E1100E72
:1003F000026F040E036FDF6ADF50596E5A6A080EEF
:10040000595C000E5A5813E2DF50EA6A180FE96E81
:10041000040EEA22EF50E66EDF50EA6A100FE96E32
:10042000040EEA22E552E750EF6EDF2AE5D70ED838
:100430000AD03DD808D0040E645C03E162964DD822
:1004400002D0000E01D0010EE55224D11ED9E65291
:10045000040104BF046B536A4F6A506A516A526ABE
:1004600055EC03F0DF6ADF50596E5A6A010E595C91
:10047000000E5A5819E2505017E1F76ADF34FE0BAC
:10048000F736F66EEC0EF6260D0EF7220900F5CFC4
:1004900059F00800F5CF5AF004D05AC0FAFF59506D
:1004A000F96EFBDFDF2ADFD79ED8E552F3D0020ECC
:1004B0004F5C0EE176D80401180E026F040E036F34
:1004C000080E016F00BD02D0C80E05D0880E03D003
:1004D000BCD8CCD88C0E006F1200040E555C0AE11B
:1004E00012C438FF0F013851000802E2050E01D096
:1004F000030E556E4F040FE110D8020E535C03E15A
:100500000401840E06D0040104BD02D0C80E01D03F
:10051000880E046F120025EF03F0B7D8020EE12613
:10052000080E515C000E52580DE251C0DEFF52C061
:10053000DDFF535002E1010E03D0530406E1020E29
:10054000536E03D0080EDE6EDD6A0401049304913D
:10055000010EDB500413DFCF05F4DE50515EDD5099
:10056000525A0001180EE26F040EE36F56A20CD02F
:1005700085D810E0E0C0F6FFE1C0F7FF0800F550B5
:1005800068D8F6E2DB06F4D779D804E087D8FCE235
:10059000DB06FAD7020EE15C02E2E16AE552E16EA7
:1005A00079D073D8020EE126030E04010015E76E20
:1005B000010EE7CFDBFF01C4DFFFDE505126DD5027
:1005C00052220001180EE06F040EE16F57D804E0CC
:1005D00065D8FCE2DB06FAD7020EE15C02E2E16AD2
:1005E000E552E16E57D06598505005E13FD8840E32
:1005F000006F040118D0040110AF17D05150165DE0
:100600005250175904E216C451F017C452F085DF56
:10061000010E4F6E2BD8800E006F0401180E066F6E
:10062000040E076FC80E046F1200020E4F6E040115
:10063000056BC80E046F0401080E016F180E026FDF
:10064000040E036FC80E006F12004F6A0401046BA2
:100650001200E2C0E9FFE3C0EAFFEF6EE22B000EFA
:10066000E323E02BE123DF06010E12000401080E54
:10067000016F100E026F040E036F1200D9CFE9FF55
:10068000DACFEAFFEE50ED101200D9CFE6FFE1CF4E
:10069000D9FF1200E552E7CFD9FF1200E0C0E9FF11
:1006A000E1C0EAFFEF5029EF03F004011051600BA5
:1006B000E842E842E842E842E842000901E012006C
:1006C0001151070A43E00B0A41E0070A34E0010A2E
:1006D00024E00B0A20E0020A1EE0030A1AE0080ADE
:1006E00010E0010A0CE00F0A08E0030A01E0120022
:1006F000010E506E040E556E1200A7EF03F0DDEFF1
:1007000003F0010E506E0001570EE06F000EE16F16
:100710000ED0F7EF03F025EF04F0010E506E1451E8
:100720000001E06FE16B580EE027000EE1235692C6
:10073000010E516E1200010E506E1451EA6A580FEC
:10074000E96E000EEA2212C4EFFF12001200800EC2
:100750000401105D31E11351030A20E0010A0BE0AE
:10076000030A29E1010E506E00012C0EE06F0D0E00
:10077000E16F120E1ED0AAD8E20EF6260D0EB8D8E2
:10078000020E0001F76AE025F66EE151F72209003A
:10079000F5CF51F00A00F5CF52F00DD097D8E60E04
:1007A000F6260D0EA5D8E0C0F6FFE1C0F7FF080061
:1007B000F550516E526A56821200010E506E0F0EA5
:1007C000E66E270EE66E0F0E9BD8010EE66E580EF3
:1007D000E66E000E95D812C457F00401125103E1E1
:1007E000050E556E1200060E556EEFEF04F0040173
:1007F000186B196B040110511F0B020A0EE0030A5B
:1008000009E0010A17E1010E506E56A013D0040151
:10081000188310D0010E506E0DD04AD801E0010EA1
:100820005ED8E2C0E9FFEA6EEF50040B03E004017A
:10083000010E186F500408E10001180EE06F040E5D
:10084000E16F5692020E516E1200040112050CE186
:1008500010511F0B000908E1010E506E030E115DCF
:1008600002E1568001D05690125121E110511F0B28
:1008700002081DE114510F0B000919E019D801E01D
:10088000010E2DD8030E0401115D02E1840E03D088
:1008900014AF07D0400EE2C0E9FFE3C0EAFFEF6EFD
:1008A0001200880EE2C0E9FFE3C0EAFFEF6E12001B
:1008B000010E506E14510F0B080DF3505A6A000FC1
:1008C000596E040E5A221451800B1200010E506E04
:1008D0001251F66EF76AD890F636F7361200040D0C
:1008E000F35000015924E26F000E5A20E36F12000A
:1008F000F7220900F5CFE0F00A00F5CFE1F0120091
:10090000E66E0FEC06F0E552E552E55212000401E6
:1009100010511F0B010801E01200145101E01200F8
:10092000060E115D21E11351230A1DE0010A0DE0BD
:10093000030A19E1020E506E570405E10001500E42
:10094000E06F0D0EE16F090E0CD0020E506E5704D1
:1009500005E10001C50EE06F0D0EE16F570403E1E4
:100960001D0E516E526A568204011051600BE8420E
:10097000E842E842E842E842010801E01200115171
:100980000B0A26E0080A19E0090A12E0080A09E041
:100990000B0A05E0080A01E01200EDEF04F0EEEFAB
:1009A00004F0020E506E00014A0EE06F000E0BD0F4
:1009B000020E506E13C44AF01200020E506E000177
:1009C0004B0EE06F000EE16F5692010E516E120059
:1009D000020E506E12C44BF01200120012004C6A4C
:1009E0000F011E0E276F0401400E096F200E0A6FC3
:1009F000040E0B6F880E086F0401600E0E6F040E5C
:100A00000F6F400E0C6F1200D9CFE6FFE1CFD9FF78
:100A1000E652FC0EDB50400805E2400EF36EFC0E81
:100A2000F3CFDBFFDF6AFC0EDB50DF5C0FE2DF5051
:100A30004DD8EF50E66EDF50EA6A600FE96E040EA3
:100A4000EA22E552E750EF6EDF2AEDD7FC0EDBCF4E
:100A50000DF4400E04010C170C7D880E0C13E552AA
:100A6000E552E7CFD9FF1200D9CFE6FFE1CFD9FF9A
:100A70004C6A040108BF25D0FC0EDBCF59F00951A8
:100A8000D880595403E2FC0E09C4DBFF4C6AFC0E0B
:100A9000DB504C5C0FE24C50EA6A200FE96E040E0A
:100AA000EA22EF50E66E4C5011D8E552E750EF6E57
:100AB0004C2AEDD70401400E096F0817087D880EF7
:100AC00008134C50E552E7CFD9FF1200E76EFD0E38
:100AD000DBCFE9FFFE0EDBCFEAFFE750E926000E91
:100AE000EA22120065A60CD8550409E165BA07D0C0
:100AF000626A0F01366B36813689020E556E12001E
:100B0000656A0F01366B6586010E556E1200656AC7
:100B10000F01366B556A120087EF05F0555001E161
:100B200012006250040B05E00F013651040B01E086
:100B300032D865B212006250010B05E00F01365148
:100B4000010B01E03BD86250100B05E00F0136515C
:100B5000100B01E01FD86250200B05E00F01365149
:100B6000200B01E019D8030E555C01E21200546A13
:100B7000040E545C0EE26250080B0BE00F0136517C
:100B8000080B07E0E5EC01F0000901E16296542A48
:100B9000EFD71200120012000F0126A10DD0800E17
:100BA0000401005D07E1840E0401045D03E104011A
:100BB0008C0E006F0F012691629A1200636A626ABE
:100BC0000F019F0E376F0F017B0E366F0F01386BD1
:100BD0000F0EE66E270EE66E0F0EE66E20D8E5527B
:100BE000E552E5520F01160E266F62A605D06296F9
:100BF00000D000D00000F9D7659825EC03F004017F
:100C0000080E016F0401100E026F040E036F040141
:100C10008C0E006F5690576A030E556E1200D9CF96
:100C2000E6FFE1CFD9FFFD0EDBCFE9FFFE0EDBCF04
:100C3000EAFFFC0EDB5004E0EE6AFC0EDB06F9D79F
:100C4000E552E7CFD9FF12001DEE00F02DEE00F0C7
:100C5000F86AF66A100EF76E0800F550FF0808E112
:100C6000010EF66E100EF76E0800F550FF0806E054
:100C700080AE02D000EF08F080AEFED701D812009F
:100C80000DD8040032D835D8060E555C05E1655004
:100C9000020B02E12BEC00F0F4D71200600ED36ED1
:100CA0009B8C580E4D6E020E4E6E4DC059F04EC0CC
:100CB0005AF04D06000E4E5A59505A10F6E165A6EC
:100CC00004D06592656ACDEC01F00F01140E396F06
:100CD000556A566A576A1FEC00F08C968C9495966C
:100CE00095940F01486B496B120072EC05F08EEF82
:100CF00005F0060E555C02E28C868C94060E555C5F
:100D000014E10001200EE65D4E0EE75902E38C86E9
:100D10008C94400EE65D9C0EE75904E38C968C841F
:100D2000E66BE76BE62B000EE723120012010002D0
:100D300000000008D8043C00020001020001090282
:100D40002900010100C03209040000020300000074
:100D5000092111010001221D000705810340000146
:100D6000070501034000010403090434034D006931
:100D700000630072006F006300680069007000206B
:100D80000054006500630068006E006F006C006F27
:100D90000067007900200049006E0063002E0026E5
:100DA0000348004900440020005500530042002041
:100DB0000042006F006F0074006C006F00610064FF
:100DC00000650072000600FF0901A1011901294018
:100DD000150026FF007508954081001901294091F2
:100DE00000C03E0D3E0D670D6B0D9F0D0E09C00E30
:100DF000F36E00EE00F00E0E01D81200EA6002D091
:100E0000EE6AFCD7F350E9601200EE6AFCD70000EE
:0610000049EF65F012004B
:0610080074EF24F0120059
:061018002FEF3AF0120078
:10102A00040074CB000000050000E900000071CA4A
:10103A000000B70E00000100000072CB0000FE04A1
:10104A00000002000000F4CA0000800200007E00D6
:10105A000000020100000000000132000000000050
:10106A000180004D00000002000000000000013273
:10107A00000000000001A700FBFFDFFF015700EF9F
:10108A00FF0400014E00F2FF0700014C00F3FF08C5
:10109A0000014A00F5FF0A00014400F8FF0B0001B5
:1010AA004800FAFF0D00014E00FCFF0F000150003E
:1010BA00FFFF100001320000000A00012E000200AA
:1010CA00090001330002000A00012D000400080093
:1010DA00012D0004000800012F000500080001315D
:1010EA000007000700012E00070006000132000871
:1010FA00000600013300090005000136000A000459
:10110A00000134000A0003000139000B000300014A
:10111A003D000C0002000141000D000100014600E3
:10112A000E0001000146000E00FFFF0141000D0004
:10113A00FFFF013D000C00FEFF013E000C00FDFF19
:10114A000139000B00FDFF0136000A00FCFF0133E4
:10115A00000900FBFF0132000800FAFF0135000810
:10116A0000F9FF012E000600F9FF012E000600F922
:10117A00FF012D000400F8FF012D000400F8FF0113
:10118A002E000200F7FF012E000200F7FF013200D5
:10119A000000F6FF012D000000F7FF012E00FEFF00
:1011AA00F7FF012900FEFFF8FF012B00FDFFF8FF02
:1011BA00012F00FBFFF8FF012B00FBFFF9FF0131B4
:1011CA0000F9FFF9FF012E00F9FFFAFF013200F8DA
:1011DA00FFFAFF013300F7FFFBFF013600F6FFFCC1
:1011EA00FF013900F5FFFDFF013900F5FFFDFF01A1
:1011FA003D00F4FFFEFF014100F3FFFFFF0146003F
:10120A00F2FFFFFF013200F6FF010001C6020000F3
:10121A008E00015B00EEFFFEFF015100F0FFFDFFB3
:10122A00014800F3FFFAFF014100F5FFF9FF013C15
:10123A0000F7FFF8FF013A00FAFFF6FF013600FC5B
:10124A00FFF6FF013C00FFFFF4FF0128000100F850
:10125A00FF0129000200F8FF0126000300F9FF013F
:10126A002B000500F9FF012E000700FAFF012F00ED
:10127A000800FBFF0133000900FBFF013F000C00DF
:10128A00FCFF010000000000000201000000000055
:10129A000132000000000001CE003F006A00020097
:1012AA0000000000000132000000000001120200EC
:1012BA000096FF0141000D000100013E000C0003F1
:1012CA00000134000A000300012F00080005000194
:1012DA0040000A000800013D0007000A00011B0047
:1012EA0002000500011B0002000500013C0001008C
:1012FA000C00013700FFFF0B00012F00FDFF090062
:10130A00013600FAFF0900013500F9FF0800013D26
:10131A0000F6FF0700013C00F5FF0500014400F359
:10132A00FF0400014600F2FF010001000000000076
:10133A00000201000000000001320000000000016C
:10134A00900164FF4AFF0200000000000001320021
:10135A000000000001A200FBFFE0FF012D00F7FFE3
:10136A00FFFF012600F9FFFDFF011D00FBFFFDFF46
:10137A00012000FBFFFCFF012700FBFFFAFF012B06
:10138A0000FDFFF8FF012E00FEFFF7FF013200FF0C
:10139A00FFF6FF0132000100F6FF0133000200F6FA
:1013AA00FF012B000300F8FF0127000500FAFF01E7
:1013BA002A000600FAFF012B000700FBFF012B00A1
:1013CA000800FDFF012F000900FDFF016000130066
:1013DA00FEFF019B001F000000012B00F9FF050022
:1013EA00012A00FAFF0600012700FBFF0600012878
:1013FA0000FCFF0700012400FCFF0600012400FE98
:10140A00FF0700012800FFFF0800012800FFFF086E
:10141A0000012D0001000900012D00010009000151
:10142A002F0003000900012D000400080001280014
:10143A0004000700012E0006000700012E00070025
:10144A000600013200080006000133000900050009
:10145A00013100090004000136000A0004000134C9
:10146A00000A000300016B00150004000173001755
:10147A00000100015000100000000151001000FEA0
:10148A00FF0148000E00FDFF014A000E00FBFF01AC
:10149A004A000E00FBFF0141000B00F9FF0140006A
:1014AA000A00F8FF0139000800F8FF013D000700B3
:1014BA00F6FF013C000500F5FF0138000200F5FFC8
:1014CA000141000100F3FF0128000000F8FF012993
:1014DA0000FEFFF8FF012400FEFFF9FF012800FCCF
:1014EA00FFF9FF012800FCFFF9FF012E00FAFFF9BE
:1014FA00FF012E00F9FFFAFF012B00F9FFFBFF01A4
:10150A0087001B0000000196000000E2FF01DE03D5
:10151A003AFF0000017D00E7FF0000016900EBFFD0
:10152A000200015600EFFF0300014400F3FF04002C
:10153A00013800F6FF0500013D00F6FF07000135FE
:10154A0000F8FF0700013D00F9FF0A00013A00FA1E
:10155A00FF0A00013F00FCFF0C00013D00FEFF0CEA
:10156A0000014600FFFF0E000150000100100001BB
:10157A004E0004000F0001480006000D000144005F
:10158A0008000B00012000040005000127000600E6
:10159A0005000122000600030001260007000300DF
:1015AA000124000700020001290008000200015579
:1015BA00001100010001000000000000020100000B
:1015CA000000000132000000000001EA008A00E584
:1015DA00FF020000000000000132000000000001CC
:1015EA006900EBFFFFFF015B00EEFFFDFF014F000B
:1015FA00F1FFFBFF012200FAFFFDFF012200FAFFC3
:10160A00FDFF013C00F7FFF8FF013900F9FFF7FF82
:10161A00013400FDFFF6FF013300FEFFF6FF01383B
:10162A00000200F5FF0134000300F6FF013900074C
:10163A0000F7FF013C000900F8FF011D000500FD4D
:10164A00FF0126000700FDFF014A000E00FBFF0113
:10165A005B001200FDFF0164001400FFFF0164003B
:10166A001400010001560011000300014F000F0091
:10167A0005000145000C000700013C0009000800B4
:10168A00013900070009000131000400090001378F
:10169A000001000B00013200FFFF0A00013600FCC6
:1016AA00FF0A00013900F9FF0900013C00F7FF08B1
:1016BA0000014300F4FF0600014A00F2FF050001A1
:1016CA005600EFFF0300015F00EDFF01000100007B
:1016DA0000000000020100000000000132000000CA
:1016EA00000001770176FF4EFF02000000000000B3
:1016FA000132000000000001A200FBFFE0FF012D03
:10170A0000F7FFFFFF012600F9FFFDFF011D00FBA7
:10171A00FFFDFF012000FBFFFCFF012700FBFFFA92
:10172A00FF012B00FDFFF8FF012E00FEFFF7FF016E
:10173A003200FFFFF6FF0132000100F6FF0133001D
:10174A000200F6FF012B000300F8FF012700050045
:10175A00FAFF012A000600FAFF012B000700FBFF2F
:10176A00012B000800FDFF012F000900FDFF0160A9
:10177A00001300FEFF019B001F000000012B00F96F
:10178A00FF0500012A00FAFF0600012700FBFF06F9
:10179A0000012400FCFF0600012800FCFF070001ED
:1017AA002400FEFF0700012800FFFF0800012800AF
:1017BA00FFFF0800012D0001000900012D000100B2
:1017CA000900012F00030009000128000400070096
:1017DA00012D0004000800012E0006000700012E5A
:1017EA000007000600013200080006000133000964
:1017FA00000500013100090004000136000A000456
:10180A00000134000A000300016B00150004000106
:10181A007300170001000150001000FFFF01500083
:10182A001000FFFF0148000E00FDFF014A000E00F4
:10183A00FBFF014A000E00FBFF0141000B00F9FF0C
:10184A000140000A00F8FF0139000800F8FF013DD5
:10185A00000700F6FF013C000500F5FF0138000211
:10186A0000F5FF0141000100F3FF0128000000F824
:10187A00FF012900FEFFF8FF012400FEFFF9FF0126
:10188A002800FCFFF9FF012800FCFFF9FF012E00E8
:10189A00FAFFF9FF012E00F9FFFAFF012B00F9FF09
:1018AA00FBFF0187001B0000000196000000E2FF19
:1018BA0001DE033AFF0000017D00E7FF0000016935
:1018CA0000EBFF0200015600EFFF0300014400F3A2
:1018DA00FF0400013800F6FF0500013D00F6FF078E
:1018EA0000013500F8FF0700013D00F9FF0A000179
:1018FA003A00FAFF0A00013F00FCFF0C00013D001C
:10190A00FEFF0C00014600FFFF0E0001500001001F
:10191A001000014E0004000F0001480006000D00EF
:10192A0001440008000B0001200004000500012406
:10193A000006000400012400060004000126000736
:10194A000003000124000700020001290008000228
:10195A000001550011000100010000000000000212
:10196A000100000000000132000000000001EA004E
:10197A008A00E5FF020000000000000132000000BA
:10198A000000016900EBFFFFFF015B00EEFFFDFFB6
:10199A00014F00F1FFFBFF012200FAFFFDFF0122C8
:1019AA0000FAFFFDFF013C00F7FFF8FF013900F9DB
:1019BA00FFF7FF013400FDFFF6FF013800FEFFF5D7
:1019CA00FF0133000200F6FF0134000300F6FF01B5
:1019DA0039000700F7FF013C000900F8FF011D006C
:1019EA000500FDFF0128000700FCFF0149000E0069
:1019FA00FCFF015B001200FDFF0164001400FFFF01
:101A0A000164001400010001560011000300014F97
:101A1A00000F0005000145000C000700013C000909
:101A2A00000800013900070009000131000400091B
:101A3A000001370001000B00013200FFFF0A00011C
:101A4A003600FCFF0A00013900F9FF0900013C00D9
:101A5A00F7FF0800014300F4FF0600014A00F2FF05
:101A6A000500015600EFFF0300015F00EDFF0100D2
:101A7A000100000000000002010000000000013225
:101A8A000000000000018D0189FF32FF0200000002
:101A9A000000000132000000000001960000001E54
:101AAA0000012C063C01000001A5000000DFFF0137
:101ABA00300290FF0000012B000700FBFF012A0003
:101ACA000600FAFF0127000500FAFF0127000500BA
:101ADA00FAFF0126000300F9FF0124000200F9FFC2
:101AEA000124000200F9FF0128000000F8FF012D7F
:101AFA00000000F7FF012900FEFFF8FF012900FEA0
:101B0A00FFF8FF012D00FCFFF8FF012F00FBFFF893
:101B1A00FF012B00FBFFF9FF012E00F9FFFAFF017D
:101B2A002B00F9FFFBFF012F00F8FFFBFF0131003B
:101B3A00F7FFFCFF013600F6FFFCFF013400F6FF59
:101B4A00FDFF013900F5FFFDFF013C00F4FFFFFF37
:101B5A00017800E8FFFEFF014600F2FF000001479E
:101B6A0000F2FF0200013D00F4FF0200013D00F413
:101B7A00FF0200013B00F5FF0400013600F6FF04F6
:101B8A0000013300F7FF0500013300F7FF050001EC
:101B9A003100F9FF0700012E00F9FF0600012B00B2
:101BAA00FBFF0700012B00FBFF0700012D00FCFFD4
:101BBA000800012400FEFF0700012900FEFF0800BB
:101BCA00012D000000090001280000000800012979
:101BDA000002000800012600030007000126000396
:101BEA0000070001270005000600012A000600067A
:101BFA0000012E0007000600012F00080005000161
:101C0A009100E3FF00000201000000000001320021
:101C1A000000000001C10074000000020000000082
:101C2A00000001320000000000015F00EDFFFFFF2D
:101C3A00015000F0FFFFFF014800F2FFFDFF0136EF
:101C4A0000F6FFFCFF012800F9FFFCFF012700FA5C
:101C5A00FFFBFF012000FBFFFCFF012300FBFFFB52
:101C6A00FF012200FDFFFAFF011B00FEFFFBFF013F
:101C7A002000FEFFFAFF0123000000F9FF013200F5
:101C8A000100F6FF0131000400F7FF0139000700E7
:101C9A00F7FF0140000A00F8FF0145000C00F9FFB8
:101CAA000154001000FBFF0156001100FDFF0169FD
:101CBA00001500FFFF01690015000100015B001219
:101CCA00000300014F000F00050001220006000377
:101CDA000001220006000300013C0009000800017F
:101CEA0035000700080001360004000A000132002E
:101CFA0001000A00013200FFFF0A00013600FCFF62
:101D0A000A00013900F9FF0900014000F6FF080046
:101D1A00014300F4FF0600014F00F1FF05000156E0
:101D2A0000EFFF0300016400ECFF01000100000066
:101D3A000000000201000000000001320000000063
:101D4A0000011001FFFF5DFF02000000000000011A
:101D5A00320000000000014B000F00FFFF014600A7
:101D6A000E00FFFF0148000E00FDFF013E000C00BF
:101D7A00FDFF013B000B00FCFF013C000B00FBFFD9
:101D8A000136000900FAFF0135000800F9FF012AAF
:101D9A00000600FAFF012B000500F9FF01280004E4
:101DAA0000F9FF0128000400F9FF012B000300F8E5
:101DBA00FF0129000200F8FF0128000100F8FF01D5
:101DCA002D000000F7FF0132000000F6FF012E008F
:101DDA00FEFFF7FF012E00FEFFF7FF012B00FDFFBC
:101DEA00F8FF012F00FBFFF8FF012B00FBFFF9FFB3
:101DFA00012E00FAFFF9FF013200F8FFFAFF013263
:101E0A0000F8FFFAFF012F00F8FFFBFF013800F688
:101E1A00FFFBFF013400F6FFFDFF013900F5FFFD6E
:101E2A00FF013D00F4FFFEFF014100F3FFFFFF0148
:101E3A004100F3FF0000016900EBFF0000016000B0
:101E4A00EDFF0200015200F0FF0400014A00F2FF18
:101E5A000500014300F4FF0600013D00F6FF0700FC
:101E6A00014000F7FF0900014000F8FF0A00013FA6
:101E7A0000FAFF0B00013C00FBFF0B00013D00FED6
:101E8A00FF0C00013C00FFFF0C0001320000000AB9
:101E9A0000012E0002000900012E000200090001C3
:101EAA002D0004000800012D0004000800012F0085
:101EBA0005000800012E0007000600013100070096
:101ECA00070001320008000600013300090005007E
:101EDA000136000A0004000134000A000300013E32
:101EEA00000C000300013D000C0002000146000E38
:101EFA000001000146000E00010001000000000080
:101F0A000002010000000000013200000000000190
:101F1A0039000000DEFF020000000000000132006C
:101F2A0000000000016900EBFFFFFF015B00EEFF0C
:101F3A00FDFF014F00F1FFFBFF012200FAFFFDFF49
:101F4A00012400FAFFFCFF014000F6FFF8FF013D03
:101F5A0000F9FFF6FF013600FCFFF6FF013C00FF27
:101F6A00FFF4FF013C000100F4FF0136000400F613
:101F7A00FF013D000700F6FF0140000A00F8FF01DB
:101F8A0024000600FCFF0122000600FDFF015400A8
:101F9A001000FBFF015B001200FDFF016900150044
:101FAA00FFFF016400140001000156001100030044
:101FBA00014F000F00050001260007000300012061
:101FCA0000050004000143000A0009000139000766
:101FDA00000900013B0004000B0001370001000B5F
:101FEA0000013C00FFFF0C00013600FCFF0A000163
:101FFA003D00F9FF0A00014000F6FF080001200039
:10200A00FBFF0400012600F9FF0300014F00F1FF66
:10201A000500015B00EEFF0300016400ECFF010014
:10202A00010000000000000201000000000001326F
:10203A00000000000001BC01B0FF02FF0200000026
:10204A000000000132000000000001AC00DEFFFBCE
:10205A00FF014300FDFF0D00013C00FFFF0C0001E2
:10206A0028000100080001230001000700012400E4
:10207A0002000700011D000300050001190003000A
:10208A0004000120000500040001190004000300F7
:10209A00011D0005000300012300070001000133B0
:1020AA00000A0002000191001D000100019402844F
:1020BA00000000017300000017000196001E0000D6
:1020CA00000173000000E9FF011D01390000000151
:1020DA00C9001700DFFF019001B0FF000001A00056
:1020EA000000E0FF019600E2FF000001A0000000EE
:1020FA002000019E027AFF0000014600F2FF000064
:10210A00012300F9FFFFFF011D00FBFFFDFF011581
:10211A0000FDFFFDFF011B00FEFFFBFF011E00FF8C
:10212A00FFFAFF0147000200F2FF01000000000071
:10213A00000201000000000001320000000000015E
:10214A0058075AFF5C040200000000000001320038
:10215A000000000001C701A8FFE9FF0141000000DB
:10216A00F3FF015C014400F1FF014C00F1FFFEFFA7
:10217A00011001CBFFF4FF0141000000F3FF01C78A
:10218A00015800E9FF013C0000000C00010701CDE5
:10219A00FF0D00015700EFFF040001570011000472
:1021AA000001050133000B00013C0000000C000196
:1021BA000601CDFF0C00016100EDFF040001610082
:1021CA001300040001060133000C00014100000065
:1021DA000D000100000000000002010000000000E4
:1021EA000132000000000001FF00A8FF83FF020087
:1021FA0000000000000132000000000001C6015882
:10220A000016000141000000F3FF010501CDFFF5B2
:10221A00FF016200EDFFFBFF0161001300FCFF01FB
:10222A0005013300F5FF0141000000F3FF0105013C
:10223A00CDFFF5FF015700EFFFFCFF01570011002A
:10224A00FCFF0107013300F3FF013C000000F4FF2B
:10225A0001C701A8FF170001410000000D0001108D
:10226A000135000C00014C000F000300015C01BCA9
:10227A00FF0F0001410000000D00020100000000F4
:10228A00000132000000000001AC00000099FF02CA
:10229A000000000000000132000000000001C60139
:1022AA0058001600013C000000F4FF010601CDFFB2
:1022BA00F4FF016200EDFFFBFF0160001300FDFF68
:1022CA000106013300F4FF0141000000F3FF01059C
:1022DA0001CDFFF5FF015700EFFFFCFF0157001189
:1022EA0000FCFF0107013300F3FF013C000000F48A
:1022FA00FF01C701A8FF170001410000000D0001FE
:10230A00100135000C00014C000F000300015C01B4
:10231A00BCFF0F0001410000000D00020100000097
:10232A00000001320000000000019B000000A3FF32
:10233A000200000000000001320000000000015508
:10234A0000110000000146000000F2FF015500EFF5
:10235A00FF000001460000000E000201000000001C
:10236A0000013200000000000197001C00AAFF02D1
:10237A0000000000000001320000000000014100DE
:10238A00FFFFF3FF012400F9FF0200012000FAFF1A
:10239A000200011900FCFF0300012000FBFF0400FA
:1023AA00011D00FDFF0500011B00FEFF0500011BCA
:1023BA0000FEFF0500011E000000060001280001C2
:1023CA00000800012400020007000124000400069E
:1023DA000001230005000500012400060004000195
:1023EA002B0008000300012E000900020001320040
:1023FA000A0000000137000B000000012E0009004E
:10240A00FEFF012B000800FDFF0128000700FCFF6A
:10241A000123000500FBFF0124000400FAFF012646
:10242A00000300F9FF0123000000F9FF0123000067
:10243A0000F9FF012200FDFFFAFF012200FDFFFA69
:10244A00FF012700FAFFFBFF012400FAFFFCFF014E
:10245A002B00F8FFFDFF012E00F7FFFEFF013700FA
:10246A00F5FFFFFF011500FCFF0100011301000049
:10247A003700012300F9FFFFFF012000FAFFFEFFEA
:10248A00011B00FBFFFEFF011600FCFFFEFF011906
:10249A0000FDFFFCFF011500FDFFFDFF011500FF18
:1024AA00FFFCFF011900FFFFFBFF011E000100FAFC
:1024BA00FF0120000400FBFF0123000500FBFF01D0
:1024CA002B000800FDFF01000000000000020100CF
:1024DA000000000001320000000000015000190055
:1024EA002900020000000000000132000000000084
:1024FA0001CD000000D7FF012D00090001000126CF
:10250A000007000300011C00040004000115000379
:10251A000003000116000200040001190000000572
:10252A000001140000000400011600FEFF0400016F
:10253A001200FEFF0300011500FDFF030001190050
:10254A00FCFF0300011600FCFF0200011900FBFF5B
:10255A000100011900FBFF0100010000000000005A
:10256A000201000000000001320000000000019793
:10257A0000C4FFBCFF02000000000000013200009E
:10258A00000000013E00FDFFF4FF011900FBFFFF00
:10259A00FF011900FCFFFDFF011D00FDFFFBFF010C
:1025AA002900FEFFF8FF0124000200F9FF012200C2
:1025BA000300FAFF0120000500FCFF0120000600CD
:1025CA00FEFF0123000700FFFF0141000D0000008C
:1025DA00012400FAFF0400011D00FDFF0500011B94
:1025EA0000FEFF0500011E00FFFF06000123000197
:1025FA000007000124000200070001200004000572
:10260A00000127000600050001260007000300015B
:10261A002B000800030001280008000100012D001A
:10262A0009000100013C000C00FFFF0139000B000A
:10263A00FDFF0138000A00FBFF012E000700FAFF28
:10264A000116000200FCFF0116000200FCFF011542
:10265A00000100FCFF0119000000FBFF011E000041
:10266A0000FAFF012200FDFFFAFF012000FCFFFB38
:10267A00FF012300FBFFFBFF0132000A00000001FB
:10268A0037000000F5FF017C01B4FF0000015A0089
:10269A00EEFF0100011E00FAFF0100011900FBFF15
:1026AA000100012F00F8FF0500012E00FAFF0700C4
:1026BA00012D00FCFF0800013200FFFF0A00012380
:1026CA00000100070001190001000500011B0002BA
:1026DA00000500011D0003000500011900040003A4
:1026EA0000011D0005000300011E00060001000193
:1026FA0023000700000001000000000000020100A2
:10270A000000000001320000000000015A003500FC
:10271A00F6FF020000000000000132000000000085
:10272A00012800F8FF0000012300F9FFFFFF012044
:10273A0000FAFFFEFF011D00FBFFFDFF011500FD72
:10274A00FFFDFF011500FDFFFDFF011500FFFFFC66
:10275A00FF011500FFFFFCFF0115000100FCFF014E
:10276A0015000100FCFF0115000300FDFF0119001F
:10277A000300FCFF011B000500FEFF01200006000C
:10278A00FEFF011E000600FFFF01280008000000EE
:10279A0001280008000000011E00060001000120B7
:1027AA000006000200011D000500030001150003D8
:1027BA0000030001150003000300011500010004D5
:1027CA000001150001000400011500FFFF040001CB
:1027DA001500FFFF0400011500FDFF0300011500AD
:1027EA00FDFF0300011D00FBFF0300011B00FBFFAF
:1027FA000200012300F9FF0100012300F9FF000094
:10280A000100000000000002010000000000013287
:10281A000000000000019100CBFFBBFF0200000096
:10282A0000000001320000000000013E00FDFFF43C
:10283A00FF011900FBFFFFFF011900FCFFFDFF016B
:10284A002200FDFFFAFF012400FEFFF9FF01290023
:10285A000200F8FF011D000300FBFF012000050034
:10286A00FCFF0122000600FDFF0123000700000013
:10287A000141000D00FFFF012700FAFF0500011DBD
:10288A0000FDFF0500011B00FEFF0500011E00FF01
:10289A00FF060001230001000700012000020006D4
:1028AA0000012400040006000124000600040001BF
:1028BA00280007000400012B00080003000128007B
:1028CA0008000100012D0009000100013C000C0074
:1028DA00FFFF0139000B00FDFF0138000A00FBFF72
:1028EA00012E000700FAFF0116000200FCFF011684
:1028FA00000200FCFF0115000100FCFF01190000A5
:10290A0000FBFF011E000000FAFF012200FDFFFA92
:10291A00FF012000FCFFFBFF012300FBFFFBFF017F
:10292A0032000A0000000137000000F5FF017C01B7
:10293A00B4FF0000015A00EEFF0100011E00FAFF79
:10294A000100011900FBFF0100012F00F8FF05003B
:10295A00012A00FAFF0600013100FCFF09000132DA
:10296A0000FFFF0A00011E0001000600011E00010F
:10297A00000600011B000200050001190003000403
:10298A0000011C0004000400011B000500020001F4
:10299A0020000600020001230007000000010000D9
:1029AA0000000000020100000000000132000000E7
:1029BA000000015A003500F6FF0200000000000086
:1029CA0001320000000000012800F8FF0000012485
:1029DA0000F9FFFEFF011E00FAFFFFFF011D00FBC9
:1029EA00FFFDFF011500FDFFFDFF011500FDFFFDC5
:1029FA00FF011500FFFFFCFF011500FFFFFCFF01AF
:102A0A0015000100FCFF0115000100FCFF0119007F
:102A1A000300FCFF0115000300FDFF011B00050078
:102A2A00FEFF0120000600FEFF011E000600FFFF58
:102A3A000128000800FFFF01280008000100011E0C
:102A4A00000600010001200006000200011B00052B
:102A5A00000200011900030004000115000300032D
:102A6A000001150001000400011500010004000125
:102A7A001500FFFF0400011500FFFF040001150007
:102A8A00FDFF0300011500FDFF0300011D00FBFF10
:102A9A000300011900FBFF0100012400F9FF0200F5
:102AAA00012300F9FF0000010000000000000201FC
:102ABA00000000000001320000000000016F00F772
:102ACA00FFBEFF020000000000000132000000000B
:102ADA0000014B000F00000001C3000000D9FF01F4
:102AEA004B00F1FF000001C30000002700020100B3
:102AFA000000000001320000000000017B00DBFF43
:102B0A00C0FF0200000000000001320000000000C7
:102B1A0001370000000B000162027A000000013C4C
:102B2A00000000F4FF01DC00D4FF000001240006CD
:102B3A0000FCFF011D000300FBFF011D000300FB59
:102B4A00FF011E000000FAFF0123000000F9FF0147
:102B5A002200FDFFFAFF012400FCFFFAFF0120001A
:102B6A00FBFFFCFF012800F9FFFCFF012900F8FF29
:102B7A00FEFF012900F8FFFEFF012D00F7FFFFFF0E
:102B8A00013700F5FF0100013300F6FF0200012BB7
:102B9A0000F8FF0300012800F9FF0400012300FBED
:102BAA00FF0500012000FCFF0500012000FEFF06D2
:102BBA0000011E00FFFF0600011E000100060001C1
:102BCA002000020006000120000400050001240084
:102BDA0006000400013700F5FF00000201000000B2
:102BEA00000001320000000000014B002D0000002F
:102BFA00020000000000000132000000000001464F
:102C0A0000F2FFFFFF012F00F7FFFDFF011D00FB90
:102C1A00FFFDFF011C00FCFFFCFF011600FEFFFC8C
:102C2A00FF011900FFFFFBFF0115000100FCFF0176
:102C3A0010000100FDFF0119000300FCFF0119004B
:102C4A000400FDFF011B000500FEFF011B0005003B
:102C5A00FEFF0123000700FFFF0128000800FFFF15
:102C6A000128000800010001230007000100011EDD
:102C7A000006000100011D00050003000115000304
:102C8A0000030001150003000300011600020004FE
:102C9A0000011400000004000114000000040001F7
:102CAA001200FEFF0300011900FDFF0400011500D8
:102CBA00FDFF0300011D00FBFF0300011E00FAFFD8
:102CCA000100012400F9FF0200012300F9FF0000BE
:102CDA0001000000000000020100000000000132B3
:102CEA000000000000016900FFFFC1FF02000000B0
:102CFA0000000001320000000000013C000C00FF4F
:102D0A00FF0133000A00FEFF012D000800FCFF014D
:102D1A002B000700FBFF0120000400FBFF011D0040
:102D2A000300FBFF0120000200FAFF01230000005C
:102D3A00F9FF0123000000F9FF012600FDFFF9FF5A
:102D4A00011D00FDFFFBFF012A00FAFFFAFF012423
:102D5A0000FAFFFCFF012B00F8FFFDFF012E00F730
:102D6A00FFFEFF013200F6FF0000014B00F1FF01F8
:102D7A0000011E00FAFF0100011B00FBFF02000117
:102D8A003300F7FF0500013100F9FF0700013100A8
:102D9A00FCFF0900012D00FFFF09000128000100C6
:102DAA0008000120000200060001240004000600B9
:102DBA000123000500050001240006000400012B80
:102DCA0000080003000133000A0002000132000A71
:102DDA0000010001000000000000020100000000E4
:102DEA0000013200000000000116000000F3FF029B
:102DFA00000000000000013200000000000128006D
:102E0A00F8FF0000012400F9FFFEFF011E00FAFF8F
:102E1A00FFFF011900FCFFFDFF011900FCFFFDFF88
:102E2A00011900FDFFFCFF011500FFFFFCFF01195E
:102E3A0000FFFFFBFF0115000100FCFF0115000167
:102E4A0000FCFF0119000300FCFF0119000400FD4A
:102E5A00FF011D000500FDFF011B000500FEFF012B
:102E6A0028000800FFFF01280008000000012300D5
:102E7A0007000000012300070001000120000600EE
:102E8A000200011D000500030001150003000300F4
:102E9A0001190003000400011500010004000115D6
:102EAA000001000400011900FFFF0500011500FFE1
:102EBA00FF0400011900FDFF0400011500FDFF03D6
:102ECA0000011D00FBFF0300011E00FAFF010001C3
:102EDA002400F9FF0200012800F8FF0000010000A9
:102EEA0000000000020100000000000132000000A2
:102EFA00000001AB00E1FF9EFF020000000000009D
:102F0A0001320000000000014200F3FFFEFF012D24
:102F1A0000FFFF0900011E0000000600011B00025D
:102F2A000005000115000300030001160004000259
:102F3A0000012300070001000137000B0001000116
:102F4A00FF0033000000012D0000000900013700D6
:102F5A000B000000012D000000F7FF016E001600B3
:102F6A000000014F000900F3FF019B00E1FF000090
:102F7A00013C000000F4FF013700F5FF0000013CAE
:102F8A000000000C00010401CCFF0000012800F839
:102F9A00FF0000011500FDFFFDFF011500FFFFFC0A
:102FAA00FF0119000000FBFF010000000000000201
:102FBA0001000000000001320000000000012200B0
:102FCA00F3FFF0FF020000000000000132000000E1
:102FDA000000015500110000000146000000F2FF48
:102FEA00015500EFFF000001460000000E0002013B
:102FFA0000000000000132000000000001960020DD
:10300A0000ACFF02000000000000013200000000D6
:10301A0000013D00FEFFF4FF012300F9FF0100015A
:10302A002000FAFF0200012200FAFF0300011C003F
:10303A00FCFF0400011C00FCFF0400011D00FDFF51
:10304A000500012000FEFF0600011900000005002E
:10305A0001280001000800012000020006000124E6
:10306A0000040006000123000500050001240006F3
:10307A00000400012B0008000300012D00090001D3
:10308A00000137000B0001000141000D00FFFF01A4
:10309A003E000C00FDFF011B000500FEFF011900A8
:1030AA000400FDFF0119000400FDFF0119000300DF
:1030BA00FCFF012D000400F8FF0132000100F6FFB9
:1030CA000119000000FBFF011E00FFFFFAFF0119B2
:1030DA0000FDFFFCFF011900FDFFFCFF011C00FCC5
:1030EA00FFFCFF011D00FBFFFDFF011B00FBFFFEB4
:1030FA00FF012300F9FFFFFF013D00FEFF0C000165
:10310A0029000800020001240006000400011D0035
:10311A0003000500011E0001000600011400000062
:10312A000400011600FEFF0400011900FDFF04005F
:10313A00011500FDFF0300011D00FBFF0300012034
:10314A0000FAFF0200012300F9FF0100012800F83C
:10315A00FF0000012800F8FF0000012300F9FFFF2B
:10316A00FF012000FAFFFEFF011D00FBFFFDFF012A
:10317A001500FDFFFDFF011500FDFFFDFF01150014
:10318A00FFFFFCFF011500FFFFFCFF012400020006
:10319A00F9FF0124000400FAFF0112000300FEFFF8
:1031AA000116000400FEFF012E000900FEFF0100C7
:1031BA0000000000000201000000000001320000CF
:1031CA000000000124000C00EEFF020000000000D5
:1031DA000001320000000000013C000C00FFFF016A
:1031EA0033000A00FEFF012D000800FCFF012B003E
:1031FA000700FBFF0120000400FBFF011D00030084
:10320A00FBFF0120000200FAFF0123000000F9FF82
:10321A000123000000F9FF012600FDFFF9FF01224A
:10322A0000FDFFFAFF012700FAFFFBFF012400FA65
:10323A00FFFCFF012B00F8FFFDFF012E00F7FFFE48
:10324A00FF013200F6FF0000014B00F1FF0100010F
:10325A001E00FAFF0100011B00FBFF020001330000
:10326A00F7FF0500013100F9FF0700013100FCFFFB
:10327A000900012D00FFFF090001230001000700DA
:10328A0001240002000700012400040006000123B3
:10329A00000500050001240006000400012B0008B7
:1032AA000003000133000A0002000132000A000193
:1032BA0000010000000000000201000000000001FF
:1032CA003200000000000116000000F3FF020000B7
:1032DA000000000001320000000000012800F8FF91
:1032EA00FFFF012300F9FFFFFF012000FAFFFEFFA5
:1032FA00011600FCFFFEFF011C00FCFFFCFF01158C
:10330A0000FDFFFDFF011500FFFFFCFF011900FF93
:10331A00FFFBFF0115000100FCFF0115000100FC85
:10332A00FF0119000300FCFF0119000400FDFF0161
:10333A001D000500FDFF011B000500FEFF0128001E
:10334A000800FFFF0128000800FFFF012300070013
:10335A00010001230007000100012000060002000D
:10336A00011D0005000300011500030003000119F7
:10337A00000300040001150001000400011500010A
:10338A00000400011900FFFF0500011500FFFF04FA
:10339A0000011500FDFF0300011900FDFF040001F3
:1033AA001B00FBFF0200012000FAFF0200012300BC
:1033BA00F9FF0100012800F8FF01000100000000E8
:1033CA0000000201000000000001320000000000BD
:1033DA00018B00D4FFB9FF02000000000000013297
:1033EA00000000000001B801580000000137000089
:1033FA0000F5FF013C00F4FF00000124000600FC78
:10340A00FF0124000400FAFF0122000300FAFF0171
:10341A0023000100F9FF012300FFFFF9FF01220049
:10342A00FDFFFAFF012300FBFFFBFF012000FAFF6B
:10343A00FEFF012B000700FBFF0127000500FAFF32
:10344A000120000200FAFF011E000100FAFF011923
:10345A00000000FBFF011900FFFFFBFF011900FD3F
:10346A00FFFCFF011500FDFFFDFF011900FCFFFD38
:10347A00FF011B00FBFFFEFF011E00FAFFFFFF0119
:10348A002300F9FF0000013101C3FF0000013C00E5
:10349A0000000C0001180138000000012300070099
:1034AA000100011E000600010001100003000100D6
:1034BA0001150003000300011600020004000114B4
:1034CA000000000400010F0000000300011500FFC6
:1034DA00FF0400011200FEFF0300011200FDFF02BB
:1034EA0000011500FDFF0300011900FBFF010001A7
:1034FA003D00F4FF020001FF00CDFF0000013C0087
:10350A0000000C00011D0139000000012D00090016
:10351A00010001200006000200011200030002005F
:10352A00010B0001000200011E0001000600011942
:10353A000000000500011D00FDFF0500011C00FC44
:10354A00FF0400012000FAFF0200012900F8FF022F
:10355A0000013200F6FF000001E600D2FF00000180
:10356A00410000000D0002010000000000013200CD
:10357A000000000001ED05CB0089FC0200000000FC
:10358A0000000132000000000001A400F5FFE1FF85
:10359A0001A100F7FFE1FF012201F1FFC8FF0105C8
:1035AA0001F5FFCDFF01DA00F9FFD5FF01B100FBFC
:1035BA00FFDDFF018700FEFFE5FF016E00FEFFEA67
:1035CA00FF020100000000000132000000000001BB
:1035DA00F8013E002801020000000000000132004C
:1035EA000000000001800280FF00000201000000CC
:1035FA00000001320000000000010C02EC0030FF64
:10360A00020000000000000132000000000001ABCF
:10361A0000F7FF2100019500F6FF1C00019600F556
:10362A00FF1C00019D00F4FF1D0001C000F0FF23F4
:10363A000001CE00ECFF2400016300F6FF11000137
:10364A006100F5FF1000016400F4FF100001600042
:10365A00F4FF0F00012A00FAFF0600012700FAFF13
:10366A000500012400FAFF0400012000FAFF02000D
:10367A00012000FAFF0200011E00FAFF0000013CCF
:10368A0000F4FF0000013D00F4FFFEFF014200F3D9
:10369A00FFFEFF014200F3FFFEFF014600F2FF00BA
:1036AA0000013700F5FF0000012D00F7FFFFFF01C1
:1036BA002B00F8FFFDFF012000FBFFFCFF010E00BD
:1036CA00FEFFFEFF010F000000FDFF011000FFFFDB
:1036DA00FDFF0115000100FCFF012D000400F8FFA9
:1036EA000140000800F6FF0120000400FBFF01244E
:1036FA00000200F9FF012E000200F7FF012D000071
:10370A0000F7FF012D00FFFFF7FF012E00FEFFF774
:10371A00FF012800FCFFF9FF012700FBFFFAFF0267
:10372A0001000000000001320000000000019E02BA
:10373A00FF00C9FE02000000000000013200000084
:10374A000000011E0006000000011500040001002F
:10375A000112000300020001160002000400011B0E
:10376A00000200050001190001000500014600FFE2
:10377A00FF0E00014C00FEFF0F00014C00FDFF0F81
:10378A0000018E00FBFF1C00018F00FAFF1C0002E3
:10379A0001000000000001320000000000012902BF
:1037AA00E9FEB4000200000000000001320000003F
:1037BA000000015D00EEFFFBFF014700F2FFFEFF84
:1037CA00013700F5FF0000012F00F7FF0300012772
:1037DA0000FAFF0500012700FBFF0600012600FD95
:1037EA00FF0700012E00FEFF0900015600FDFF1130
:1037FA0000012D00FFFF0900012900FEFF0800015A
:10380A002600FDFF0700012000FCFF05000124003F
:10381A00FAFF0400012800F8FF0100018A01EFFF06
:10382A00B3FF011E000000FAFF0119000100FBFFAF
:10383A000136000400F6FF013A000600F6FF0136E1
:10384A00000600F7FF0160000C00F1FF01280004E8
:10385A0000F9FF0120000200FAFF010B00FFFFFE42
:10386A00FF011000FFFFFDFF012E00F9FFFAFF0123
:10387A008A00EBFFEEFF014B00F4FFF7FF014A005D
:10388A00F6FFF5FF014300F7FFF6FF011D00FDFFFC
:10389A00FBFF011B00FEFFFBFF014B01F3FFBFFF14
:1038AA00010401F6FFCDFF0119000500000001190E
:1038BA0000050001000116000400020001160004C0
:1038CA0000020001350007000800013A0006000A5C
:1038DA00000194000C001B00015E000800110001A9
:1038EA00600009001100011D0003000500011C0011
:1038FA00040004000144000B000800014A000D0006
:10390A000700014A000E0005000147000E000200F0
:10391A00012300070000000123000700FFFF012028
:10392A00000600FEFF011D000500FDFF0120000545
:10393A0000FCFF0124000400FAFF0131000400F733
:10394A00FF013E000300F4FF0141000100F3FF0103
:10395A0046000000F2FF02010000000000013200F0
:10396A0000000000010A000600000002000000003A
:10397A00000001320000000000016600140004008B
:10398A0001510010000200013C000C00000001334C
:10399A00000A00FEFF012D000800FCFF01320008AA
:1039AA0000FAFF0135000800F9FF0143000900F69B
:1039BA00FF014E000A00F4FF014E000A00F4FF0165
:1039CA009E001200E6FF0138012100CBFF015500DD
:1039DA000800F1FF015C000900F0FF01BE000F00C2
:1039EA00DDFF01BF000D00DCFF01B1000A00DEFFB0
:1039FA0001F7000C00D0FF01F5000A00D0FF015AC0
:103A0A00000100EEFF011E00FFFFFAFF011500FF93
:103A1A00FFFCFF011200FEFFFDFF011200FDFFFE89
:103A2A00FF011000FDFFFFFF011000FDFF01000173
:103A3A002E00F7FF0200012F00F7FF0300013900F3
:103A4A00F5FF0300013200F6FF0100013200F6FF24
:103A5A000000012E00F7FF0200013100F7FF040009
:103A6A00013600F7FF0600013900F7FF0700013CA5
:103A7A0000F8FF0900014300F7FF0A00014400F8BB
:103A8A00FF0B00018900F1FF1700019200F1FF19F5
:103A9A0000018B00F2FF1800018000F3FF160002FC
:103AAA0001000000000001320000000000019B013B
:103ABA00C4FFEF0002000000000000013200000015
:103ACA000000015F00EDFF0000015100F0FFFEFF62
:103ADA00013D00F4FFFEFF013100F7FFFCFF011575
:103AEA0000FDFFFDFF011500FDFFFDFF011600FEB1
:103AFA00FFFCFF011500FFFFFCFF013C00FFFFF484
:103B0A00FF014C000200F1FF0156000300EFFF0124
:103B1A0061000400EDFF0162000500EDFF01650090
:103B2A000700EDFF0165000900EEFF013200060003
:103B3A00F8FF0132000600F8FF0135000700F8FF20
:103B4A000131000700F9FF0132000800FAFF0133D2
:103B5A00000900FBFF020100000000000132000022
:103B6A00000000011D00F1FF090002000000000032
:103B7A00000132000000000001FF00F6FFCEFF0145
:103B8A005601F2FFBDFF02010000000000013200F1
:103B9A00000000000186023D01DF00020000000073
:103BAA00000001320000000000019300F7FFE4FF6B
:103BBA00018200F9FFE7FF010701F3FFCDFF019F33
:103BCA0000F9FFE1FF01C500FAFFD9FF01D400FAAD
:103BDA00FFD6FF01DD00FCFFD4FF02010000000058
:103BEA000001320000000000018F01F7FFEF000220
:103BFA0000000000000001320000000000017F0008
:103C0A000B00E9FF014600F2FFFFFF017D00F6FF0E
:103C1A0017000141000D0001000100000000000032
:103C2A00020100000000000132000000000001173C
:103C3A0000F2FF0000020000000000000132000054
:103C4A00000000016A00FDFFEBFF0172000900EBB2
:103C5A00FF015D00050012000201000000000001E2
:103C6A00320000000000012700F4FF1400020000E7
:103C7A000000000001320000000000014F01BDFFFA
:103C8A00FFFF0201000000000001320000000000F6
:103C9A00016E004000EFFF02000000000000013248
:103CAA000000000000010901CBFF00000201000032
:103CBA0000000001320000000000016F003F00EB2D
:103CCA00FF020000000000000132000000000001B5
:103CDA00FA00CEFF000002010000000000013200DD
:103CEA00000000000179003A002C000200000000E8
:103CFA0000000132000000000001F2021D009400E1
:103D0A00020100000000000132000000000001046E
:103D1A0001D5FF6AFF020000000000000132000026
:103D2A0000000001F7021D009500020100000000DA
:103D3A000001320000000000011D01FCFF55FF02D6
:103D4A000000000000000132000000000001BF0274
:103D5A001B008A000201000000000001320000007E
:103D6A000000012B0002001A0002000000000000FF
:103D7A0001320000000000012800FFFF08000124B2
:103D8A0000FEFF0700010700FFFF0100010700FF17
:103D9A00FF0100010E00FEFFFEFF012800FCFFF9F3
:103DAA00FF020100000000000132000000000001D3
:103DBA001800F2FFFEFF02000000000000013200BE
:103DCA0000000000012400020007000115000300A2
:103DDA000300010B00020001000141000D00000078
:103DEA00020100000000000132000000000001EFA3
:103DFA00007AFF33000200000000000001320000D8
:103E0A000000000126000700FDFF0126000700FD53
:103E1A00FF0132000800FAFF012E000700FAFF0135
:103E2A0035000700F8FF0136000600F7FF013600EB
:103E3A000600F7FF013A000600F6FF013800050008
:103E4A00F6FF013B000400F5FF0139000300F5FF0E
:103E5A000133000200F6FF0137000100F5FF012DD2
:103E6A00000000F7FF013200FFFFF6FF012D00FC02
:103E7A00FFF8FF012600FDFFF9FF012300FBFFFB0E
:103E8A00FF011D00FBFFFDFF012200FAFFFDFF01FC
:103E9A001E00FAFFFFFF011E00FAFFFFFF011E00CE
:103EAA00FAFF0100012300F9FF0100013F00F4FFBE
:103EBA000400014300F4FF0600013900F7FF070080
:103ECA00013500F8FF07000201000000000001327E
:103EDA00000000000001F30085003C000200000021
:103EEA000000000132000000000001D600D7FFF4F4
:103EFA00FF02010000000000013200000000000182
:103F0A0040002500F5FF0200000000000001320019
:103F1A000000000001C100DBFF0B000201000000ED
:103F2A00000001320000000000016B003F000C009D
:103F3A000200000000000001320000000000014001
:103F4A0001400000000136013E0000000176027EB9
:103F5A0000FDFF014C000F00FEFF012D000900FFCC
:103F6A00FF0110000300FFFF010B000100FEFF012B
:103F7A0010000100FDFF0119000000FBFF012800ED
:103F8A00FFFFF8FF010B00FFFFFEFF010B00FEFF22
:103F9A00FFFF012D00F7FFFFFF015000F0FFFFFFB9
:103FAA00017B0281FF0100013B01C1FF01000140C9
:103FBA0001C0FF0300010B00FEFF0100010E00FE1D
:103FCA00FF0200011500FFFF0400011900000005AF
:103FDA00000119000100050001150001000400019B
:103FEA00120002000300011000030001000100009A
:103FFA000000000002010000000000013200000081
:10400A0000000147001500DBFF020000000000006D
:10401A000132000000000001BA00EFFFDFFF015982
:10402A0000F8FFF0FF015E00F8FFEFFF0201000059
:10403A0000000001320000000000016D00EBFFC229
:10404A00FF02000000000000013200000000000131
:10405A006200FBFFEDFF016000FEFFEDFF01600063
:10406A00FEFFEDFF015F00FFFFEDFF01C30001004E
:10407A00D9FF01B9000100DBFF02010000000000C6
:10408A0001320000000000015B014300C50002008C
:10409A0000000000000132000000000001C800D842
:1040AA00FFFFFF02010000000000013200000000D3
:1040BA0000015002EBFE22FF020000000000000196
:1040CA00320000000000012800080001000126005B
:1040DA000700030001270006000500012300050070
:1040EA00050001550008000F0001620008001200D7
:1040FA0001B6000D0022000201000000000001329A
:10410A00000000000001F20156001E01020000003A
:10411A0000000001320000000000010C01E8FF303D
:10412A00000201000000000001320000000000014E
:10413A0054002100DAFF02000000000000013200F2
:10414A000000000001FF00EAFF2E0002010000004B
:10415A00000001320000000000019B00B4FFCAFF0A
:10416A0002000000000000013200000000000111FE
:10417A0001E6FF30000201000000000001320000E9
:10418A0000000001EC008A001F000200000000008D
:10419A000001320000000000011C01E9FF340002A6
:1041AA0001000000000001320000000000017C0054
:1041BA00E6FFBAFF02000000000000013200000022
:1041CA00000001C201A6FF01000201000000000078
:1041DA0001320000000000019C005C00F0FF0200B8
:1041EA0000000000000132000000000001C701A524
:1041FA00FF0200020100000000000132000000007E
:10420A000001E60068005B000200000000000001F7
:10421A0032000000000001BD01A7FF0100020100F9
:10422A000000000001320000000000019400590063
:10423A00FFFF020000000000000132000000000041
:10424A00018C01F2FFB2FF020100000000000132FE
:10425A000000000000017C00190046000200000076
:10426A0000000001320000000000018701F2FFB3E4
:10427A00FF020100000000000132000000000001FE
:10428A00CB00AAFF56000200000000000001320025
:10429A0000000000018E01F0FFB2FF0201000000E1
:1042AA0000000132000000000001DD007400C0FFC0
:1042BA00020000000000000132000000000001BD01
:1042CA0001A7FF0100020100000000000132000006
:1042DA00000000019B004B003700020000000000B4
:1042EA000001320000000000014100F5FF07000252
:1042FA000100000000000132000000000001170068
:10430A000000F2FF0200000000000001320000007D
:10431A000000014600FFFF0E00020100000000003D
:10432A00013200000000000119000100F1FF020043
:10433A000000000000013200000000000144000BF0
:10434A000008000201000000000001320000000025
:10435A000001B60093FF0100020000000000000106
:10436A0032000000000001350007000800020100C9
:10437A000000000001320000000000011B000200E2
:10438A00F0FF0200000000000001320000000000FF
:10439A00013900F7FF0700020100000000000132A6
:1043AA00000000000001F2007B004D000200000046
:1043BA0000000001320000000000014400F5FF087F
:1043CA0000020100000000000132000000000001AC
:1043DA00A000A0FFF9FF0200000000000001320067
:1043EA0000000000018A01EFFFB3FF020100000094
:1043FA00000001320000000000015C001A00CFFF3B
:10440A000200000000000001320000000000011359
:10441A0001E7FF3100020100000000000132000044
:10442A00000000016D002200C8FF02000000000029
:10443A000001320000000000013900F7FF07000206
:10444A000100000000000132000000000001A40089
:10445A006200F9FF020000000000000132000000C3
:10446A000000014E0007000E0002010000000000DB
:10447A000132000000000001D40086FF240002007F
:10448A0000000000000132000000000001410000AD
:10449A00000D0002010000000000013200000000CF
:1044AA000001770008004700020000000000000138
:1044BA00320000000000013100070007000201007D
:1044CA000000000001320000000000014302620007
:1044DA00B3FE0200000000000001320000000000EC
:1044EA00015101F2FFBEFF0201000000000001328B
:1044FA000000000000016B0019003B0002000000F0
:10450A0000000001320000000000014B01F3FFBF70
:10451A00FF0201000000000001320000000000015B
:10452A0045002300160002000000000000013200CE
:10453A0000000000014B01F3FFBFFF020100000071
:10454A0000000132000000000001FD009EFF74001F
:10455A0002000000000000013200000000000155C6
:10456A0001F3FFBDFF02010000000000013200005C
:10457A000000000118000300F2FF02000000000022
:10458A00000132000000000001FB001A00D5FF0202
:10459A0001000000000001320000000000017B0061
:1045AA003000380002000000000000013200000064
:1045BA000000018101B3FF010002010000000000B8
:1045CA00013200000000000186004F00F2FF0200E5
:1045DA00000000000001320000000000017C01B46C
:1045EA00FF0000020100000000000132000000008C
:1045FA0000017F004C0000000200000000000001E2
:10460A0032000000000001F4001700D5FF0201008B
:10461A000000000001320000000000015600F3FF14
:10462A003200020000000000000132000000000019
:10463A0001ED001600D6FF02010000000000013261
:10464A00000000000001C400ECFF7400020000003A
:10465A0000000001320000000000018101B3FF00E8
:10466A000002010000000000013200000000000109
:10467A00FD00580084FF0200000000000001320023
:10468A0000000000016D01B7FF00000201000000F8
:10469A0000000132000000000001E400490074003B
:1046AA00020000000000000132000000000001EDDD
:1046BA00001600D6FF0201000000000001320000CF
:1046CA00000000015B00D3FFE1FF020000000000D0
:1046DA000001320000000000013D000A000700024C
:1046EA000100000000000132000000000001160075
:1046FA00F4FF060002000000000000013200000082
:10470A0000000143000C00FAFF0201000000000053
:10471A0001320000000000011700F4FF0700020048
:10472A000000000000013200000000000147000202
:10473A0000F2FF0201000000000001320000000048
:10474A0000018500B1FF0D00020000000000000119
:10475A00320000000000013E000300F4FF020100E5
:10476A000000000001320000000000017F00040088
:10477A004C000200000000000001320000000000AE
:10478A00015001F3FFBEFF020100000000000132E8
:10479A0000000000000102000000FFFF020000000C
:1047AA00000000013200000000000143000900F689
:1047BA00FF020100000000000132000000000001B9
:1047CA001600F7FF0A000200000000000001320094
:1047DA00000000000124000600040002010000009D
:1047EA00000001320000000000010D00FAFFFBFF8B
:1047FA000200000000000001320000000000010277
:10480A00011B00D4FF020100000000000132000079
:10481A000000000102000000FFFF0200000000008B
:10482A0000013200000000000135000800F9FF0213
:10483A000100000000000132000000000001CB006E
:10484A00EBFF7800020000000000000132000000C7
:10485A000000012000050004000201000000000021
:10486A00013200000000000182004E000000020038
:10487A000000000000013200000000000141000BAE
:10488A0000F9FF02010000000000013200000000F0
:10489A000001C30001008BFF0200000000000001BC
:1048AA00320000000000013900080008000201007F
:1048BA00000000000132000000000001AF0E3200CB
:1048CA00CF080201000000000001320000000000D1
:1048DA000201000000000000000000000000E9CF13
:1048EA00E4FFEACFE4FFE6528EEC34F0E6529EA0F3
:1048FA0001D29E90FE0ECF6E3D0ECE6E91C4B2F4E2
:10490A000401B36B010EB46FB7EC37F014E0D88032
:10491A00000E9255000E9355190E9455000E95559A
:10492A0005E2926B936B946B956B05D09207000E20
:10493A00935B945B955BB7EC37F001E0B46B780559
:10494A0004E0050E785D01E0A3D09F5103E1A05178
:10495A0001E128D1050E785D1FE19F5146E0BCECCC
:10496A0037F001E19F6BD7EC37F07CAF02D0800EB5
:10497A007C2794EC36F0A4AF02D0E0EC37F0E9ECF7
:10498A0037F080AF02D0800E8027A5EC36F0A8AFB2
:10499A002CD0F2EC37F029D09F5110E0D7EC37F049
:1049AA007CAF02D0800E7C2794EC36F0A4AF06D000
:1049BA00E0EC37F0BCEC37F001E19F6BA05115E059
:1049CA00E9EC37F080AF02D0800E8027A5EC36F0F4
:1049DA00A8AF0BD0F2EC37F08D07000E8E5B8F5B21
:1049EA00905B4AEC38F001E1A06B9F5102E1A051C3
:1049FA0001E0B46BB35101E1D5D0E65110E191A3C6
:104A0A0002D08C8E01D08C9E91A702D08C8A01D0C4
:104A1A008C9AB2B18C8CB2A512D08C8810D0E605D3
:104A2A000EE191A302D08B8401D08B9491A702D07E
:104A3A00898401D08994B2B18B8CB2B5898AB2A12A
:104A4A000DD091A306D0AA07000EAB5BAC5BAD5BA1
:104A5A0005D0AA2B000EAB23AC23AD23B2A50DD0F3
:104A6A0091A706D0AE07000EAF5BB05BB15B05D075
:104A7A00AE2B000EAF23B023B123E65103E18C9C89
:104A8A008C9890D0E60501E08DD08B9C899A8AD0CB
:104A9A00030E785D59E1F3513AE09905DF6E9651BC
:104AAA0097111AE1A1EC37F0EF500E01EA6AAC2532
:104ABA00E96EAD51EA22EF6A6AEC39F0EE6AED6A04
:104ACA0070EC39F0EE6AED6AA1EC37F0EF6A8FEC20
:104ADA0039F0EE6AED6A1BD06AEC39F09AC4EEFF3F
:104AEA009BC4EDFF70EC39F096C4EEFF97C4EDFF5E
:104AFA00A1EC37F098C4EFFF8FEC39F0EE50ED10CF
:104B0A0006E18FEC39F096C4EEFF97C4EDFF0E0173
:104B1A00B6510401985D46E10E01B051040196199F
:104B2A000CE10E01B1510401971907E1010EE76F7B
:104B3A00E36BF25137E08A9835D0E76B010EE36FE9
:104B4A00F25130E08A882ED0040E785D2BE19C5118
:104B5A0022E09DC430F09EC431F0D8903132303218
:104B6A00D890313230323050BB6EF0C432F0F1C4DA
:104B7A0033F0040ED89032363336E804FBE1300EB7
:104B8A003216000E3316CF0EBA143210306E33C0FE
:104B9A0031F0E85003D0BB6ACF0EBA14BA6E0401E2
:104BAA00010EB46FB45101E19BD0B7EC37F001E0CC
:104BBA0097D0786BA95101E08FD0B6C478F4B7C406
:104BCA0079F4B8C47AF4B9C47BF4BAC47CF4BBC42B
:104BDA007DF4BCC47EF4BDC47FF4BEC480F4BFC4FB
:104BEA0081F4C0C482F4C1C483F4C2C484F4C3C4CB
:104BFA0085F4C4C486F4C5C487F4C6C488F4C7C49B
:104C0A0089F4C8C48AF4C9C48BF4CAC48CF4CBC46A
:104C1A008DF4CCC48EF4CDC48FF4CEC490F4CFC43A
:104C2A0091F4D0C492F4D1C493F4D2C494F4D3C40A
:104C3A0095F4D4C496F4D5C497F4D6C498F4D7C4DA
:104C4A0099F4D8C49AF4D9C49BF4DAC49CF4DBC4AA
:104C5A009DF4DCC49EF4DDC49FF4DEC4A0F4B66BFC
:104C6A00B76BB86BB96BBA6BBB6BBC6BBD6BBE6B0E
:104C7A00FBEC37F0CF6BD06BD16BD26BD36BD46BB1
:104C8A00D56BD66BD76BD86BD96BDA6BDB6BDC6BFE
:104C9A00DD6BDE6B780503E0050E785D1AE19CA1F9
:104CAA0004D0A16BA26BA36BA46B9CA304D0A56BCD
:104CBA00A66BA76BA86B92EC39F003E0010E9F6F0D
:104CCA0001D09F6B4AEC38F003E0010EA06F01D0CF
:104CDA00A06B010EA96F04D0926B936B946B956BCA
:104CEA008050800B05E0EE5105E08150010B02E196
:104CFA00010EED6FE552E552E5CFDAFFE7CFD9FFB6
:104D0A00E552E5CFEAFFE5CFE9FF1100D9CFE6FF8B
:104D1A00DACFE6FFE1CFD9FFE2CFDAFFE652DF6A68
:104D2A00DFCF00F0020EE76E0018E8AE02D0E734DB
:104D3A0002D0E750005C3CE2DFCFE9FFEA6AE9BE55
:104D4A00EA68D890E936EA36D890E936EA36790E32
:104D5A00E926040EEA22010EEE6EEE6AEE6AEE6AA9
:104D6A00DFCFE9FFEA6AE9BEEA68D890E936EA36AF
:104D7A00D890E936EA36890EE926040EEA22EE6A66
:104D8A00EE6AEE6AEE6ADFCFE9FFEA6AE9BEEA682E
:104D9A00D890E936EA36D890E936EA36810EE9261D
:104DAA00040EEA22EE6AEE6AEE6AEE6ADF2AB8D7E3
:104DBA000401786B0401916B0401926B936B946B01
:104DCA00956B0401966B976B0401986B0401996BC0
:104DDA0004019A6B9B6B0401010EA96FCD82CD9ED3
:104DEA00CD9CCD9ACD98CD96CD94FE0ECF6E3D0E2C
:104DFA00CE6ECD809F809E909D8092809F9C010E5A
:104E0A00E66EE66A7BEC42F0E552E552010EE66E8A
:104E1A000B0EE66E7BEC42F0E552E5528D849694D9
:104E2A008D829692898C929C8D8096908B82949298
:104E3A008C9C959C8C9E959E8C9895988C9A959A0C
:104E4A00949E828E00000000000000000000000016
:104E5A000000000000000000000000000000000048
:104E6A0000000000000000000000948E829E0401F1
:104E7A00010EF26F0401010EF36F8A9893988996D6
:104E8A0092960401010EE36F0401E66B0401010E20
:104E9A00E76F0401EC6B0401E86BE96BEA6BEB6BFF
:104EAA000401ED6B9380F19E0401010EEE6F93965F
:104EBA00819631EC34F0E552E552E5CFDAFFE7CFDF
:104ECA00D9FF12008EEC34F0F9EC35F0E6EC39F04B
:104EDA00E66AD950FFEC39F00601B45101E0B7D0C7
:104EEA00DF0426E111EC3AF00CE10401010EF26F45
:104EFA00F36BE7EC36F002E2E16AE552E16E00504C
:104F0A000FD0D3EC38F0010EEE1806E1ED5004E1B3
:104F1A000401F26B010E03D00401010EF26FF36F6C
:104F2A00000EE66EE66AE7C4E6FF16EC38F08DD0AE
:104F3A00020EDF5C30E111EC3AF009E10401E66BA4
:104F4A0096909492959C959E9598959A1DD0D3EC9F
:104F5A0038F0010EEE180DE1ED500BE10401010EDF
:104F6A001FEC38F094949294949C929A959292920F
:104F7A006CD0D3EC38F0020EEE1867E1ED5065E123
:104F8A000401020E1FEC38F094849284948C928A65
:104F9A00958292825AD0040EDF5C07E1010EDBCFC4
:104FAA00B0FE020EDBCFB1FE50D0050EDF5C07E18A
:104FBA00010EDBCFAEFE020EDBCFAFFE46D0080EEF
:104FCA00DF5C0FE1D3EC38F0180ED880EE54000EF7
:104FDA00ED5403E2180E27EC38F0010EDBCFAAFEDF
:104FEA0034D0090EDF5C0FE1D3EC38F0060ED8801E
:104FFA00EE54000EED5403E2060E27EC38F0010ED3
:10500A00DBCFABFE22D00A0EDF5C03E12EEC38F0D8
:10501A0009D00B0EDF5C03E12EEC38F016D00C0E33
:10502A00DF5C07E1010EDBCFB4FE020EDBCFB5FE7B
:10503A000CD00D0EDF5C09E111EC3AF004E004013A
:10504A00010EEE6F02D00401EE6BE7EC41F042EC88
:10505A0039F0C9EF34F08EEC34F0420EE12402E369
:10506A00E168E65297EC39F0410EAEEC38F0080FE1
:10507A00CDEC39F0100FCDEC39F0040FEBEC34F035
:10508A00070E5BEC34F0E66AD9500C0FCDEC39F020
:10509A00140FD9EC39F0410F15EC3AF001E075D153
:1050AA001AEC36F002E388EC37F0DCEC39F046EC27
:1050BA0039F00BE3040EDB68050EDB68060EDB68CD
:1050CA007F0EF36E070EF3CFDBFFFAEC38F005E143
:1050DA0056EC35F078EC36F003E0B6EC36F035E114
:1050EA00040EDBCF0CF0050EDBCF0DF0060EDBCF86
:1050FA000EF0070EDBCF0FF00C500D100E100F1034
:10510A0011E1140EDBCF10F0150EDBCF11F0160EE5
:10511A00DBCF12F0170EDBCF13F010501110121064
:10512A00131011E00C0EDBCF14F00D0EDBCF15F0CF
:10513A000E0EDBCF16F00F0EDBCF17F01450151042
:10514A001610171002E1B48D20D1410EDB5003086E
:10515A0005E2030EF36E410EF3CFDBFFD1EC39F01B
:10516A0002E678EC34F009E2B7EC38F027EC35F0D7
:10517A006FEC38F002EC36F008D056EC35F090ECD3
:10518A0037F06FEC38F063EC35F07DEC36F0D9503F
:10519A00140F6BEC38F002E678EC34F005E21CEC04
:1051AA0035F04FEC39F004D070EC35F054EC39F0AE
:1051BA001DEC36F0410EDB50E76E3C0EE7CFDBFF0D
:1051CA00320EDB6A330EDB6A340EDB6A350EDB6ABB
:1051DA00310EDB6A8D908B92D950080F6BEC38F048
:1051EA0002E678EC34F007E2310EDB500209E76E92
:1051FA00310E05EC3AF0D5EC39F002E678EC34F0F1
:10520A000BE2310EDB500809E76E310EE7CFDBFF08
:10521A0096EC38F02AEC36F06FEC38F0C7EC36F042
:10522A001C0EEECFDBFFF0EC39F0290EEECFDBFFE0
:10523A002A0EEECFDBFF2B0EEECFDBFF2C0EEECFCE
:10524A00DBFF3FEC39F0DCEC39F017EC37F00C0FF0
:10525A0062EC34F02D0EEECFDBFF2E0EEECFDBFF2D
:10526A002F0EEECFDBFF300EEECFDBFFD950140F3F
:10527A0062EC34F037EC36F0010EF36E180EF3CF11
:10528A00DBFF0401A951FDE0180EDBCFB6F4190EBD
:10529A00DBCFB7F41A0EDBCFB8F41B0EDBCFB9F4B1
:1052AA001C0EDBCFBAF41D0EDBCFBBF41E0EDBCF18
:1052BA00BCF41F0EDBCFBDF4200EDBCFBEF4210EF3
:1052CA00DBCFBFF4220EDBCFC0F4230EDBCFC1F459
:1052DA00240EDBCFC2F4250EDBCFC3F4260EDBCFC0
:1052EA00C4F4270EDBCFC5F4280EDBCFC6F4290E93
:1052FA00DBCFC7F42A0EDBCFC8F42B0EDBCFC9F401
:10530A002C0EDBCFCAF42D0EDBCFCBF42E0EDBCF67
:10531A00CCF42F0EDBCFCDF4300EDBCFCEF4310E32
:10532A00DBCFCFF4320EDBCFD0F4330EDBCFD1F4A8
:10533A00340EDBCFD2F4350EDBCFD3F4360EDBCF0F
:10534A00D4F4370EDBCFD5F4380EDBCFD6F4390ED2
:10535A00DBCFD7F43A0EDBCFD8F43B0EDBCFD9F450
:10536A003C0EDBCFDAF43D0EDBCFDBF43E0EDBCFB7
:10537A00DCF43F0EDBCFDDF4400EDBCFDEF4A96BAD
:10538A000601E35102E0E7EC41F0420EE15C02E281
:10539A00E16AE552E16EC9EF34F08EEC34F03E0E6C
:1053AA00E12402E3E168E652E16EDE6A29EC39F0B3
:1053BA00F1EC38F03D0EAEEC38F0040FCDEC39F0DC
:1053CA000C0FCDEC39F0080FCDEC39F0100FD9ECF9
:1053DA0039F03D0F15EC3AF001E022D1FAEC38F041
:1053EA0010E0040EDBCF04F0050EDBCF05F0060E4D
:1053FA00DBCF06F0070EF4EC39F005E1B6EC36F037
:10540A0002E1B48D0DD13D0EDB50030805E2030E17
:10541A00F36E3D0EF3CFDBFF3D0EDB50E76E380E29
:10542A00E7CFDBFF2E0EDB6A2F0EDB6A300EDB6A5C
:10543A00310EDB6A2D0EDB6A8D908B92D950040FE8
:10544A006BEC38F002E678EC34F00BE22D0EDB5010
:10545A000209E76E2D0EE7CFDBFFA2EC38F044EC31
:10546A0036F0D950080F6BEC38F002E678EC34F0DD
:10547A0007E22D0EDB500809E76E2D0E05EC3AF017
:10548A00D5EC39F002E678EC34F005E2C2EC38F0FB
:10549A004FEC39F004D002EC35F054EC39F01DEC45
:1054AA0036F0D1EC39F002E678EC34F009E2B7ECE8
:1054BA0038F027EC35F0F0EC39F002EC36F008D091
:1054CA0056EC35F090EC37F0F0EC39F063EC35F04F
:1054DA003AEC37F0DCEC39F0B7EC35F0180EEECFD9
:1054EA00DBFF6FEC38F037EC36F019EC3AF017ECDA
:1054FA0037F0080F62EC34F0C7EC36F01C0EEECF32
:10550A00DBFF290EDB6A35EC38F03FEC39F0050E8B
:10551A00F36E140EF3CFDBFF0401A951FDE0140E64
:10552A00DBCFB6F4150EDBCFB7F4160EDBCFB8F42B
:10553A00170EDBCFB9F4180EDBCFBAF4190EDBCF96
:10554A00BBF41A0EDBCFBCF41B0EDBCFBDF41C0E72
:10555A00DBCFBEF41D0EDBCFBFF41E0EDBCFC0F4D3
:10556A001F0EDBCFC1F4200EDBCFC2F4210EDBCF3E
:10557A00C3F4220EDBCFC4F4230EDBCFC5F4240E12
:10558A00DBCFC6F4250EDBCFC7F4260EDBCFC8F47B
:10559A00270EDBCFC9F4280EDBCFCAF4290EDBCFE6
:1055AA00CBF42A0EDBCFCCF42B0EDBCFCDF42C0EB2
:1055BA00DBCFCEF42D0EDBCFCFF42E0EDBCFD0F423
:1055CA002F0EDBCFD1F4300EDBCFD2F4310EDBCF8E
:1055DA00D3F4320EDBCFD4F4330EDBCFD5F4340E52
:1055EA00DBCFD6F4350EDBCFD7F4360EDBCFD8F4CB
:1055FA00370EDBCFD9F4380EDBCFDAF4390EDBCF36
:10560A00DBF43A0EDBCFDCF43B0EDBCFDDF43C0EF1
:10561A00DBCFDEF4A96B0601E35102E0E7EC41F0CF
:10562A003E0EE15C02E2E16AE552E16EC9EF34F056
:10563A008EEC34F0110EE12402E3E168E65272ECDA
:10564A0034F0100EAEEC38F0040FD9EC39F0080F34
:10565A00D9EC39F0100FB3EC38F00E01B75101E173
:10566A007AD0FAEC38F002E10601B48D0601B451A1
:10567A0001E07ED025EC37F004E2FB0E006EB70E97
:10568A0061D0D1EC36F002E6BAEC34F005E2DCEC9B
:10569A0039F047EC37F004D0A2EC38F02AEC36F0B7
:1056AA00CFEC34F002E64CEC35F004E2CD0E006E9D
:1056BA00B70E48D0C2EC38F0ABEC34F004E29D0EE1
:1056CA00006EB70E3FD02FEC39F00C0F25EC39F0F5
:1056DA0009E302EC35F078EC36F004E0770E006E60
:1056EA00B70E30D0DCEC36F002E6BAEC34F005E264
:1056FA00F0EC39F047EC37F004D074EC38F02AECCF
:10570A0036F0CFEC34F002E64CEC35F004E2490E08
:10571A00006EB70E17D0C2EC38F0ABEC34F004E2EE
:10572A00190E006EB70E0ED02FEC39F00C0F25ECC7
:10573A0039F00BE302EC35F078EC36F006E0F30EC4
:10574A00006EB60E1DEC3AF013D0100EDB500308B3
:10575A0002E2100EDB6A100EBFEC39F002E2E16AD7
:10576A00E552E16E00500601E35102E0E7EC41F038
:10577A00110EE15C02E2E16AE552E16EC9EF34F032
:10578A008EEC34F0250EE12402E3E168E65297EC50
:10579A0039F0180EDB6A04EC38F0A8EC37F0010E89
:1057AA00F36E200EF3CFDBFF210EDB6A220EDB6ADB
:1057BA00230EDB6A240EDB6AEBEC39F036EC37F0A9
:1057CA00040FD9EC39F0080F67EC38F0FAEC38F02E
:1057DA0003E10601B48D8CD10401A951FDE0200E2C
:1057EA00DB040AE1F29EB7EC37F004E1785102E1FA
:1057FA00200EDB6AF28EF3D7AAC404F0ABC405F01C
:10580A00ACC406F0ADC407F0C3EC37F0040F5EEC8D
:10581A0039F054EC37F0AEC404F0AFC405F0B0C4AC
:10582A0006F0B1C407F0C3EC37F0080F5EEC39F0AC
:10583A0061EC37F0D5EC39F002E678EC34F005E2A9
:10584A0096EC38F051EC36F004D0D9500C0F1EEC1F
:10585A0039F0D1EC39F002E678EC34F00FE212ECD0
:10586A0039F0180E18C0DBFF190E19C0DBFF1A0E2B
:10587A001AC0DBFF1B0E1BC0DBFF07D021EC3AF07E
:10588A00180EEECFDBFFC7EC36F0D8EC35F002E6A7
:10589A004CEC35F013E3180EDBCF1DF0190EDBCFFD
:1058AA001EF01A0EDBCF1FF01B0EDBCF20F02034C8
:1058BA00000E201802E64CEC35F004E2C30E006E2E
:1058CA00B60E94D0E3EC35F0DBCF03F0D950140FC9
:1058DA0062EC34F0030EEBCFF3FF0350F318E8AE9B
:1058EA0002D0F33408D0EE50005CEE500158EE506E
:1058FA000258EE50035870E21CEC35F034EC34F0E8
:10590A00C8EC35F004E2900E006EB60E6FD0D7ECFC
:10591A0038F0180F25EC39F001E2CCD0180EDBCFA5
:10592A0004F0190EDBCF05F01A0EDBCF06F01B0EC2
:10593A00F4EC39F001E1BED0E3EC35F034EC34F0AC
:10594A00CFEC34F002E6BAEC34F006E237EC35F08C
:10595A0002E6BAEC34F029E3D5EC39F002E678EC49
:10596A0034F006E237EC35F002E6BAEC34F00CE338
:10597A00CFEC34F002E6BAEC34F00BE2D1EC39F0B9
:10598A0002E678EC34F005E212EC39F06EEC37F00E
:10599A000ED0D5EC39F002E678EC34F008E2D1EC1E
:1059AA0039F002E678EC34F002E23FEC39F0F8EC38
:1059BA0039F0210FC7EC39F002E2E16AE552E16EF3
:1059CA00005002EC35F076EC39F054EC37F0F1EC9B
:1059DA0038F01CEC35F06CD0E3EC35F034EC34F0F4
:1059EA00C8EC35F006E25D0E006EB60E1DEC3AF01C
:1059FA007FD0D7EC38F0140F25EC39F05BE39BEC41
:105A0A0039F058E01CEC35F034EC34F037EC35F072
:105A1A0002E6BAEC34F006E2CFEC34F002E6BAEC75
:105A2A0034F029E3D1EC39F002E678EC34F006E2FE
:105A3A00CFEC34F002E6BAEC34F00CE337EC35F094
:105A4A0002E6BAEC34F00BE2D5EC39F002E678EC77
:105A5A0034F005E296EC38F06EEC37F010D0D1EC69
:105A6A0039F002E678EC34F00AE2D5EC39F002E6D5
:105A7A0078EC34F004E219EC3AF0F5EC34F0030E69
:105A8A00E66ED950210F89EC38F0D9500C0FC7ECCB
:105A9A0039F002E2E16AE552E16E005056EC35F067
:105AAA0076EC39F061EC37F08DEC38F0E3EC35F058
:105ABA0034EC34F0D9501C0F62EC34F00A0E62EC6C
:105ACA0039F007E20A0EF36E1C0EF3CFDBFFA8ECE7
:105ADA0037F0F8EC39F00C0FC7EC39F002E2E16A62
:105AEA00E552E16E00500601E35102E0E7EC41F0B5
:105AFA00250EE15C02E2E16AE552E16EC9EF34F09B
:105B0A008EEC34F0190EE12402E3E168E65297ECD8
:105B1A0039F0180EAEEC38F00C0FCDEC39F0100F4E
:105B2A00D9EC39F0180FB3EC38F0180EDB50030833
:105B3A0005E2030EF36E180EF3CFDBFFFAEC38F032
:105B4A0002E10601B48DB7EC38F0DBCF03F019ECB3
:105B5A003AF002EC36F01DEC36F002EC35F021ECAE
:105B6A003AF05EEC36F03AEC37F0D1EC36F002E679
:105B7A00BAEC34F005E2D950040F1EEC39F004D027
:105B8A00A2EC38F051EC36F025EC37F004E2FB0ECB
:105B9A00006EB70E4ED0D8EC35F002E64CEC35F07C
:105BAA0004E2CD0E006EB70E44D01CEC35F0ABEC1F
:105BBA0034F004E29D0E006EB70E3BD02FEC39F0A4
:105BCA00140F25EC39F007E39BEC39F004E0770E6B
:105BDA00006EB70E2ED0DCEC36F002E6BAEC34F0EA
:105BEA0005E2D950080F1EEC39F004D074EC38F0F5
:105BFA0051EC36F0D8EC35F002E64CEC35F004E224
:105C0A00490E006EB70E15D01CEC35F0ABEC34F033
:105C1A0004E2190E006EB70E0CD02FEC39F0140FF7
:105C2A0025EC39F009E39BEC39F006E0F30E006E3F
:105C3A00B60E1DEC3AF00DD00601B4510AE1180E69
:105C4A00BFEC39F002E2E16AE552E16E0050E7EC9E
:105C5A0041F0190EE15C02E2E16AE552E16EC9EF38
:105C6A0034F08EEC34F0390EE12402E3E168E652B6
:105C7A0072EC34F0F10EDB50030805E2030EF36E0A
:105C8A00F10EF3CFDBFFF10EDB50E76E340EE7CFF8
:105C9A00DBFF0FEC35F08FEC36F017E1E5EC38F06E
:105CAA0014E1020EF36E100EF3CFDBFFDAEC34F0E0
:105CBA002A0E18C0DBFF2B0E19C0DBFF2C0E1AC0F0
:105CCA00DBFF2D0E1BC0DBFF7BD135EC38F02D0E30
:105CDA00DB6A290EDB6A8D908B92AFEC37F0F0EC21
:105CEA0034F002E678EC34F01FE2290EDB500209A8
:105CFA00E76E290EE7CFDBFFF60EDBCF1CF0F70EBF
:105D0A00DBCF1DF0F80EDBCF1EF0F90EB2EC34F04B
:105D1A00F60E18C0DBFFF70E19C0DBFFF80E1AC02B
:105D2A00DBFFF90E1BC0DBFFB3EC37F0F0EC34F00D
:105D3A0002E678EC34F01FE2290EDB500809E76E20
:105D4A00290EE7CFDBFFF20EDBCF1CF0F30EDBCF21
:105D5A001DF0F40EDBCF1EF0F50EB2EC34F0F20EAD
:105D6A0018C0DBFFF30E19C0DBFFF40E1AC0DBFF0D
:105D7A00F50E1BC0DBFF0FEC35F08FEC36F001E1BE
:105D8A0078D0AFEC37F0F0EC34F002E60DEC38F0F6
:105D9A0026E2DAEC34F044EC36F00FEC35F00F0E74
:105DAA001F0B03E0C1EC35F0FDE19EEC34F0EEECA4
:105DBA0035F00FEC35F00F0E1F0B03E0C1EC35F098
:105DCA00FDE17CEC39F014E2F6EC36F003E0C1ECCC
:105DDA0035F0FDE19EEC34F07BEC37F009D00FECA6
:105DEA0035F00BEC36F03CEC38F0FDE1E0EC39F044
:105DFA0030EC37F00EE26FEC38F095EC34F0280E08
:105E0A00006EB60E34EC39F002E2E16AE552CDECEE
:105E1A0037F0FAEC38F014E1F60EDBCF04F0F70EA7
:105E2A00DBCF05F0F80EDBCF06F0F90EF4EC39F013
:105E3A0007E0FD0E006EB50EC0EC34F09CEC37F0B6
:105E4A0042EC35F00BE205EC37F003E043EC38F0B6
:105E5A00FDE1D9500C0F5EEC39F008D067EC34F054
:105E6A00100E1F0B03E0C1EC35F0FDE17DEC36F0BE
:105E7A0003D0DE6A29EC39F01AEC36F002E388EC3A
:105E8A0037F06FEC38F0110EEECFDBFF120EEECFCB
:105E9A00DBFF130EEECFDBFF140EEECFDBFFAFEC12
:105EAA0037F0F5EC34F004EC38F097EC35F08FEC81
:105EBA0036F06DE0B3EC37F0F0EC34F002E60DECBE
:105ECA0038F026E2DAEC34F044EC36F097EC35F0B0
:105EDA000F0E1F0B03E0C1EC35F0FDE19EEC34F030
:105EEA00EEEC35F097EC35F00F0E1F0B03E0C1EC2A
:105EFA0035F0FDE17CEC39F014E2F6EC36F003E023
:105F0A00C1EC35F0FDE19EEC34F07BEC37F009D0C2
:105F1A0097EC35F00BEC36F03CEC38F0FDE1E0ECB8
:105F2A0039F030EC37F00EE26FEC38F095EC34F0E3
:105F3A00C80E006EB50E34EC39F002E2E16AE552A1
:105F4A00CDEC37F0FAEC38F00AE1E5EC38F007E08E
:105F5A009D0E006EB50EC0EC34F09CEC37F042ECAE
:105F6A0035F00BE205EC37F003E043EC38F0FDE1E5
:105F7A00D9500C0F5EEC39F008D067EC34F0100EF3
:105F8A001F0B03E0C1EC35F0FDE17DEC36F01AECB5
:105F9A0036F002E388EC37F06FEC38F0B7EC35F006
:105FAA00180EEECFDBFFB3EC37F037EC36F0A8EC87
:105FBA0037F0200EDB6A010EF36E100EF3CFDBFF13
:105FCA000401A951FDE0100EDBCFB6F4110EDBCFB0
:105FDA00B7F4120EDBCFB8F4130EDBCFB9F4140EFC
:105FEA00DBCFBAF4150EDBCFBBF4160EDBCFBCF455
:105FFA00170EDBCFBDF4180EDBCFBEF4190EDBCFC4
:10600A00BFF41A0EDBCFC0F41B0EDBCFC1F41C0E9B
:10601A00DBCFC2F41D0EDBCFC3F41E0EDBCFC4F4FC
:10602A001F0EDBCFC5F4200EDBCFC6F4210EDBCF6B
:10603A00C7F4220EDBCFC8F4230EDBCFC9F4240E3B
:10604A00DBCFCAF4250EDBCFCBF4260EDBCFCCF4A4
:10605A00270EDBCFCDF4280EDBCFCEF4290EDBCF13
:10606A00CFF42A0EDBCFD0F42B0EDBCFD1F42C0EDB
:10607A00DBCFD2F42D0EDBCFD3F42E0EDBCFD4F44C
:10608A002F0EDBCFD5F4300EDBCFD6F4310EDBCFBB
:10609A00D7F4320EDBCFD8F4330EDBCFD9F4340E7B
:1060AA00DBCFDAF4350EDBCFDBF4360EDBCFDCF4F4
:1060BA00370EDBCFDDF4380EDBCFDEF4A96B390EF9
:1060CA00E15C02E2E16AE552E16EC9EF34F08EEC7E
:1060DA0034F0110EE12402E3E168E652E16EDF6A70
:1060EA00010EDB6A020EDB6A030EDB6AADEC39F0E5
:1060FA00100EDB6A0401A95102E1B60502E0780537
:10610A0002E1010EDF6EB60525E1B66B090EC7C4C2
:10611A00DBFF0A0EC8C4DBFF0B0EC9C4DBFF0C0E83
:10612A00CAC4DBFF0D0ECBC4DBFF0E0ECCC4DBFFF3
:10613A000F0ECDC4DBFF100ECEC4DBFFFBEC37F035
:10614A00BF6BC06BC16BC26BC36BC46BC56BC66BD9
:10615A00010EA96F780529E1786B010E89C4DBFF6E
:10616A00020E8AC4DBFF030E8BC4DBFF040E8CC451
:10617A00DBFF050E8DC4DBFF060E8EC4DBFF070EA8
:10618A008FC4DBFF080E90C4DBFF896B8A6B8B6BB5
:10619A008C6B8D6B8E6B8F6B906B816B826B836B51
:1061AA00846B856B866B876B886BE7EC41F0110E0D
:1061BA00E15C02E2E16AE552E16EE6D3E7C400F08F
:1061CA00016A00BE016854EC38F0980E026EB50EF2
:1061DA006BEC36F002E2E16AE552E16E0550E7EF58
:1061EA0041F0FEEC38F0DE6ADD6A010EE66E9FECE5
:1061FA0039F0030E5BDB0601B4510FE10401E70538
:10620A0004E159EC38F0E66A04D059EC38F0010E92
:10621A00E66E16EC38F0E7EC41F0E552E552B4D3FD
:10622A00FEEC38F0F9EC35F096EC37F003EC39F087
:10623A0036EC37F0030FB3EC38F01AEC38F00601FD
:10624A00B45129E1030EDB50070802E296EC37F05D
:10625A00DF50010802E2010EDF6E030EDB50030F6E
:10626A000E01B65D0CE0E7EC36F002E2E16AE552B7
:10627A00E16E0050030EDB50030F0E01B66F010EE4
:10628A00DBCFE6FF020EDBCFE6FFDFCFE6FF16EC41
:10629A0038F0E7EC41F0050EE15C02E2E16AE55212
:1062AA00E16E72D3FEEC38F0E652E652FD0EDB04E4
:1062BA000BE1B0CEDEFFB1CEDDFF020EB2CEDBFFC8
:1062CA00030EB3CEDBFF0AD0AECEDEFFAFCEDDFFCC
:1062DA00020EB4CEDBFF030EB5CEDBFF89861DC5E9
:1062EA0019F51EC51AF51FC51BF520C51CF5FB0EB1
:1062FA00DBCFE6FFFC0EDBCFE6FF020EDBCFE6FFCD
:10630A00030EDBCFE6FFB6CEE6FF59EC38F0DCEC45
:10631A005FF0006E070EE15C02E2E16AE552E16EAF
:10632A000050040EE15C02E2E16AE552E16E2CD310
:10633A00FEEC38F0E652E6EC39F0E76E020EE7CFF3
:10634A00DBFFDB5039E10601B4515BE10401E651A0
:10635A0003E0020EE65D28E1DF50000821E2E65183
:10636A0001E18D90DF0403E18D848D82898C020E18
:10637A00DF5C03E18D848D82899C030EDF5C03E17F
:10638A008D948D82899C040EDF5C03E18D848D924D
:10639A00899C050EDF5C10E18D948D92899C0CD04E
:1063AA00E6510AE18D8008D0E60506E1DF500008D3
:1063BA0002E28C9201D08C8236EC37F0010FB3ECFA
:1063CA0038F0E76E020EE7CFDBFFDB5017E106017C
:1063DA00B45117E10401E65108E1010EDB5000084F
:1063EA0002E28B920BD08B8209D0E60507E1010EFF
:1063FA00DB50000802E2899201D0898219DAE7ECBF
:10640A0041F042EC39F0C0D2FE0E0401E85DFF0E05
:10641A00E959FF0EEA59FF0EEB5905E2E82B000E87
:10642A00E923EA23EB23E7EF41F00401E851E911FC
:10643A00EA11EB1105E0E807000EE95BEA5BEB5BAA
:10644A00E7EF41F0FEEC38F0E652E652E652EBECAA
:10645A0039F01AEC38F0DB500BE1DFCFE8F4010E2B
:10646A00DBCFE9F4020EDBCFEAF4030EDBCFEBF469
:10647A00E7EC41F0050EE15C02E2E16AE552E16E09
:10648A0083D2E8C4E6FFE9C4E6FFEAC4E6FFEBC448
:10649A00E6FF8F0E006EB50E34EC39F002E2E16AC7
:1064AA00E5525EEF38F0E66AEC0EE66E040EE66E32
:1064BA00010EFCD90601B45101E01200E7EF41F0E8
:1064CA00ECC400F0016A00BE016854EC38F0880E92
:1064DA00026EB50E6BEC36F002E2E16AE552E16E4D
:1064EA000550E7EF41F0EDC400F0016A00BE016813
:1064FA0054EC38F0820E026EB50EE8DB02E2E16A75
:10650A00E552E16E0401ED5101E0ED6BE7EF41F078
:10651A009DBCFED716C1E6FF17C1E6FF00C1E6FF24
:10652A0001C1E6FF760E006EB50E34EC39F002E2D8
:10653A00E16AE5525EEF38F0ECD9E652C4D8DF6E74
:10654A000F0EDF14DF6E0401E75103E0100EDF10B7
:10655A00DF6EED5103E0200EDF10DF6E81A403D061
:10656A00400EDF10DF6E81AA03D0800EDF10DF6ECF
:10657A00DFCFE6FFE66A6F0E006EB50EFCD9036E3A
:10658A00050EE15C02E2E16AE552E16E03500401A4
:10659A00ED5101E0ED6BE552F7D1FEEC38F0A4ECD9
:1065AA0039F003EC39F01AEC38F036EC37F0030F17
:1065BA0015EC3AF001E07FD0D3EC38F0FF0ED8802A
:1065CA00EE54030EED5405E2010EDB68030E62EC95
:1065DA0038F0DF50010802E2010EDF6E030EDB50D5
:1065EA00010802E296EC37F0DF0409E1040EDB5001
:1065FA00030805E10401F06B020EF16F06D0010EEB
:10660A00DBCFF0F4020EDBCFF1F4CAB415D0CB68BD
:10661A00FC0ECA140009CA6E9D920F015281529350
:10662A00F00EBA140C09BA6E3F0EBA140009BA6E0B
:10663A000E010E0ECC6FCA84030EDB502AE1DF5026
:10664A0023E0F0C400F0F1C401F0D8900132003226
:10665A00D890013200320050BB6EF0C402F0F1C48F
:10666A0003F0040ED89002360336E804FBE1300E3C
:10667A000216000E0316CF0EBA1400010210006EA5
:10668A0003C001F0E85003D0BB6ACF0EBA14BA6E49
:10669A0010D00401A951FDE0F0C4DBF4F1C4DCF42C
:1066AA00D06BD16BD26BD36BDFCFDAF4040EB66F3B
:1066BA00A96BE7EC41F0050EE15C02E2E16AE55202
:1066CA00E16E62D1120025D9E652A4EC39F0F29EAD
:1066DA000401B7EC37F002E0010EDF6E785102E0F8
:1066EA00010EDF6EA95106E1010EDF6EF36E030E95
:1066FA00F3CFDBFFDF5006E092EC39F003E0DE5225
:10670A00010EDD6EDF5006E04AEC38F003E0010EC0
:10671A0062EC38F0F28E030EDBCFE6FF020EDB509E
:10672A00E824016E010EDB50040DF3CF00F0DF50B8
:10673A00080DF35000100110E552E710006E040E28
:10674A00E15C02E2E16AE552E16E00501DD1FEEC25
:10675A0038F0A4EC39F0B7DF1AEC38F0DBB0E1DB43
:10676A00040EDBA203D0010E62EC38F0040EDBA4A7
:10677A0003D0DE52010EDD6E040EDBA602D0010E3E
:10678A00DF6E030EDBCFE6FFE66A020EDBCFE6FF23
:10679A00E66A010EDBCFE6FFE66ADFCFE6FFE66ACE
:1067AA005E0E006EB50EE7D8036E0B0EE15C02E2D8
:1067BA00E16AE552E16E0350050EE15C02E2E16A2C
:1067CA00E552E16EE1D0A5D8080EE12402E3E168C2
:1067DA00E652E16EF29EAAC4DFFF010EABC4DBFFF4
:1067EA00020EACC4DBFF030EADC4DBFF040EAEC465
:1067FA00DBFF050EAFC4DBFF060EB0C4DBFF070EDE
:10680A00B1C4DBFFF28E29EC3AF0540E006EB50EDD
:10681A00B2D8036E0B0EE15C02E2E16AE5525EEC6D
:10682A0038F0080EE15C02E2E16AE552E16EACD0B2
:10683A00F29E0401AA6BAB6BAC6BAD6BAE6BAF6B2C
:10684A00B06BB16BA16BA26BA36BA46BA56BA66BB0
:10685A00A76BA86BF28E1200EBDFE7EF41F0DBCFFC
:10686A0003F082EC39F080EC38F043EC64F018C0A5
:10687A0000F019C001F01AC002F01BC003F018C0E2
:10688A001CF019C01DF01AC01EF01BC01FF007EC47
:10689A0039F01C0E1CC0DBFF1D0E1DC0DBFF1E0ED7
:1068AA001EC0DBFF1F0E1FC0DBFF1200E66ED2EC1C
:1068BA0048F042EC39F0E5521200E96E000EDA2097
:1068CA00EA6E12006FEC38F0EECF00F0EECF01F076
:1068DA00EECF02F0EFCF03F01200E16EDE6A29EC90
:1068EA0039F0ADEF39F0000E62EF39F0216E050E86
:1068FA00226E236A246A80EC38F0FAEC64F01CC039
:10690A0000F01DC001F01EC002F01FC003F0D950F4
:10691A0012009FEC39F0E1CFD9FFE2CFDAFF120083
:10692A00EECFE6FFEECFE6FFEECFE6FFEFCFE6FFD4
:10693A001200E1DB040EDBCF21F0050EDBCF22F0E3
:10694A00060EDBCF23F0070E25EF3AF0DBCF03F07C
:10695A00D2DB07EC39F03AEF39F0DBCF1FF02168D0
:10696A0022682368246843EF64F0D8800AEC3AF07E
:10697A00000E20541200016E026A00C0E6FFE66EA5
:10698A0002C0E6FF6CEF63F0E552E5CFDAFFE7CF2E
:10699A00D9FF12000C0EDBCF1DF00D0EDBCF1EF05F
:1069AA000E0EDBCF1FF00F0EF3D3FA0EDBCF00F083
:1069BA00FB0EDBCF01F0FC0EDBCF02F0FD0EDBCFCE
:1069CA0003F058EC39F097DB43EF64F0E66E000E03
:1069DA00DA20E66E1200D890030EEB50000A12007D
:1069EA00210EEECFDBFF220EEECFDBFF230EEECF22
:1069FA00DBFF240EEECFDBFF12000C0EDBCF04F020
:106A0A000D0EDBCF05F00E0EDBCF06F00F0EDBCF3F
:106A1A0007F01200F60EDBCF00F0F70EDBCF01F025
:106A2A00F80EDBCF02F0F90EDBCF03F01200140EE2
:106A3A00DBCF00F0150EDBCF01F0160EDBCF02F034
:106A4A00170E1200DBCF03F0000E006C011E0122AC
:106A5A00021E0222031E0322D8900332023201329E
:106A6A0000321200100EDBCF1DF0110EDBCF1EF02C
:106A7A00120EDBCF1FF0130E8BD3D950FA0FA8ECEE
:106A8A0039F0D8801E0EEE54000E89EF39F0D88006
:106A9A00FF0E1D54FF0E1E54FF0E1F54000E2054ED
:106AAA001200100EDBCF04F0110EDBCF05F0120E30
:106ABA00DBCF06F0130EDBCF07F012000450EE5CBA
:106ACA00006E0550EE58016E0650EE58026E0750E1
:106ADA00EE58036E1200140EDBCF04F0150EDBCF56
:106AEA0005F0160EDBCF06F0170EDBCF07F012000B
:106AFA00080E18C0DBFF090E19C0DBFF0A0E1AC008
:106B0A00DBFF0B0E1BC0DBFF12000450EE24006EED
:106B1A000550EE20016E0650EE20026E0750EE2060
:106B2A00036E1200F20EDBCF00F0F30EDBCF01F0A2
:106B3A00F40EDBCF02F0F50EDBCF03F01200EE50BD
:106B4A001C5CEE501D58EE501E58EE501F58120095
:106B5A0043DB140EDB6A150EDB6A160EDB6A170EB0
:106B6A00DB6A1200150EEECFDBFF160EEECFDBFF4F
:106B7A00170EEECFDBFF1200D89000360136023630
:106B8A000336E8061200A6DAEECF1CF0EECF1DF0AF
:106B9A00EECF1EF0EFCF1FF0B0DBFAEC64F065D356
:106BAA00E66A9FEF39F0140EDBCF1DF0150EDBCF2E
:106BBA001EF0160EDBCF1FF0170EEAD2180EDBCF2F
:106BCA0000F0190EDBCF01F01A0EDBCF02F01B0E1C
:106BDA0012001CC0DEFF1DC0DEFF1EC0DEFF1FC08C
:106BEA00DDFFDD52DD521200E652E652E652DF6A5E
:106BFA00010EDB6A020EDB6A1200EE500026EE502E
:106C0A000122EE500222EE500322120074DAFA0E2A
:106C1A00DBCF21F0FB0EDBCF22F0FC0EDBCF23F023
:106C2A00FD0E25EC3AF00F0E120054DA46EF39F059
:106C3A00040E00C0DBFF050E01C0DBFF060E02C01A
:106C4A00DBFF070E03C0DBFF12000C0E18C0DBFFD0
:106C5A000D0E19C0DBFF0E0E1AC0DBFF0F0E1BC094
:106C6A00DBFF1200250EEECFDBFF260EEECFDBFF99
:106C7A00270EEECFDBFF280EEECFDBFF1200040E4D
:106C8A0018C0DBFF050E19C0DBFF060E1AC0DBFFBA
:106C9A00070E1BC0DBFF1200140E18C0DBFF150E17
:106CAA0019C0DBFF160E1AC0DBFF170E1BC0DBFF75
:106CBA001200EE50045C006EEE500558016EEE5064
:106CCA000658026EEE500758036E1200036E046AED
:106CDA0002C0E6FFE66E04C0E6FF6CEC63F0056EE8
:106CEA00050EE15C12000450051006100710120090
:106CFA0000C0DFFF010E01C0DBFF020E02C0DBFF96
:106D0A00030E03C0DBFF1200EA6ADF34FE0BEA3629
:106D1A00E96E120000500110021003101200790EE1
:106D2A00E96E040EEA6EA151EE24A16FA251EE2083
:106D3A00A26FA351EE20A36FA451EE20A46F1200FC
:106D4A007D0EE96E040EEA6EA551EE24A56FA651DA
:106D5A00EE20A66FA751EE20A76FA851EE20A86FCC
:106D6A001200080EDBCF08F0090EDBCF09F00A0E7D
:106D7A00DBCF0AF00B0EDBCF0BF0085009100A101C
:106D8A000B101200190EEECFDBFF1A0EEECFDBFF4F
:106D9A001B0EEECFDBFF1200040EDBCF1DF0050E3B
:106DAA00DBCF1EF0060EDBCF1FF0070EF1D1080E67
:106DBA00DBCF1DF0090EDBCF1EF00A0EDBCF1FF072
:106DCA000B0EE6D1000EE66EE66AE66EE66AB6CE0F
:106DDA00E6FFE66EE66ADCEC5FF0006E070EE15C49
:106DEA001200080EDBCF00F0090EDBCF01F00A0E0D
:106DFA00DBCF02F00B0EDBCF03F0100E1F0B1200DD
:106E0A0069D9EECF04F0EECF05F0EECF06F0EFCF62
:106E1A0007F0100E1F0B120036EC2EF0006E0D0E4E
:106E2A00E15C12001D0EEECFDBFF1E0EEECFDBFF84
:106E3A001F0EEECFDBFF200EEECFDBFFD950120084
:106E4A0049D9D880FF0EEE54FF0EEE54FF0EEE54D1
:106E5A00000EEE5412003ED9D880000EEE54800E79
:106E6A0053D2010EE66ED9501200080E00C0DBFFA5
:106E7A00090E01C0DBFF0A0E02C0DBFF0B0E03C0C6
:106E8A00DBFF12000C0EEECFDBFF0D0EEECFDBFFA9
:106E9A000E0EEECFDBFF0F0EEECFDBFF12000C0E55
:106EAA0000C0DBFF0D0E01C0DBFF0E0E02C0DBFFD0
:106EBA000F0E03C0DBFF1200100E00C0DBFF110E25
:106ECA0001C0DBFF120E02C0DBFF130E03C0DBFFA3
:106EDA001200210E18C0DBFF220E19C0DBFF230EA1
:106EEA001AC0DBFF240E1BC0DBFF12000C0E1CC0F5
:106EFA00DBFF0D0E1DC0DBFF0E0E1EC0DBFF0F0EEB
:106F0A001FC0DBFF1200DE68DE68DE687F0EDD6E02
:106F1A00DD52DD521200D8900732063205320432B1
:106F2A001200010EF36E030EF3CFDBFF1200A5D998
:106F3A00010EDE6E29EF39F0DF50EA6A310FE96E91
:106F4A000E0EEA2212001D0EDB6A1E0EDB6A1F0EEF
:106F5A00DB6A1200D950F60FA8EF39F0D950F20FB8
:106F6A00A8EF39F0925193119411951112008907E3
:106F7A00000E8A5B8B5B8C5B92EF39F0000E046C1F
:106F8A00051E0522061E0622071E0722D9501200D8
:106F9A00E16E0350DE6A800EDE6EDE6ADD6ADD5265
:106FAA00DD5212008151792782517A2383517B2342
:106FBA0084517C2312007F0EA415A46F010EB21116
:106FCA00B26F010EB36F120085517D2786517E2361
:106FDA0087517F238851802312007F0EA815A86F3E
:106FEA00040EB211B26F010EB36F1200C76BC86BF9
:106FFA00C96BCA6BCB6BCC6BCD6BCE6B1200190E07
:10700A00DB6A1A0EDB6A1B0EDB6A1C0EDB6A1200D5
:10701A00FF0EEE5CFF0EEE58010EEE58000EEE5813
:10702A00120057EC31F042EF39F0E76E040EE7CF69
:10703A00DBFF1200E66F96809482958C958E958878
:10704A00958A1200F36E010EF3CFDBFF020EDB6AA4
:10705A001200010EDBCFB2FE020EDBCFB3FE12002E
:10706A002A0EDB6A2B0EDB6A2C0EDB6A1200D89022
:10707A001C361D361E361F36E8061200D890043616
:10708A00053606360736E80612008D518E118F1125
:10709A0090111200010EE9260E0EEA22120000C01B
:1070AA00E6FF01C0E6FF1200DECFE6FFDDCFE6FF16
:1070BA001200E16E0350E7EF41F0F36E020EF3CFD8
:1070CA00DBFF120083DC060E5BEF34F062EC34F077
:1070DA00F0EF34F0D9CFE9FFDACFEAFF1200080E59
:1070EA00DBCF1CF0090EDBCF1DF00A0EDBCF1EF042
:1070FA000B0EB2EF34F000C01CF001C01DF002C04C
:10710A001EF003C01FF0120062EC34F095EF34F069
:10711A000C0EDB6A0D0EDB6A0E0EDB6A0F0EDB6AE3
:10712A0012000C0EDBCF1CF00D0EDBCF1DF00E0E85
:10713A00DBCF1EF00F0EB2EF34F0040EDBCF1CF0E3
:10714A00050EDBCF1DF0060EDBCF1EF0070EB2EFE9
:10715A0034F0DB6A3BD9E66AD950120037DC010EFB
:10716A005BEF34F0100EDBCF00F0110EDBCF01F035
:10717A00120EDBCF02F0130E12000C0EDBCF00F062
:10718A000D0EDBCF01F00E0EDBCF02F00F0E120058
:10719A00DBCF20F02034000E20181200D950010F46
:1071AA0062EF34F01C0EDBCF00F01D0EDBCF01F0D6
:1071BA001E0EDBCF02F01F0EDBCF03F07BEF34F0A5
:1071CA00F20EDBCF04F0F30EDBCF05F0F40EDBCFCB
:1071DA0006F0F50EF4EF39F0100EDB6A110EDB6AD9
:1071EA00120EDB6A130EDB6A120067EC34F08FEFC3
:1071FA0036F08EEC34F0E652E6521200E2D831DE76
:10720A00FFEF39F0DFCF21F0010EDBCF22F0020EC3
:10721A00DBCF23F0030E25EF3AF0100EDBCF1CF084
:10722A00110EDBCF1DF0120EDBCF1EF0130EB2EFE4
:10723A0034F062EC34F0140EEECFDBFFB7EF35F02A
:10724A0062EC34F0A4EF35F0DE6ADE6ADD6ADD5204
:10725A00DD52120067EC34F01F0E7BEF34F0C0EC05
:10726A0034F0036E070EE15C1200D880190E1C542C
:10727A000AEF3AF0E1D8F5EF34F0E552E552E5527B
:10728A001200FF0EEE5CFF0EEE58FF0EEE587F0E58
:10729A00EE58120027EC35F08AD802EF36F03BDEC2
:1072AA0086D863EF35F0190E216E226A236A246AA2
:1072BA00120062EC34F08AEF35F0EE5C000EEE5804
:1072CA00000EEE58000EEE5812001EDD790EE92669
:1072DA000E0EEA22120018DD490EE9260E0EEA22E7
:1072EA001200D950210F62EC34F05EEF36F09EECBA
:1072FA0034F07DEC35F042EF35F0E80E216E030EE6
:10730A00226E236A246A1200EE54000EEE54000E16
:10731A00EE541200F9DC4FEF38F089518A118B11C3
:10732A008C11120072EC34F0ADEF35F070EC35F0E0
:10733A0078EF36F0D9CFE6FFDACFE6FF120054DC59
:10734A00030EDB6A1200E96EFF0EDA20EA6E120003
:10735A00040EDB6A050EDB6A060EDB6A070EDB6AC1
:10736A00080EDB6A090EDB6A0A0EDB6A0B0EDB6AA1
:10737A008DEF38F0DBCFE6FFD950080FC5DE64D8B1
:10738A0011EF37F0C1DED9501C0FBEDE11EF37F016
:10739A0099DEE66AD9501200D950100F6BEF38F017
:1073AA00D9500C0F6BEF38F08DDE36EF37F0D9502D
:1073BA00040F62EF34F077DFFAEC64F00ADC8DEF49
:1073CA0038F0D5EC35F0010E5BEF34F0D5EC35F042
:1073DA00070E5BEF34F0D950080F62EF34F0DBCFC1
:1073EA0007F078EF36F0030EE66ED950100F8CDEF8
:1073FA00D9501200010FEBEC34F0030E5BEF34F0BE
:10740A00E7CFDBFF6CDE7DEF35F0000E1D54000E7A
:10741A001E54000E1F541200C1DEEE50ED10120071
:10742A009DDE0601B4511200D9500C0F62EF34F000
:10743A00C0EC34F042EF39F0D950100F62EF34F05B
:10744A00DBCF24F0FAEF64F0D950040F5DDE42DEA0
:10745A0095EF34F0D8CFE4FFE0CFE4FFE46EE9CF54
:10746A00E4FFEACFE4FFF3CFE4FFF4CFE4FFE65210
:10747A00E0EC4CF044EC4CF0030EDB6AA4A6B5D168
:10748A00A4960E01002B0E01AB510E01005D01E224
:10749A0084D0006B0E0110EC4CF0EF6A79907B6A95
:1074AA007A6A0E01A92B0E01AA510E01A95D01E308
:1074BA00A96BD6EC4CF0EA22EE50ED106EE0A5EC8A
:1074CA004DF052EC4DF002E12F502D1847E0EAEC56
:1074DA004CF0EA22EE50ED103AE00DEC4DF0E8ECFB
:1074EA004BF0D6EC4CF0EA22EE502E5C2C6EEE50AD
:1074FA002F582D6E020E2CC0DBFF030E2DC0DBFFB2
:10750A005FEC4CF02D3412E22C500008000E2D5482
:10751A000DE25FEC4CF0EAEC4CF023EC4DF017E294
:10752A008BEC4DF0EE262D50ED2218D05FEC4CF08E
:10753A002C6C2D1E000E2D22EAEC4CF023EC4DF0A3
:10754A0006E28BEC4DF0EE5E2D50ED5A07D0A5EC1D
:10755A004DF0EA222CC0EEFF2DC0EDFF10EC4CF0EE
:10756A00120EEF6EF29E0E01D6EC4CF0A4EC4BF02C
:10757A002DC02CF02D6A2C50B66ED6EC4CF0A4EC33
:10758A004BF02C50B56EF00EB4140009B46EF00E28
:10759A00B4140909B46E7980F28E0601000ED880FF
:1075AA00AA55000EAB552EE2B82B000EB923AA51EC
:1075BA00B85DAB51B95926E3B86BB96B030EAE5D32
:1075CA001FE2AC51EA6A200FE96E010EEA2280CF6F
:1075DA00EFFFAC51EA6A230FE96E010EEA2281CF6E
:1075EA00EFFFAC51EA6A260FE96E010EEA2282CF5A
:1075FA00EFFFAC2B030EAC5D01E3AC6BAE2B02D0FC
:10760A00AA6BAB6B000ED880AF55000EB0551CE2CA
:10761A00000ED880BE55000EBF5516E2BA2B000EDA
:10762A00BB23AF51BA5DB051BB590EE3BA6BBB6B0A
:10763A00030EB35D07E2B12B030EB15D01E3B16B3B
:10764A00B32B02D0AF6BB06BBE51BF110BE0050E6E
:10765A00BD5D07E3C18C9E9C9D8CC280C282BD6BBE
:10766A0001D0BD2B0501005101E1AAD0DE6ADD6A15
:10767A00DECF2CF0DDCF2DF0040E2C5C000E2D5841
:10768A0001E39ED08BEC4BF0010EEEEC4BF0FDE1EA
:10769A00010EE926050EEA22EE50ED1075E08BEC9C
:1076AA004BF0010EEEEC4BF0FDE156EC4DF0EE50D6
:1076BA00ED1016E15BEC4DF001E181805FEC4DF0DD
:1076CA0003E1ED5001E1818263EC4DF003E1ED50FD
:1076DA0001E1818467EC4DF003E1ED5001E181861F
:1076EA008BEC4BF0010EEEEC4BF0FDE103EC4DF0B0
:1076FA00EEEC4BF0FDE1010EE926050E52EC4DF0E1
:10770A0019E12F502D1816E15BEC4DF001E1819043
:10771A005FEC4DF003E1ED5001E1819263EC4DF035
:10772A0003E1ED5001E1819467EC4DF003E1ED5086
:10773A0001E181968BEC4BF0010EEEEC4BF0FDE192
:10774A0056EC4DF0EE2A000EEF228BEC4BF0010EB8
:10775A00EEEC4BF0FDE103EC4DF0EEEC4BF0FDE10D
:10776A00090EE926050E52EC4DF024E12F502D1892
:10777A0021E18BEC4BF0010EEEEC4BF0FDE156EC07
:10778A004DF0EE6AED6A16D05BEC4DF001E18190A6
:10779A005FEC4DF003E1ED5001E1819263EC4DF0B5
:1077AA0003E1ED5001E1819467EC4DF003E1ED5006
:1077BA0001E18196DF2A010E01E25AD7DB2A58D766
:1077CA000401EF5101E0EF07050119511A111B11CC
:1077DA001C110BE01907000E1A5B1B5B1C5B19518D
:1077EA001A111B111C1101E189969EAC3DD09E9C79
:1077FA00C1AC07D0C19C010E0601C06FC16BBC6B46
:10780A0018D0C4502E6E2F6E2E6AC35000012E104F
:10781A002C6E2FC02DF00601BC51E96EEA6A39ECD4
:10782A004CF02CC0EEFF2DC0EDFFD890C037C13709
:10783A00BC2B100EBC5D0EE2C051BE152C6EC151A0
:10784A00BF152D6E2C502D1005E1BC2BD890C037DA
:10785A00C137EFD7100EBC5D02E39D9C05D0BC5129
:10786A00040DF328C26EC282F2A435D0D59EF294DA
:10787A00F29A040E2C6E0601B7514AEC4CF0EF5006
:10788A002C5C29E1080EB75D0AE27DEC4CF004E0BD
:10789A00E846FE0B2C06FCE1E81C891616D0100EF1
:1078AA00B75D0AE27DEC4CF004E0E846FE0B2C06DC
:1078BA00FCE1E81C8A1609D07DEC4CF004E0E846AD
:1078CA00FE0B2C06FCE1E81C8B160601B7514AECAC
:1078DA004CF0020EEF6E040EE15C02E2E16AE55240
:1078EA00E16EE552E5CFDAFFE7CFD9FFE552E5CF02
:1078FA00F4FFE5CFF3FFE5CFEAFFE5CFE9FFE55077
:10790A00E5CFE0FFE5CFD8FF100091EC4DF0E6524D
:10791A00896A92680601BE6BBF6B8A6A93688B6A32
:10792A0094688C968C9495969594928E010EE36F3A
:10793A000401FE69FF690601B26BB16BB36BAD6BF3
:10794A00AC6BAE6BAA6BAB6BAF6BB06BB86BB96B56
:10795A00BA6BBB6BBC6B76827680769C769A76889D
:10796A007696FA0E776EDE6ADD6AD3EC4BF004E6A1
:10797A00100E005C000E01580BE28BEC4BF039EC58
:10798A004CF0EE6AED6ADF2A010EEFE3DB2AEDD74F
:10799A000601DD6BDE6BDB6BDC6BDE6ADD6AD3EC6A
:1079AA004BF004E6400E005C000E01580CE28BEC32
:1079BA004BF0000EE926020EEA22EF6ADF2A010ED8
:1079CA00EEE3DB2AECD7DE6ADD6AD3EC4BF004E6A1
:1079DA00400E005C000E01580CE28BEC4BF0400E9E
:1079EA00E926020EEA22EF6ADF2A010EEEE3DB2A1B
:1079FA00ECD7DE6ADD6AD3EC4BF004E6000E005CDD
:107A0A00010E01580AE28BEC4BF089EC4CF0EF6A5C
:107A1A00DF2A010EF0E3DB2AEED70601DF6BE06B0B
:107A2A00E16BE26BB56BB66BB76BDE6ADD6AD3EC02
:107A3A004BF004E6180E005C000E015812E28BECC3
:107A4A004BF093EC4CF0EE6AED6A8BEC4BF0290E9E
:107A5A00E926010EEA22010EEF6EDF2AE8E3DB2AAD
:107A6A00E6D7D586D59AD59CF294F29AF1940F016D
:107A7A00498FBE0EC16ED08E7694A386A5968BECE6
:107A8A0026F00FEC5FF0F28EF28C7684A2EC47F0CF
:107A9A00040EE15C02E2E16AE552E16E6EEF4BF040
:107AAA00E0EC4CF0E65244EC4CF0030EDB6A040EB8
:107ABA00DB6A92EC4AF00601AE5100080AE22CECAD
:107ACA0043F00601AD2B030EAD5D01E1AD6BAE07D0
:107ADA00F2D7B35100080AE24EEC43F00601B22B8A
:107AEA00030EB25D01E1B26BB307F3D7200E0101B9
:107AFA00E76E7119E8AE02D0E73402D0E750715D43
:107B0A0001E23AD16550020B01E036D1400EE66E31
:107B1A00400EE66E020EE66EA6EC5DF095EC4DF0B8
:107B2A00E76E030EE7CFDBFFDB50000801E3E7D087
:107B3A00040EDB6A030EDB50F36E040EF1EC4BF01D
:107B4A0001E3DDD0040EDB50EA6A400FE96E020E53
:107B5A00EA22EFCFDFFF0501655134E10D0EAFECEC
:107B6A004BF005E00A0E016EDF50015C2BE1010EBD
:107B7A00656F0601FBEC4BF00D0EEF6EDD2B010E6F
:107B8A00DB6ADD51F36E010EF1EC4BF016E28EEC7E
:107B9A004CF0E9BEEA6889EC4CF0EF50E66E8EECE8
:107BAA004CF0E9BEEA68210EE926050EEA22E55202
:107BBA00E750EF6E010EDB2AE4D73BD90601DD6BF5
:107BCA00DE6B8DD01B0EDF5C09E1615107E1010E0E
:107BDA00616F1B0E626F636B646B81D061050BE191
:107BEA005B0EDF5C08E11B0E625D05E1635103E198
:107BFA005B0E636F74D061054AE1410EDF5C47E1B9
:107C0A001B0E625D44E15B0E635D41E1626B636B77
:107C1A00646B616B010EDB6ADBCFE9FFEA6AE9BEDE
:107C2A00EA6889EC4CF0EF500D0816E08EEC4CF047
:107C3A00E9BEEA68210EE926050EEA22EF50E66E51
:107C4A008EEC4CF0E9BEEA6889EC4CF0E552E7505C
:107C5A00EF6E010EDB2AE0D7010EDBCFDDF606015F
:107C6A00FBEC4BF0EF6A120E006EBA0ECCEC4CF045
:107C7A00000EE66E030EE66E0F0E006EBA0ED3EC21
:107C8A004CF002E2E16AE552E16E035028D0080E98
:107C9A00DF5C0EE10601DD5100080AE2DD07FBECBC
:107CAA004BF0EF6A0C0E006EBA0ECCEC4CF017D00B
:107CBA000D0EDF5C14E00A0EDF5C11E0200EDF5CC3
:107CCA000EE30501626B636B646B616B0601FBEC8F
:107CDA004BF0DFCFEFFF0501656B0601DD2B0601D7
:107CEA00DD51006E016A000E001806E1010E01184E
:107CFA0003E1B487DD6BDE6B040EDB2A1BD70601BA
:107D0A00B45139E0B4A105D0060E006EBA0ECCEC1F
:107D1A004CF00601B4A305D0E70E006EB90ECCEC08
:107D2A004CF00601B4A505D0CB0E006EB90ECCEC12
:107D3A004CF00601B4A705D0AF0E006EB90ECCEC1C
:107D4A004CF00601B4A905D0900E006EB90ECCEC29
:107D5A004CF00601B4AD05D06F0E006EB90ECCEC36
:107D6A004CF00601B4AF05D0560E006EB90ECCEC3D
:107D7A004CF00601B46B37D8050EE15C02E2E16A09
:107D8A00E552E16E6EEF4BF0E0EC4CF0DBC6DFFF44
:107D9A00DF2A400EAFEC4BF001E1DF6A0601DC514D
:107DAA00DF5C01E120D80601DB51EA6A000FE96EC7
:107DBA00020EEA22FD0EDBCFEFFFDB2B400EDB5D6E
:107DCA0001E1DB6BDC51DB5D01E1B485FD0EDBCF4C
:107DDA0000F0016A00BE016800C0F3FF01C0F4FFB1
:107DEA00E5526EEF4BF0E0EC4CF00601DB51DC5D46
:107DFA001DE00601905105E030EC5EF031EC4EF0EA
:107E0A00F8D70601DC51D880DB5507E2DC51DB5D8F
:107E1A00C5EC4BF0DBC6DCF607D0400ED880DC554B
:107E2A00C5EC4BF00601DC6B30EC5EF0E5526EEF10
:107E3A004BF091EC4DF0E652DE6ADD6A020EDB6A27
:107E4A00030EDB6A060174EC4BF09FEC4CF0020E59
:107E5A00F3CFDBFF060190EC4BF004E1010E0118B1
:107E6A0001E1DE6B020EDB50DE6EDD6A74EC4BF074
:107E7A002C0824E074EC4BF00D0820E074EC4BF075
:107E8A009FEC4CF0030EF3CFDBFF060190EC4BF0B6
:107E9A0004E1010E011801E1DE6B020EDBCF02F0F4
:107EAA0002C003F0026A030EDB5000010224006ED6
:107EBA00000E0320016E00C0DEFFDD6E000EDFCF74
:107ECA001EF0010EDBCF1FF04D0E1E1802E1480E08
:107EDA001F1801E147D2520E1E1802E1530E1F1855
:107EEA0001E13DD2520E1E1802E1510E1F1801E1A6
:107EFA0033D2420E1E1802E1520E1F1801E129D296
:107F0A00540E1E1802E1510E1F1801E11FD2540E21
:107F1A001E1802E1530E1F1801E115D2530E1E1846
:107F2A0002E1430E1F1801E10BD2530E1E1802E1A3
:107F3A00510E1F1801E101D24D0E1E1802E1580E12
:107F4A001F1801E1F7D1530E1E1802E1450E1F1842
:107F5A0001E1EDD1430E1E1802E1410E1F1801E1A5
:107F6A00E4D14D0E1E1802E1510E1F1801E1DAD1BB
:107F7A004D0E1E1802E1520E1F1801E1D0D1320E29
:107F8A001E1802E1530E1F1801E1C6D1450E1E1834
:107F9A0002E1530E1F1801E1BCD1470E1E1802E17F
:107FAA00510E1F1801E1B2D1430E1E1802E1510E03
:107FBA001F1801E1A8D14B0E1E1802E1430E1F182B
:107FCA0001E19ED14C0E1E1802E1420E1F1801E17A
:107FDA0094D1440E1E1802E14E0E1F1801E18AD1F7
:107FEA00490E1E1802E14E0E1F1801E180D1420E01
:107FFA001E1802E1510E1F1801E176D14C0E1E180F
:10800A0002E1510E1F1801E16CD14C0E1E1802E15B
:10801A00530E1F1801E162D14E0E1E1802E1510ED5
:10802A001F1801E158D14E0E1E1802E1530E1F18F7
:10803A0001E14ED1430E1E1802E1530E1F1801E151
:10804A0044D14D0E1E1802E1450E1F1801E13AD126
:10805A00500E1E1802E1510E1F1801E130D1500EC8
:10806A001E1802E1540E1F1801E126D1500E1E18E7
:10807A0002E1530E1F1801E11CD14D0E1E1802E138
:10808A00530E1F1801E112D1470E1E1802E1500EBD
:10809A001F1801E108D1430E1E1802E1500E1F18E5
:1080AA0001E1FED0490E1E1802E1430E1F1801E13C
:1080BA00F4D0490E1E1802E1520E1F1801E1EAD04F
:1080CA00490E1E1802E1530E1F1801E1E0D0530EAB
:1080DA001E1802E1520E1F1801E1D6D0530E1E18C7
:1080EA0002E1530E1F1801E1CCD0530E1E1802E113
:1080FA00420E1F1801E1C2D0430E1E1802E1420EC1
:10810A001F1801E1B8D0430E1E1802E1520E1F18C3
:10811A0001E1AED04F0E1E1802E1420E1F1801E116
:10812A00A4D0570E1E1802E14D0E1F1801E19BD074
:10813A00520E1E1802E14D0E1F1801E192D0440E94
:10814A001E1802E1500E1F1801E189D04F0E1E18A9
:10815A0002E1500E1F1801E180D0490E1E1802E1FB
:10816A00500E1F1801E177D0580E1E1802E1540E66
:10817A001F186EE0540E1E1801E11F5067E0410EF1
:10818A001E1801E11F5060E0560E1E1801E11F5033
:10819A0059E0490E1E1801E11F5052E04F0E1E18F9
:1081AA0001E11F504BE0550E1E1802E1430E1F1845
:1081BA0043E0580E1E1802E1430E1F183AE0430E20
:1081CA001E1801E11F5033E0520E1E1801E11F5024
:1081DA002CE0580E1E1802E1520E1F1823E04D0E15
:1081EA001E1802E14C0E1F181AE0540E1E1802E166
:1081FA004C0E1F1811E0030EDB5001E0B6D0020E40
:10820A0050EC4CF050EC4CF0330E006EB90E12EC00
:10821A004DF001E3B9D0B6D0D2EC29F0B7D030ECAA
:10822A0028F0B4D07AEC45F0B1D0D5D8AFD037D950
:10823A00ADD07CEC45F0AAD0D2D8A8D0D4D9A6D05B
:10824A0006DAA4D021DAA2D024DAA0D0FFD89ED0B0
:10825A0078EC45F09BD044DB99D0B0DB97D0ABDA11
:10826A0095D08ADA93D076DA91D0F2EC45F08ED0B6
:10827A007EEC45F08BD0F0EC45F088D0F4EC45F07C
:10828A0085D0F6EC45F082D0F8EC45F07FD0FAECD8
:10829A0045F07CD0FCEC45F079D0FEEC45F076D088
:1082AA0000EC46F073D05AEC46F070D01DEC2BF07F
:1082BA006DD015EC31F06AD0F6EC30F067D0E3EC13
:1082CA0030F064D09DEC31F061D067EC27F05ED0DD
:1082DA0027EC32F05BD046EC32F058D058EC32F052
:1082EA0055D065EC32F052D078EC32F04FD009EC30
:1082FA0032F04CD01AEC32F049D090EC46F046D02D
:10830A00E7EC46F043D08DEC32F040D0A1EC32F0ED
:10831A003DD0D2EC32F03AD087EC5FF037D067EC40
:10832A0033F034D0ACEC33F031D049D92FD06CECE7
:10833A0030F02CD085EC2DF029D0E8EC33F026D0A3
:10834A0031EC34F023D009EC48F020D04EEC48F060
:10835A001DD098EC46F01AD09FEC46F017D0B1EC3D
:10836A0046F014D0C5EC2BF011D029EC4DF029ECD5
:10837A004DF00B0E006EB90E5CEC4BF0036E0B0E5B
:10838A00E15C02E2E16AE552E16E0350060174EC37
:10839A004BF00D080DE0B4510BE1520E006E016A6C
:1083AA00DF50001803E1DE52DD50011801E0B48FFE
:1083BA00DDC6DEF6040EE15C02E2E16AE552E16E38
:1083CA006EEF4BF00601E35105E03C0E006ECA0E5B
:1083DA00CCEC4CF012008AEC3CF0E7EF41F0E0EC18
:1083EA004CF07AEC4DF07DEC4BF0020E7FEC4DF048
:1083FA002BE1DF0412E12EEC4DF00AE0010E006ED3
:10840A00016ADB50001808E1020EDB50011804E192
:10841A00010EDBCFE3F601D0B48D020EAFEC4BF0C8
:10842A0012E12EEC4DF00AE0010E006E016ADB50FB
:10843A00001808E1020EDB50011804E1010EDBCF3F
:10844A00B7FE01D0B48DBEDFE8EF4CF068EC4BF01C
:10845A0044EC4CF0E66AA80EE66E060EE66EA9EC4F
:10846A004DF01BE1020EDB500CE1A851A91103E10A
:10847A00AA6BAB6B11D07684A8C6AAF6A9C6ABF6CE
:10848A000BD0A851A91103E1AF6BB06B05D076846C
:10849A00A8C6AFF6A9C6B0F695DFE8EF4CF091ECA6
:1084AA004DF07AEC4DF0BEEC4DF0020FBEEC4DF003
:1084BA00030FBEEC4DF0040FCFEC4CF00FE1DF5090
:1084CA00926E010EDB50936E020EDB50946E030E19
:1084DA00DB50956E040EDB50966E74DF050EE15C80
:1084EA0002E2E16AE552E16E6EEF4BF068EC4BF0A6
:1084FA00FD0EDB50100805E2100EF36EFD0EF3CFF1
:10850A00DBFFFC0EDB502BE0FD0EDB5065EC65F06B
:10851A00F3500601BE13F450BF13080EF36EFD0E9E
:10852A00F1EC4BF00DE2010EF36EFD0EDB5003E0B1
:10853A0097EC4BF0FDE1F350F31C0F0148173DD0C7
:10854A00FD0EDB500C0839E3A6EC4CF004E0E846DB
:10855A00FE0B0006FCE1E81C0F0149172ED0FD0EA8
:10856A00DB5065EC65F0F3CF00F0F4CF01F0001EAC
:10857A00011E00500601BE170150BF17080EF36E08
:10858A00FD0EF1EC4BF00CE2010EF36EFD0EDB502A
:10859A0003E097EC4BF0FDE1F3500F0148130DD0C7
:1085AA00FD0EDB500C0809E3A6EC4CF004E0E846AB
:1085BA00FE0B0006FCE10F0149136EEF4BF068EC6D
:1085CA004BF07AEC4DF0CFEC4CF009E1010EDBCF29
:1085DA00E6FFDFCFE6FF8ADFE552E552F3DEE5523A
:1085EA00E5526EEF4BF068EC4BF087EC4BF0010E66
:1085FA0065EC4BF0DAEC4BF026E1010EDB5002E1C0
:10860A00DF50896EE3EC4CF01EE1010EDB5002E113
:10861A00DF508A6EE3EC4CF016E1010EDB5002E10A
:10862A00DF508B6EE3EC4CF00EE1010EDB5002E101
:10863A00DF508C6EE3EC4CF006E1010EDB5002E1F8
:10864A00DF508D6EBFDEE552E5526EEF4BF084507F
:10865A00E66EE66A8350E66EE66A8250E66EE66A7F
:10866A008150E66EE66A8050E66EE66AEE0E006EAD
:10867A00B80E5CEC4BF0036E0D0EE15C02E2E16AAF
:10868A00E552E16E03501200440E006ECA0ECCEFA2
:10869A004CF091EC4DF0DF6A010EF36EDB6E020EC8
:1086AA00DB6AEC0E006EB80ECCEC4CF09DBCFED72B
:1086BA00DF6ADFCF00F0100EE76E0018E8AE02D0D6
:1086CA00E73402D0E750005C3EE2010EDB500601BF
:1086DA00BE150001006E020EDB500601BF15000137
:1086EA00016E005001101EE0DFCFE9FFEA6AE9BE21
:1086FA00EA6839EC4CF0EECFE6FFEFCFE6FFDFCFCA
:10870A0000F0016A00BE01686BEC4DF0E10E026EEA
:10871A00B80E54EC4CF0070EE15C02E2E16AE55255
:10872A00E16E0550010EDBCF00F0020EDBCF01F047
:10873A00D89000360136010E00C0DBFF020E01C0E0
:10874A00DBFFDF2AB6D7410E006ECA0ECCEC4CF026
:10875A00E8EF4CF0E0EC4CF087EC4BF0A9EC4DF074
:10876A0009E16BEC4CF005E28BEC4BF0020EDBCF2F
:10877A00EFFF28DEE8EF4CF0E0EC4CF087EC4BF032
:10878A00030E7FEC4DF015E16BEC4CF005E28BEC3F
:10879A004BF0020EEFCFDBFF020E50EC4CF0D70E7F
:1087AA00006EB80ED3EC4CF002E2E16AE552E16EDB
:1087BA000350E8EF4CF0C2EC4DF001E08FD0020E0E
:1087CA00DB50010801E287D0010EDB50070801E205
:1087DA0082D0410EAFEC4BF016E1020EDB500AE1FB
:1087EA00A0EC4BF003E097EC4BF0FDE1F350F31CE7
:1087FA00921673D0A0EC4BF003E097EC4BF0FDE13E
:10880A00F35092126AD0420EAFEC4BF016E1020E10
:10881A00DB500AE1A0EC4BF003E097EC4BF0FDE1F2
:10882A00F350F31C931659D0A0EC4BF003E097ECED
:10883A004BF0FDE1F350931250D0430EAFEC4BF0E6
:10884A0016E1020EDB500AE1A0EC4BF003E097ECD4
:10885A004BF0FDE1F350F31C94163FD0A0EC4BF023
:10886A0003E097EC4BF0FDE1F350941236D0440E3E
:10887A00AFEC4BF016E1020EDB500AE1A0EC4BF034
:10888A0003E097EC4BF0FDE1F350F31C951625D06D
:10889A00A0EC4BF003E097EC4BF0FDE1F35095129E
:1088AA001CD0450EAFEC4BF016E1020EDB500AE18C
:1088BA00A0EC4BF003E097EC4BF0FDE1F350F31C16
:1088CA0096160BD0A0EC4BF003E097EC4BF0FDE1D1
:1088DA00F350961202D0B48D01D074DDE8EF4CF05B
:1088EA0068EC4BF044EC4CF0B8EC4DF0050EC8ECDB
:1088FA004CF0010FCFEC4CF05FE1010EDB500708A2
:10890A0047E3410EAFEC4BF009E1A0EC4BF003E07A
:10891A0097EC4BF0FDE1F350801433D0420EAFECEC
:10892A004BF009E1A0EC4BF003E097EC4BF0FDE1D2
:10893A00F350811426D0430EAFEC4BF009E1A0ECC2
:10894A004BF003E097EC4BF0FDE1F350821419D0A1
:10895A00440EAFEC4BF009E1A0EC4BF003E097ECCE
:10896A004BF0FDE1F35083140CD0450EAFEC4BF005
:10897A000FE1A0EC4BF003E097EC4BF0FDE1F35074
:10898A008414E76E020EE7CFDBFFDB5008E002D06B
:10899A00B48D12D0010EF36E020EF3CFDBFF020E7E
:1089AA0050EC4CF0CE0E006EB80ED3EC4CF002E256
:1089BA00E16AE552E16E0350E8EF4CF0C2EC4DF08B
:1089CA0001E08FD0020EDB50010801E287D0010ED0
:1089DA00DB50070801E282D0410EAFEC4BF016E102
:1089EA00020EDB500AE1A0EC4BF003E097EC4BF0EF
:1089FA00FDE1F350F31C891673D0A0EC4BF003E0B1
:108A0A0097EC4BF0FDE1F35089126AD0420EAFECBD
:108A1A004BF016E1020EDB500AE1A0EC4BF003E04A
:108A2A0097EC4BF0FDE1F350F31C8A1659D0A0ECF9
:108A3A004BF003E097EC4BF0FDE1F3508A1250D073
:108A4A00430EAFEC4BF016E1020EDB500AE1A0EC4C
:108A5A004BF003E097EC4BF0FDE1F350F31C8B165F
:108A6A003FD0A0EC4BF003E097EC4BF0FDE1F35064
:108A7A008B1236D0440EAFEC4BF016E1020EDB50EF
:108A8A000AE1A0EC4BF003E097EC4BF0FDE1F35068
:108A9A00F31C8C1625D0A0EC4BF003E097EC4BF0BE
:108AAA00FDE1F3508C121CD0450EAFEC4BF016E1F1
:108ABA00020EDB500AE1A0EC4BF003E097EC4BF01E
:108ACA00FDE1F350F31C8D160BD0A0EC4BF003E044
:108ADA0097EC4BF0FDE1F3508D1202D0B48D01D02A
:108AEA0071DCE8EF4CF0E7EF41F0E7EF41F0E7EF38
:108AFA0041F0E0EC4CF0E65274EC4DF00AEC4DF02B
:108B0A0062E1D950020F9BEC4BF0720ED880EE5402
:108B1A002E0EED543DE3D950020F9BEC4BF0EE5074
:108B2A00ED101FE003680468056A2D0EE76E020E59
:108B3A00DBCF06F0030EDBCF07F0E7500626000E68
:108B4A000722086A0650035C006E07500458016E3B
:108B5A0008500558026E020E00C0DBFF030E01C06A
:108B6A00DBFF010EDB50070813E3410EAFEC4BF0BD
:108B7A0002E1DF6A0FD0420EAFEC4BF002E1080EC1
:108B8A0005D0430EAFEC4BF003E1100EDF6E02D0BE
:108B9A00B48D19D0010EDB50DF24E96EEA6A93EC3A
:108BAA004CF0ADEC4CF0010EDB50DF244AEC4CF0FB
:108BBA00EF0407E1010EDB50DF244AEC4CF0020E11
:108BCA00EF6EE7EC41F0040EE15C02E2E16AE55285
:108BDA00E16E6EEF4BF0E7EF41F0E7EF41F0E7EFC0
:108BEA0041F0E7EF41F0E7EF41F0E7EF41F0E7EF5F
:108BFA0041F0E7EF41F068EC4BF0070EE12402E3A5
:108C0A00E168E652B4EC4CF0030EC8EC4CF00AEC06
:108C1A004DF043E1DECF01F5DDCF02F5020EDBCFE9
:108C2A0009F5030EDBCF0AF5040EDB6A030EF36EB9
:108C3A00040EF1EC4BF02FE2010EBCEC4BF0030EEC
:108C4A0034EC4DF0010EE66ED950B4EC4DF065EC03
:108C5A004BF0E76E060EE7CFDBFF0601B4511DE1CC
:108C6A00050EDB5018E1060EDB5015E199EC4CF0CD
:108C7A00010EE926050EEA22DECFEEFFDDCFEDFF7B
:108C8A0099EC4CF0090EE926050EEA22ADEC4CF0FF
:108C9A00040EDB2ACBD7E7EC41F0070EE15C02E2D7
:108CAA00E16AE552E16E6EEF4BF0E0EC4CF0B8ECA5
:108CBA004DF0010E7FEC4DF00DE1DF5007E0F00EB4
:108CCA009314936E0501010E006F02D00501006B2B
:108CDA00E7EC41F0E5526EEF4BF0D9CFE6FFDACF81
:108CEA00E6FFE1CFD9FFE2CFDAFFE652DF6AFF0EF5
:108CFA00DF5C0AE2E868E85005E0E80600D000D048
:108D0A0000D0F9D7DF2AF3D7E552E552E5CFDAFFEB
:108D1A00E7CFD9FF1200F29EF29C6592656ADDDF09
:108D2A000FEF00F01200F29EF29C6592656AD5DFA1
:108D3A00FF0012008050080B01E0010EE66EE66AA1
:108D4A00C80E006EB80ED3EC4CF002E2E16AE552AE
:108D5A00E16E0350E7EF41F068EC4BF0060EE124B8
:108D6A0002E3E168E652B4EC4CF0070E65EC4BF016
:108D7A00010EE66ED950040F7DEC4BF0010E34EC77
:108D8A004DF00601B45116E1DFCF1DF5010EDBCF20
:108D9A001EF5020EDBCF1FF5030EDBCF20F5050E05
:108DAA00DB5006E1040EDB5002E0898601D0899689
:108DBA00E7EC41F0060EE15C02E2E16AE552E16E9F
:108DCA006EEF4BF068EC4BF0100EE12402E3E16821
:108DDA00E652E16EE66AD950010F7DEC4BF0E66A85
:108DEA003AEC4DF0B8EC4DF0010EC8EC4CF0040F23
:108DFA007DEC4BF0020EC8EC4CF0B4EC4DF0C8EC34
:108E0A004CF00A0F7DEC4BF0060EC8EC4CF0060F46
:108E1A007DEC4BF0070EC8EC4CF00E0F7DEC4BF0DE
:108E2A00040EC8EC4CF00F0F7DEC4BF0050E65EC10
:108E3A004BF0010EDBCF00F0016A00BE01686BEC5B
:108E4A004DF0BC0E026EB80E54EC4CF0050EE15C0F
:108E5A0002E2E16AE552E16E0550DFCFE6FFE66A1B
:108E6A00B00E006EB80ED3EC4CF002E2E16AE552A5
:108E7A00E16E0350040EDBCFE6FF050EDBCFE6FF03
:108E8A00A40E006EB80ED3EC4CF002E2E16AE55291
:108E9A00E16E0350020EDBCFE6FF030EDBCFE6FFE7
:108EAA00980E006EB80ED3EC4CF002E2E16AE5527D
:108EBA00E16E0350D9500A0F9BEC4BF074EC4CF066
:108ECA008B0E006EB80E12EC4DF002E2E16AE5522A
:108EDA00E16E0350D950060F9BEC4BF074EC4CF04A
:108EEA007E0E006EB80E12EC4DF002E2E16AE55217
:108EFA00E16E03500E0E50EC4CF0720E006EB80E7E
:108F0A00D3EC4CF002E2E16AE552E16E03500F0E37
:108F1A0050EC4CF0660E006EB80ED3EC4CF002E248
:108F2A00E16AE552E16E0350E7EC41F0100EE15CB4
:108F3A0002E2E16AE552E16ECCD3C5DB120EE1240E
:108F4A0002E3E168E652E16E110EDB6AF36EDBCFF3
:108F5A00F4FFE850F45C03E2EFEC4CF0F7D71CECBA
:108F6A004DF002E2E16AE552E16E0050110EDB6A51
:108F7A00100EF36E110EF1EC4BF02DE217EC4DF0E2
:108F8A00EF50006E016A013404E200508008000EBE
:108F9A00015421E317EC4DF0EFCF04F0200E045CEE
:108FAA001AE317EC4DF0EF50E66E180E0201016A53
:108FBA00FA25006EFB511EEC4CF0DB50D924B6DBCF
:108FCA00EF50E66E020E016AFC25006EFD511EECA2
:108FDA004CF0DB2ACDD7110EDB50E824180FFAC269
:108FEA00E9FFFBC2EAFFEF6E110EDB50E824020F25
:108FFA00FCC2E9FFFDC2EAFFEF6E120EE15C02E27B
:10900A00E16AE552E16E65D35EDB130EE12402E309
:10901A00E168E652E16E110EDB6A120EDB6A110E8E
:10902A00F36E120ED9DB08E2BEEC4CF0120EAEEC77
:10903A004DF0120EDB2AF3D7100E99DB6CD895ECA3
:10904A004DF0E76E110EE7CFDBFFE668FB0EE66E2A
:10905A00E66A3FEC4DF054EC62F0006E080EE15CFB
:10906A0002E2E16AE552E16E00506FDBC1EC60F0AA
:10907A00006E080EE15C02E2E16AE552E16E005020
:10908A00E7EC41F0130EE15C02E2E16AE552E16EBF
:10909A0020D319DB120EE12402E3E168E652E16E05
:1090AA00110EDB6AF36EDBCFF4FFE850F45C03E2E7
:1090BA00EFEC4CF0F7D71CEC4DF002E2E16AE55216
:1090CA00E16E0050DF50006E016AD890015004E64C
:1090DA00800E005C000E015803E2200EDF5C06E2FF
:1090EA001E0E006EBA0ECCEC4CF00CD0DBEC4CF041
:1090FA00610E006EB80ED3EC4CF002E2E16AE55262
:10910A00E16E0350E7EC41F0120EE15C02E2E16A23
:10911A00E552E16EDED2E0EC4CF0DF6A4DDBEF6A3D
:10912A0046EC4DF002E1B4890CD0D9DA2C080BE0F8
:10913A0083EC4DF002E2E16AE552E16E035006016A
:10914A00B48B000E28D0E7DA04E1010E011801E120
:10915A00DE6B0D0E70EC4DF009E02C0E016EBFDADD
:10916A00015C04E0FB0EDB50DF5C02E3DF5013D04E
:10917A00B6DAE66E21DBE552E750EF6ECCDA04E1AF
:10918A00010E011801E1DE6BDF2AFC0EDB2AFD0E5F
:10919A00E0E3DB2ADED7E5529CD295DA090EE12418
:1091AA0002E3E168E652E16E080EDB6A46EC4DF036
:1091BA0005E1FA0EDB5021E1B4891FD090DA2C08C0
:1091CA000EE0FA0EDB5009E183EC4DF002E2E16AAF
:1091DA00E552E16E03500601B48B020E25D19BDAEB
:1091EA0004E1010E011801E1DE6B0D0E70EC4DF089
:1091FA0006E1FA0EDB5001E1B489030E15D12D0EFA
:10920A0070EC4DF020E1040E5CDB1DE0050E026EF1
:10921A00FD0EDB50025C17E0FD0EDB0401E1CAD053
:10922A00030E28DB01E1C6D0070E4BDB01E1C2D0F9
:10923A00010EF36E080EF3CFDBFF6DDA04E1010EC7
:10924A00011801E1DE6B040E15DB09E0050E39DBBE
:10925A0006E00A0E8CDAF1D895EC4DF036D0DE51E4
:10926A00BFDBEFCF00F0000E00C0DFFF010EDB6AAC
:10927A00020EDB6A030EDB6A050EFCDA1FE1000E42
:10928A00DFCFE6FF010EDBCFE6FFD4EC64F0E55258
:10929A00E552F3CF00F0F4CF01F0026A036A01AE9F
:1092AA0002D00268036800C0DFFF010E01C0DBFFC5
:1092BA00020E02C0DBFF030E03C0DBFF06012BDA3E
:1092CA0004E1010E011801E1DE6B080EDB5044E0F7
:1092DA00FD0EDB5007E1BBEC4DF0800E4BDA000EC1
:1092EA00EE5414E3020EC6DA07E1BBEC4DF0000EB1
:1092FA00EE54800E3FDA0AE3060EE3DA09E1BBEC2C
:10930A004DF0000E37DA800EEE5402E2060152D01A
:10931A00F4D99DDA080EDB5055E0040EDBCF1CF0C1
:10932A00050EDBCF1DF0060EDBCF1EF0070EDBCFDE
:10933A001FF0216822682368246843EC64F0040E55
:10934A0018C0DBFF050E19C0DBFF060E1AC0DBFFD3
:10935A00070E1BC0DBFF36D0FD0EDB5007E1BBEC6E
:10936A004DF07F0EEE54000E05DA23E3FD0EDB040A
:10937A0004E13CDB000EFED91CE3020E7BDA04E1B9
:10938A0035DB7F0EF7D915E3030E9BDA04E12EDBFA
:10939A00FF0EF0D90EE3060E026EFD0EDB50025CE4
:1093AA000CE124DBFF0EEE54FF0EEE547F0EEE545A
:1093BA0004E20601B48D010E37D0070E5BDA02E033
:1093CA009CD945DAFD0EDB50070A21E0010A17E0B5
:1093DA00050A11E0010A0FE0030A08E0050A06E09F
:1093EA00010A04E0050A02E0040E1ED002DA040EA5
:1093FA00DBCFEFFF18D04BDBDBCFEDFF14D047DB21
:10940A00DBCFEEFF060EDBCFEEFF070E0AD0F1D957
:10941A00DFCFEEFF010EDBCFEEFF020EDBCFEEFF5A
:10942A00030EDBCFEEFF000E006E090EE15C02E2D6
:10943A00E16AE552E16E00504CD1BDDAE652BCD980
:10944A00EE6AEE6AEE6AEE6A010EDB6AFB0EDB502A
:10945A00F36E010EC1D94FE20601DE51C1DAEFCF38
:10946A00DFFF300EDF5C42E3DF5039083FE3A4D967
:10947A00EECF00F0EECF01F0EECF02F0EFCF03F027
:10948A000A0E216E226A236A246A00C01CF001C0F7
:10949A001DF002C01EF003C01FF043EC64F018C0B8
:1094AA0000F019C001F01AC002F01BC003F0300E20
:1094BA00DF5C046E056A066A076AE85000260550F2
:1094CA000122065002220750032276D900C0EEFF7D
:1094DA0001C0EEFF02C0EEFF03C0EEFF06011BD97A
:1094EA0007E1010E011804E1DE6B02D0000E04D080
:1094FA00010EDB2AABD7010EE552E552EAD006018E
:10950A00AE51E66EE66A2E0E006EB80E47DA02E239
:10951A00E16AE552E16E035012000101715108E05F
:10952A00010E006E6550020B01E0010E005C17E1AE
:10953A00E5D90BE169516A1111E18C86A00E696FB8
:10954A000F0E6A6F010E6B6F120069516A1152E1B8
:10955A008C96A00E696F0F0E6A6F6B6B1200710505
:10956A0009E0020E715D06E0040E715D03E0100E63
:10957A00715D17E1C3D90BE169516A1111E18C865A
:10958A00200E696F4E0E6A6F010E6B6F12006951E1
:10959A006A1130E18C96200E696F4E0E6A6F6B6B02
:1095AA001200200E715D26E1A9D907E169516A11FD
:1095BA0021E18C86E3D9010E15D06B0507E16951CB
:1095CA006A1118E18C96DAD9020E0CD0020E6B5D84
:1095DA000BE169516A110EE18C86A00E696F860E45
:1095EA006A6F030E6B6F120069516A1103E18C9660
:1095FA00C5D96B6B120067D8B5D9E8AE02D0003472
:10960A0003D0E750D880005423E3FC0EDB5010E06F
:10961A00E8D8E9BEEA68A2D804E0E846FE0B0106EB
:10962A00FCE1006EDED8E9BEEA687EDAEF1210D0FD
:10963A00D8D8E9BEEA6892D804E0E846FE0B0106EB
:10964A00FCE1E81C006ECDD8E9BEEA686DDAEF16D7
:10965A0040D039D887D9E8AE02D0003403D0E750D9
:10966A00D880005423E3FC0EDB5011E1BAD8E9BEDE
:10967A00EA6874D804E0E846FE0B0106FCE1E81C3F
:10968A00006EAFD8E9BEEA6855DAEF160FD0A9D84E
:10969A00E9BEEA6863D804E0E846FE0B0106FCE18D
:1096AA00006E9FD8E9BEEA6845DAEF1212D0016E61
:1096BA00026A00C0E6FFE66E02C0E6FF6CEF63F0E6
:1096CA00E66E3AEF4DF072D9E1CFD9FFE2CFDAFF79
:1096DA001200E552E5CFDAFFE7CFD9FF1200DE51DB
:1096EA007FD9EF501200A951E96EEA6AFFEF4CF0F8
:1096FA00E66E000EDA20E66E1200D9CFE9FFDACF65
:10970A00EAFF1200E652E652B8EF4DF0DECFE9FF6B
:10971A00DDCFEAFF1200DE2BDE51006E016A000E79
:10972A0000181200D890F336E8061200E96E000E0F
:10973A00DA20EA6E1200010EF36EDB501200EA2202
:10974A00EECF2CF0EFCF2DF0120030D9100EE66ECE
:10975A003FEF4DF0006EDF50005C1200D00EE9269C
:10976A00050EEA22EF50016E010E01521200E66E5A
:10977A00DBEF4CF0EE54000EEE54000EEE541200E5
:10978A00DF6EDFCFE6FFDC51016A000F006E020ECA
:10979A0001229CD9E9EC5DF095EF4DF0DECF00F0A7
:1097AA00DDCF01F0D89001501200E76E010EE7CF2D
:1097BA00DBFF0601B4511200FC0EDBCFE9FFFD0E00
:1097CA00DBCFEAFF1200EA22EECF2EF0EFCF2FF026
:1097DA00120010D9E8061200DBCFF4FFF350F45C54
:1097EA001200FD0EDBCFE9FFEA6A1200DD51F5EF48
:1097FA004CF0FB0EDBCFE9FFFC0EDBCFEAFF1200D9
:10980A00EA22EE50EFCFEAFFE96E00501200036E33
:10981A00050EE15C1200A951EA6A310FE96E0E0EDB
:10982A00EA22EF500E01EA6AAC25E96EAD51EA224E
:10983A0012000122110EDB50E8240024E96E000E0A
:10984A000120EA6EE552E750EF6E110E1200040E87
:10985A00EECFDBFF050EEECFDBFF060EEECFDBFF12
:10986A00070EEECFDBFF1200C5D8000EE926010E67
:10987A00EA221200006EFD0EDB50005C1200E65276
:10988A00E652E652020EDB6A1200EA6A290FE96E14
:10989A00010EEA221200DBCFE6FFE66A1200036E2F
:1098AA00046A02C0E6FFE66E04C0E6FF6CEC63F0F1
:1098BA00056E1200020EDBCF2CF0030EDBCF2DF06B
:1098CA001200016EFD0EDB50015C1200DECF00F0CB
:1098DA00DDCF01F0000E005C100E01581200EECF31
:1098EA00E6FFEECFE6FFEECFE6FFEFCFE6FF120090
:1098FA00070EB7152C6E010E2C52120005016907CE
:10990A00000E6A5B6B511200000EE926030EEA2272
:10991A001200010EDBCFE9FFEA6A12006BD8410E92
:10992A00E926010EEA221200040EDB28E96EEA6A31
:10993A00FFEF4CF0E66EE66AD4EC64F0E552E552CD
:10994A001200FD0EDB50F80F006E010E00521200DD
:10995A00020EDBCFEEFF030EDBCFEDFF1200E16E4E
:10996A00B8EF4DF0FD0EDBCF00F0190EE76E0018D0
:10997A001200D9CF00F0DACF01F01200100E696F91
:10998A00270E6A6F12009CDEE66AD95012008FDE3B
:10999A0095EF4DF0ADDE010E7FEF4DF088DE0CEF56
:1099AA004CF0A1DE010EE9260E0E1200D9CFE6FF19
:1099BA00DACFE6FF120087DEE6521200010ED7DE8A
:1099CA007FDEDAEF4BF0ACD884D68DDE790EE9264D
:1099DA000E0E1200CEDF110EBCD8110EDB2A1200B9
:1099EA00EA6A000FE96E030EEA221200BFD8FF0EE0
:1099FA00EE541200D890E936EA361200110EE92622
:109A0A00050E9DDE83DE010E1200A9D87FEF4DF010
:109A1A006ADE490EE9260E0E120049DE036E070EB3
:109A2A00E15C1200110EDB50D9249BEF4BF08DDE66
:109A3A00B8EC63F0006E080EE15C1200C4DE2C5034
:109A4A002E5C2D502F581200030E25DF020E50EF08
:109A5A004CF0D950010F6ADEEE50ED10120030DEE4
:109A6A00E76E050EE7CFDBFF1200D2EC48F058D8BC
:109A7A00E5521200E66AE66AF80EE66EE66AE66AF9
:109A8A0012000D0E006E06012ADE005C1200B1DE25
:109A9A00040EDBCFEEFF050E120095DE2E502C18B9
:109AAA001200110EE926050EEA22120026DEEE50F9
:109ABA00ED10120022DE010EEE1812001EDE020E5A
:109ACA00EE1812001ADE030EEE18120000C0E6FFAE
:109ADA0001C0E6FF1200006E02DE005C120012DE18
:109AEA00050E51DF010FBEEF4DF00CDE010E4BDF0C
:109AFA00010F1200E5DD0601B4511200F0DDE66E39
:109B0A00E66A3A0E006EB80ED3EF4CF05EDF17DE4F
:109B1A0048DFEA222C5012004EDFE652E6521200CB
:109B2A00E552E552E552120065DF9E0EE926050E62
:109B3A0005EF4CF05FDF6C0EE926050E05EF4CF0E1
:109B4A0067DFFDDDD6EF4CF0030E1DDF020FCFEF0E
:109B5A004CF0DB500F01D924E9DDEF6A1200020F45
:109B6A00C7DD030E1200E66ADBEF4CF0C6DDD880D3
:109B7A001200BEDD010EC8EF4CF01DDFB0DF020F90
:109B8A00CFEF4CF079EC53F0A098636A626A0F0148
:109B9A00266B41EC54F002E2E16AE552E16E0050B4
:109BAA000F0105EC54F0DF6ADF50006E016A0C0EFB
:109BBA00005C000E015810E2DF50040DF3CFE9FFFC
:109BCA00F4CFEAFF000EE926040EEA22EE6AEE6AF4
:109BDA00EE6AEE6ADF2AE8D7658C0F01386B659862
:109BEA00659C62A607D062960101886B8D6B8E6BAD
:109BFA008F6BF7D70101010EA16FA26FA36BA46B44
:109C0A00956BDF6A030EDF5C11E2EA6ADF346EEC01
:109C1A0054F0EA22EE6AED6AEA6ADF3475EC54F02F
:109C2A00EA22EE6AED6AB7EC53F0ECD70101080EAE
:109C3A007E6F040E7F6F0F01160E266F0401300E21
:109C4A00026F040E036F400E016F840E006F010154
:109C5A00726B716B7CEF53F079EC53F082BE06D0D5
:109C6A00656A0F01366B0101716B7CD0010171517C
:109C7A000CE1656A0F01366B05EC54F065B602D04B
:109C8A006586FCD70101010E716F71050AE165BA9B
:109C9A0008D0626A0F01366B368136890101020EDD
:109CAA00716F6250040B06E00F013651040B02E09B
:109CBA00629459DB65B256D06250010B09E00F017C
:109CCA003651010B05E05EDF0101040E716F6290EF
:109CDA006250100B06E00F013651100B02E033DB25
:109CEA00629862AC15D00F0136AD0AD00CEC54F074
:109CFA00730E83EC53F002E2E16AE552E16E005022
:109D0A00629C01019F5101E09F079F5101E1F3D835
:109D1A006250200B05E00F013651200B01E002DBF7
:109D2A006250020B14E00F013651020B10E00CECEA
:109D3A0054F0E6687F0EE66E01EC62F0006E060EE5
:109D4A00E15C02E2E16AE552E16E0050636A040EE8
:109D5A000101E76E7119E8AE02D0E73402D0E7508C
:109D6A00715D02E2A19834D00F0136A730D0DF6AC4
:109D7A00040EDF5C2CE262A62AD064CF96F10101C0
:109D8A009651780BE842E842E842976F629696B598
:109D9A0004D097517CEC54F003D0975181EC54F0E5
:109DAA00EA22EF70975102E1F0DA0FD0000EE66E68
:109DBA00E66A960EE66E010EE66E720E83EC53F0BC
:109DCA0002E2E16AE552E16E0050DF2AD1D7A1989A
:109DDA007CEF53F06BEC54F0FC0EDBA403D0E66A84
:109DEA00F5EC53F0FC0EDBA204D0010EE66EF5ECA6
:109DFA0053F0FD0EDB50016A260F006E0F0EEFECDA
:109E0A0053F08BEC53F0FC0EDBCFEFFFE5527CEF07
:109E1A0053F06BEC54F0FC0EDB5003E07EEC53F095
:109E2A0002D0A8EC53F0DBEC53F0D9CFE9FFDACF3C
:109E3A00EAFFEE50ED1003E1F36AF46A28D08BECE6
:109E4A0053F090EC54F0FA0EDBCFEEFFFB0EDBCFB3
:109E5A00EDFF8BEC53F0EE52F90EDBCFEFFF400E25
:109E6A0086EC54F0880E95EC54F0FC0EDB5003E0BF
:109E7A007EEC53F002D0A8EC53F0EA22EF74DECF66
:109E8A0000F0DDCF01F000C0F3FF01C0F4FFE5529E
:109E9A007CEF53F06BEC54F0FD0EDB5003E14AEC1F
:109EAA0054F009D0ADEC53F01FEC54F0ADEC53F084
:109EBA00010F1FEC54F0E5527CEF53F051EC54F0D3
:109ECA0065A817D064EC54F0400EEE16EE6AEE6AFE
:109EDA00EE6A64EC54F0EE7C7EEC53F0EA22EF7406
:109EEA00400E006E64EC54F00050EF1664EC54F02F
:109EFA00EF7C3BEF54F00101A15127E1010EA16F64
:109F0A00A25123E1010EA26F020E855D09E190ECD8
:109F1A0053F0EE52EF6A90EC53F0C80EEF6E120057
:109F2A00850513E1986B9DEC53F0EE52400EEF6EEF
:109F3A009DEC53F02BEC54F09DEC53F0840EEF6E35
:109F4A00010E986FCDDB800EEF6E12000101A36B3C
:109F5A00A46B020E855D07E18AEC54F0A2EC53F083
:109F6A001AEC54F010D089510401365D01018A516E
:109F7A000401375904E236C489F137C48AF15CD83E
:109F8A00CADBDBDBC8DBC80EEF6E12006BEC54F0E9
:109F9A00000EDE6E040EDD6EDBDB040DF4CF01F085
:109FAA00D9CFE9FFDACFEAFFF350EE260150ED22CE
:109FBA00ADDBEF9EFC0EDB5002E1C5DB01D099DB85
:109FCA00EA22DECFEEFFDDCFEDFFA0DBEF9C9EDBCA
:109FDA00040EE926000EEA22EF8CE55288D3659832
:109FEA00010188BF0DD08DAF09D0020E856FA45133
:109FFA0001E1ACDF0101A26BA16B12004AEF54F040
:10A00A00040130AF0DD00101010E856FA35101E1AA
:10A01A009DDF0101A26BA16BA0510DE180EF4FF012
:10A02A000101020E856F5CDB840EEF6EA26BA16BE1
:10A03A00A05101E160DF120057DB400EDF6E010123
:10A04A00895D000E8A590AE289C1DFFF845102E163
:10A05A00010E03D0840502E1020E846FDF50016A0B
:10A06A00E850895D896F01508A598A6F54DBEE5234
:10A07A00DFCFEFFF380E926F040E936F88B10DD0C9
:10A08A00DF5017E086C1F6FF87C1F7FF862B000E67
:10A09A0087230800F5507DDBF3D7DF500AE086C13D
:10A0AA00E9FF87C1EAFF862B000E8723EF5071DB99
:10A0BA00F4D71DD36BEC54F03BDBEE52EFCFDFFF4E
:10A0CA00DFCF00F0005001018E5D000E8F5902E2D1
:10A0DA008EC1DFFFDF50006E016AE8508E5D8E6F21
:10A0EA0001508F598F6F010EDB6ADF50F36E010E3C
:10A0FA00DBCFF4FFF350F45C16E2010EDB50EA6AA0
:10A10A00380FE96E040EEA22EF50E66E8BC1E9FFC2
:10A11A008CC1EAFF8B2B000E8C23E552E750EF6EC1
:10A12A00010EDB2AE2D7000ED8808E55000E8F551D
:10A13A000DE2EBDB02DBFCDAEF50400B03E175DBEF
:10A14A00C80E02D072DB880EEF6E12D0C9DA840E06
:10A15A00EF6E9051911107E005D091C1FAFF01010C
:10A16A009051F96EFADF01018D9FA05101E1C3DE22
:10A17A00E552BDD2B9DA0101888F7EDB02E2E16ADB
:10A18A00E552E16E0050300EE66EE66AE66A000EAF
:10A19A00E66E040EF1DA02E2E16AE552E16E00507F
:10A1AA00658CDF6A030EDF5C02E2DCDAFBD7010EA4
:10A1BA00E66EE66AE66A730EE66E010EDDDA02E222
:10A1CA00E16AE552E16E0050659C0101080E7E6F5E
:10A1DA00040E7F6F000E746F040E756F74C176F1F2
:10A1EA00776F32C472F1725102E1100E10D0010E73
:10A1FA00E66EE66A720EE66E010EE66E010E7EDA13
:10A20A0002E2E16AE552E16E00500101200E716F2F
:10A21A006ED2800E0401305D4EE10101C00E886FDE
:10A22A0004013351030A25E0010A09E0030A41E166
:10A23A000101500E866FC90E876F120E34D032514B
:10A24A00F66EF76AD890F636F736A50EF626C90ED8
:10A25A00F7220900F5CF86F10A00F5CF87F1020E41
:10A26A000101DCDAF5CF89F1030ED8DAF5CF8AF1EC
:10A27A001200040E325D1AE2010188810401325192
:10A28A00E96EEA6AD890E936EA36F60EE926020E4F
:10A29A00EA22EECF86F1EDCF87F186C1E9FF87C1C9
:10A2AA00EAFFEF500101896F8A6B12000101886B86
:10A2BA0012000101886B120009DB0401386B396B4B
:10A2CA0030511F0B020A11E0030A0CE0010A1EE1D9
:10A2DA000101888F040138810101940517E1040105
:10A2EA00388314D00101888F11D00101888F0401AD
:10A2FA0034BF02D0DADA01D0DDDA58DAE3DA06E07E
:10A30A0005DAEF50040B02E0010E386F010188AF45
:10A31A0007D0380E866F040E876F8881020E896F08
:10A32A00E552E5D10F0126A10CD002DAEF508008E0
:10A33A0007E1F1D9EF50840803E1FAD98C0EEF6EE8
:10A34A002691629A12000F01368562986582010190
:10A35A00010E956F31DA750ED1D902E2E16AE55242
:10A36A00E16E005012000101956B26DA740EC6D90F
:10A37A0002E2E16AE552E16E005065920F013695FC
:10A38A0062A402D06294FCD71200AED901012D0E4C
:10A39A009F6FFD0E961539E17E0E9615E8407F0BEC
:10A3AA00040DF3CF74F1F4CF75F1000E7427040E87
:10A3BA00752374C176F175C177F17675B9D9EF5005
:10A3CA003C0BE842E8420D081EE1DF6A080EDF5C3A
:10A3DA0016E2AED9020EE926000ED5D9EF50E66E86
:10A3EA00DF50EA6A300FE96E040EEA22E552E750BE
:10A3FA00EF6E9ED990DAEE2AEF22DF2AE7D798D9B4
:10A40A0025DA09D807D027D805D0FD0E96150408F5
:10A41A0001E130D86CD10101846BA06BA36BA46BF2
:10A42A00986B856B78D9EF9E7E7575D9EF9E7E7590
:10A43A00FCD9EF9E886B896B8A6B8D6B8E6B8F6BE9
:10A44A0055D8BAD9030E5AD902E2E16AE552E16E49
:10A45A000050F4EF4FF0020E0101855D02E15FEF5B
:10A46A0050F0856B985104E13BD98C0EEF6E1200C7
:10A47A00986B120039D94FD9EF50400B01E0010E09
:10A48A00DF6E01017E75080E715D0BE132C438FF83
:10A49A000F01385103E00101100E02D00101040E30
:10A4AA00716F850513E137D948D9C6DD020E01015E
:10A4BA00845D03E130D9840E07D0DF5003E12BD944
:10A4CA00C80E02D028D9880EEF6E0FD08DAF0CD0EF
:10A4DA009051911107E005D091C1FAFF0101905105
:10A4EA00F96EFADF01018D9F856B01D104013051AC
:10A4FA00600BE842E842E842E842E842000901E02B
:10A50A00120031510C0A4AE00B0A3FE00C0A31E012
:10A51A00010A22E00B0A1EE0020A1CE0030A18E004
:10A52A00080A10E0010A0CE00F0A08E0030A01E039
:10A53A0012000101888F080E716F12000EEF51F0A0
:10A54A00BFEF50F00101720E866F010E876F0CD0BB
:10A55A0061EF51F0D4EF52F034510101866F876BED
:10A56A00730E8627010E87238881010E896F888FD3
:10A57A0012000101888F04013451EA6A730FE96EEF
:10A58A00010EEA2232C4EFFF120016D9020EB6D823
:10A59A0002E2E16AE552E16E00501200120096D919
:10A5AA00E652E652E6520401320510E130511F0B21
:10A5BA0000090CE10101888F030E0401315D04E1F9
:10A5CA000101010E946F02D00101946B0401325112
:10A5DA0001E07FD030511F0B020801E07AD03451DC
:10A5EA000F0B000901E175D034510F0B020871E31A
:10A5FA00200E0101715D6DE1888F040134BF04D022
:10A60A0054D9D4D8DFD803D055D9D0D8DFD8EA2244
:10A61A00020EEFCFDBFFECD8010B02E1DF9401D091
:10A62A00DF8434BF02D041D901D044D9EA22DECF37
:10A63A00EEFFDDCFEDFF030E315D0CE143D907E0FC
:10A64A0034BF02D0BFD801D0C1D8EA22EF82840E2B
:10A65A0067D93FD0DF7436D90BE058D8EF9E56D869
:10A66A00EF8CFAD802E2E16AE552E16E005002D0BC
:10A67A004DD8EF8CDF74BCD8020B02E123D912E06B
:10A68A00040134BF02D09ED801D0A0D8EA22EF92AA
:10A69A003B0E006E36D9E0D802E2E16AE552E16E7D
:10A6AA00005002D03B0E2DD9040134510F0B016A20
:10A6BA00260F006E0F0E0122030E00C0DBFF040EF0
:10A6CA0001C0DBFF030EDBCFE9FF040EDBCFEAFF9D
:10A6DA00EF90050EE15C02E2E16AE552E16EC6D056
:10A6EA0014D9B4D81AEF54F0D7D8E6521200E5526A
:10A6FA00BDD0FD0EEA6ADB346EEF54F0E66EE66A10
:10A70A0001EC62F0006E060EE15C1200DECFE9FF9A
:10A71A00DDCFEAFF12007EC1E9FF7FC1EAFF120026
:10A72A0034510F0BE96EEA6AD890E936EA3612001C
:10A73A0074C1E9FF75C1EAFF1200EDD8380EEE6E5A
:10A74A00040EED6E1200FD0EEA6ADB3475EF54F06A
:10A75A00FC0EDB50E824026EFD0EDB50040DF350B4
:10A76A0002241200DF50C8D8EA22EF6ADF50BFD8AD
:10A77A00EA22EF6ADF2A1200E66E1FEC63F0006E2F
:10A78A00050EE15C1200EA22EE50EFCFEAFFE96E15
:10A79A001200E66E92C1E9FF93C1EAFF922B000E06
:10A7AA009323E552E750EF6EDF061200EA22EECF5E
:10A7BA00DEFFEDCFDDFF1200000EE66EE66AE66E02
:10A7CA00E66A120034510F0B7CEF54F034510F0B30
:10A7DA0081EF54F0012200C0DEFF01C0DDFF12004C
:10A7EA00FD0EDBCFE6FFCBEC4FF0E552E55212004F
:10A7FA00D950020FE96E000EDA20EA6EEF5012000D
:10A80A00160E396F9F0E376F7B0E366F1200010ED0
:10A81A00E66EE66A000EE66EE66A1200F76A8625BA
:10A82A00F66E8751F7220800120076C1E9FF77C158
:10A83A00EAFF1200040DF3CF00F0F4CF01F0000E8E
:10A84A000026040EC7DF840E95EF54F064D8300E4C
:10A85A00EE6E040EED6E1200020EE66EE66ADECFB2
:10A86A00E6FFDDCFE6FF050E83EF53F0E552E5CFB5
:10A87A00DAFFE7CFD9FF1200020EE66EE66AE66A51
:10A88A00270EE66E0F0EC1EF53F02ADF8C0EEF6E25
:10A89A0042DF840EEF6E1200D9CFE6FFDACFE6FF71
:10A8AA00E1CFD9FFE2CFDAFF12003ADF780EE926CC
:10A8BA00010E120035DF7E0EE926010E120019DFA5
:10A8CA00C8EF53F023DFEF50800B12000DDFE65282
:10A8DA001200FE0BEA36E96E7E0EE926010E120020
:10A8EA00FE0BEA36E96E780EE926010E1200EA6AD4
:10A8FA009C0FE96E010E1200EA6A990FE96E010EC9
:10A90A00120004DFE850EF1612008FDFEE52400EFD
:10A91A00EF6E1AEF54F0020EE926000EEA22120038
:10A92A00F5DEE850EF121200D5EC59F0FB0EDBCF42
:10A93A00F3FFDB06F35000090AE023EC5AF0FA0EA3
:10A94A008EEC5AF0F3E1011CF1E1010E01D0000E88
:10A95A0004EF5AF0D5EC59F03B0EE12402E3E1682A
:10A96A00E652E16E010EDB6A020EDB6AF90EDBCFFC
:10A97A00F6FFFA0EDBCFF7FFFB0EDBCFF8FF08007E
:10A98A00F550DF6EDF5002E128EF59F0250EDF5C4B
:10A99A0002E01BEF59F0030EDB6A040EDB6A050EB8
:10A9AA00DB6A060EDB6A070EDB6A3DEC59F02D0EF8
:10A9BA00DF5C0CE02B0EDF5C09E0200EDF5C06E0BA
:10A9CA00230EDF5C03E0300EDF5C1AE1DF50300A51
:10A9DA0014E0130A0FE0030A0AE00B0A05E0060A6C
:10A9EA00E4E1030EDB80E1D7030EDB82DED7030E40
:10A9FA00DB84DBD7030EDB86D8D7030EDB88D5D7FB
:10AA0A002A0EDF5C1BE139EC59F087EC59F010E0B3
:10AA1A00030EDB801E681F68130EDBCF23F0140EB3
:10AA2A00DBCF24F07BEC64F0040E1CC0DBFF03D008
:10AA3A00130E70EC59F03DEC59F00BD0090EDB6A9D
:10AA4A00DEEC59F003E052EC5AF0FAD7090E70EC3A
:10AA5A0059F0030EDBB0DB982E0EDF5C1BE13DECF8
:10AA6A0059F02A0EDF5C0BE139EC59F087EC59F00A
:10AA7A0003E1130EC2EC59F03DEC59F00BD0090E6C
:10AA8A00DB6ADEEC59F003E052EC5AF0FAD7090E11
:10AA9A00C2EC59F0680EDF5C07E13DEC59F0680E34
:10AAAA00DF5C1DE1030E18D0740EDF5C17E07A0E2E
:10AABA00DF5C14E0480EDF5C06E0540EDF5C03E066
:10AACA005A0EDF5C02E1020E07D06C0EDF5C03E077
:10AADA006A0EDF5C04E1010E15EC5AF0C9DBDF50A7
:10AAEA006E0A01E17FD31E0A01E192D1200A01E137
:10AAFA008FD13F0A01E149D11A0A01E146D10D0A73
:10AB0A0001E143D1200A01E140D13A0A01E13DD1F4
:10AB1A00200A01E13AD1260A01E135D10D0A01E103
:10AB2A0032D11A0A01E1D9D0200A4AE0300A1FE0DC
:10AB3A00460A0EE0250A01E083D3D950F90FE96EDF
:10AB4A00FF0EDA20EA6E010EEE5E000EEE5AEE5AA3
:10AB5A0023EC5AF0250EE66E95DB03E1011C01E1B8
:10AB6A0069D31FEC5AF001E26BD3DB2A69D3080ED2
:10AB7A00DB6A040EDB50010806E2040EDB04E7EC94
:10AB8A0059F0DB508BDB080EDB5009E0030EDB507B
:10AB9A00010B05E172DB01E04DD3080EDB6A64DBD1
:10ABAA00EFCFDFFF97EC5AF003E1011C01E142D33A
:10ABBA001FEC5AF001E3DB2A60DB01E141D33AD30F
:10ABCA00070EDB5002080FE163EC5AF0030E2AEC81
:10ABDA005AF00E0EEECFDBFF0F0EEECFDBFF100E9C
:10ABEA00EECFDBFF20D0F70EDBCF03F0F80EDBCF82
:10ABFA0004F0020E035E000E045AF70E03C0DBFFD8
:10AC0A00F80E04C0DBFF03C0E9FF04C0EAFF1AEC38
:10AC1A005AF0026A0E0E00C0DBFF0F0E01C0DBFF06
:10AC2A00100E02C0DBFF0E0EDBCFE6FF0F0EDBCFEE
:10AC3A00E6FF100EDBCFE6FF47EC63F0E552E55284
:10AC4A00E552130E1DC0DBFF140E1EC0DBFF060EFD
:10AC5A00DB5005E0130E5EEC5AF001E26ADB82EC8F
:10AC6A005AF002E2130E37DB45EC5AF006E0040E06
:10AC7A005EEC5AF002E2050E2EDB030EDBB005D0C5
:10AC8A00FCDA01E0D7D2080EDB6A090EDB6A0E0E87
:10AC9A00DBCFF6FF0F0EDBCFF7FF100EDBCFF8FF8F
:10ACAA000800F550DF6EDF5014E088EC5AF011E22C
:10ACBA0097EC5AF003E1011C01E1BCD2BBDB01E3D2
:10ACCA00DB2A090EDB2AD9500E0FE96E000ECBDB08
:10ACDA00E7D7D3DA01E1B4D2ADD2C6DA110EEECF9C
:10ACEA00DBFF120EEDCFDBFF110EDBCFE6FF120EFC
:10ACFA00DBCFE6FF39EC63F0E552E552130EF3CFF2
:10AD0A00DBFF140EF4CFDBFF060EDB5004E0130E5C
:10AD1A00D0DB01E20EDB82EC5AF002E2130EDBDA40
:10AD2A00AFDB05E0040EC5DB02E2050ED4DA030E42
:10AD3A00DBB005D0A2DA01E07DD2080EDB6A090E8B
:10AD4A00DB6A110EDBCFE9FF120EDBCFEAFFEFCF92
:10AD5A00DFFFDF5014E0D7DB12E2E4DB03E1011C82
:10AD6A0001E168D267DB01E3DB2A090EDB2A110E57
:10AD7A00DB2ADBCFE9FF120EE8E3DB2AE6D77DDA2E
:10AD8A0001E15ED257D2030EDB8E070EDB0410E11F
:10AD9A0095DB040E5ADB0A0EEECFDBFF0B0EEECF6D
:10ADAA00DBFF0C0EEECFDBFF0D0EEECFDBFF6CD020
:10ADBA00070EDB5003082CE1030EDBAE0DD0B2DA2E
:10ADCA00020E76DAEFCF00F0016A026A036A00AE79
:10ADDA0039D00168026835D0F70EDBCF01F0F80EE2
:10ADEA00DBCF02F0020E015E000E025AF70E01C01E
:10ADFA00DBFFF80E02C0DBFF01C0E9FF02C0EAFF79
:10AE0A00EFCF00F00A0E00C0DBFF0B0EDB6A38D072
:10AE1A00070EDB50020809E1030EDBAE04D059DB52
:10AE2A0002AE10D00ED055DB0DD0030EDBAE12D021
:10AE3A0079DA020E3DDAF9DA026A036A01AE02D061
:10AE4A0002680368E2DA0C0E02C0DBFF0D0E03C0D3
:10AE5A00DBFF1AD0F70EDBCF02F0F80EDBCF03F0E0
:10AE6A00020E025E000E035AF70E02C0DBFFF80E56
:10AE7A0003C0DBFF02C0E9FF03C0EAFFD6DAC5DA86
:10AE8A000C0EDB6A0D0EDB6A060EDB5005E1010EC5
:10AE9A00F36E050EF3CFDBFF150EDB6A160EDB6AC7
:10AEAA00D950370F006E000EDA20016E390E00C03D
:10AEBA00DBFF3A0E01C0DBFF380EDB6A080EDB6AE5
:10AECA000A0EAEDADF50780A12E0200A10E0280AE9
:10AEDA000CE0200A0AE03F0A06E00D0A02E0200A16
:10AEEA0008E1020E05D0080E03D0080EDF26100E68
:10AEFA0097DA030EDBBE02D0DB92DB94DB50800BC9
:10AF0A0024E08ADAD890030EEB50000A08E6000E15
:10AF1A00EE5C000EEE58000EEE58000EEE5815E2EA
:10AF2A0013DA216822682368246843EC64F00A0E65
:10AF3A0018C0DBFF0B0E19C0DBFF0C0E1AC0DBFFBB
:10AF4A000D0E1BC0DBFF2D0E08D0030EDBA202D0B4
:10AF5A002B0E03D0DBA408D0200EF36E170EF3CF0E
:10AF6A00DBFF150EDB2A02D0170EDB6A050EDB505B
:10AF7A0003E1B7D901E189D0E00E006ECA0E016E75
:10AF8A00000E026E070EDBCF03F0046A056A066A3A
:10AF9A0003C021F004C022F005C023F006C024F04B
:10AFAA00D3D9FAEC64F000501824F36E015019203A
:10AFBA00F46E02501A20F86EF4CFF7FFF3CFF6FFC3
:10AFCA000800090EF5CFDBFF580EDF5C0FE1610EBA
:10AFDA00F36E090E7BD90AE3200E006E090EDBCF51
:10AFEA00E7FF0050E75E090EE7CFDBFF070EDBCF76
:10AFFA0000F0016A026A036A0FDA00C021F001C098
:10B00A0022F002C023F003C024F0EECF1CF0EECFF2
:10B01A001DF0EECF1EF0EFCF1FF0FAEC64F01FC068
:10B02A00EDFF1EC0EDFF1DC0EDFF1CC0EFFF390E86
:10B03A00DBCFE9FFDB063A0EDBCFEAFF01E2DB06F4
:10B04A00090EDBCFEFFF150EDB2A4BD995E1030E74
:10B05A00DBA61DD06F0EDF5C06E1C1D918E3150E21
:10B06A00DB285BDA14D0780EDF5C09E0580EDF5C6F
:10B07A0006E0620EDF5C03E0420EDF5C08E1020ECE
:10B08A00F36E160EF3CFDBFF02D0150EDB6A030E4A
:10B09A00DB50100B0EE0040EDBCF00F0050EDB5088
:10B0AA00D880005406E2060EDB5003E1040EDB50A2
:10B0BA0034DA95D90AE2050EDBCFE7FF150EDB502D
:10B0CA00E75E050EE7CFDBFF02D0050EDB6A040E52
:10B0DA00DBCF00F0160E45D9D880005414E2160EC4
:10B0EA00DBCFE6FF150EDBCFE6FF040EDBCFE6FF74
:10B0FA00050EDB50E552E75CE552D880E754E5528D
:10B10A00D880E7545FD9030EDB50010B0BE1080E20
:10B11A00DB5008E0B2D801E08DD0080EDB50BED873
:10B12A00080EDB6A170EDB5007E088D9170EF1D933
:10B13A0003E1011C01E17ED0160EDB5016E07ED938
:10B14A00300EE66E9FD802E1011C74E077D9DFCF9A
:10B15A00E6FF01EC64F0E552E552E552F4CF01F066
:10B16A000001F31C02E1011C65E0050EDBCF00F0D3
:10B17A00160EDB50D880005409E2050EDBCFE7FF3C
:10B18A00160EDB50E75E050EE7CFDBFF300EE66EEC
:10B19A00050ECBD94FE1390EDB2ADBCFE9FF3A0E98
:10B1AA0001E3DB2ADBCFEAFF090EEFCFDBFFDB503F
:10B1BA000EE044D9090EADD902E1011C3BE0390E7B
:10B1CA00DB2ADBCFE9FF3A0EEDE3DB2AEBD755D8D2
:10B1DA0031E1160EDBCFE6FF080EC3D8E552E724AD
:10B1EA005DD82ED0070EDB50030A1CE0010A14E0DA
:10B1FA00030A07E07BD9DBCFEEFF020EDBCFEDFFC0
:10B20A001FD0F5D8056A03AE02D0046805682CD8A9
:10B21A00BCD805C0EEFF14D0EAD803BE046824D80F
:10B22A00B4D80ED063D9DBCFEFFF0AD07BD905E1C2
:10B23A00011C03E1F368F46810D0FCD801E3DB2AAF
:10B24A0079D9C4EF54F0010EDBCF00F0020EDBCF48
:10B25A0001F000C0F3FF01C0F4FF3B0EE15C02E223
:10B26A00E16AE552E16ECBD029D9020E2AEF5AF0F3
:10B27A0061D90800F550DF6E1200200EE66E080E46
:10B28A009AEF5AF001EC64F0E552E552E552F3CF39
:10B29A0000F0F4CF01F00001F31C1200006E016A05
:10B2AA00D950010F4DD90050EE260150ED2212005F
:10B2BA00045E000E055AF70E04C0DBFFF80E05C047
:10B2CA00DBFF04C0E9FF05C0EAFF1200DBCFF4FF91
:10B2DA00F350F45C1200DB50E76E040EE7CFDBFF9D
:10B2EA0012000A0EDBCF00F00B0EDBCF01F00C0EC2
:10B2FA00DBCF02F00D0EDBCF03F00050011002107D
:10B30A0003101200130EEECFDBFF140EEDCFDBFF9E
:10B31A00130EDBCF00F0140EDBCF01F00001800E1C
:10B32A0001141200F70EDBCF04F0F80EDBCF05F0A4
:10B33A001200050EDB50E66ED950130F01D9E55203
:10B34A00E750EE6EED6A12000A0EDBCF1CF00B0E10
:10B35A00DBCF1DF00C0EDBCF1EF00D0EDBCF1FF086
:10B36A001200DBCFE6FF150EDBCFE6FF050EDB5042
:10B37A00E552E724E552E7241200DB50CED8010E4D
:10B38A00F36E060EF3CFDBFF1200EE50EFCFEAFFAB
:10B39A00E96E02C0EEFF03C0EEFF04C0EEFF12002A
:10B3AA00D9CFE6FFDACFE6FFE1CFD9FFE2CFDAFF66
:10B3BA001200DFCFE6FFE66AE8EC64F0E552E552F8
:10B3CA00F3501200E76E080EE7CFDBFF1200EECF54
:10B3DA0000F0EECF01F0EFCF02F0036A1200050E83
:10B3EA00DBCF00F0150EDB50D88000541200010E9E
:10B3FA00DBCF02F0020EDBCF03F0046A1200E55243
:10B40A00E5CFDAFFE7CFD9FF12000A0E00C0DBFF53
:10B41A000B0E01C0DBFF1200D9500A0FA5EF5AF03C
:10B42A00F36E070EF3CFDBFF1200EECF00F0EFCF83
:10B43A0001F01200010EDB2A020E1200FC0EDBCF15
:10B44A00E6FFFD0EDBCFE6FF1200005E000E015A9A
:10B45A00F70E00C0DBFFF80E01C0DBFF00C0E9FFFA
:10B46A0001C0EAFF1200DA20EA6EEF2AEECFF6FFF9
:10B47A00000EEF22EECFF7FFEF22EECFF8FF120019
:10B48A00040EDBCFE6FF130EDB50E552E75C9ADFD2
:10B49A00DB5004DF060EDB501200090EDB500A0DEA
:10B4AA00F350DF24D00FE76E090EE7CFDBFF3DEF45
:10B4BA0059F0DB50F36E050E6BEF59F0F70EDBCF48
:10B4CA0000F0F80EDBCF01F01200DFCFE6FF47EF06
:10B4DA0059F028DF030EECDEECEF59F099EC54F04A
:10B4EA00E552E552E552E55200091200BDDEEE5082
:10B4FA00EFCFEAFFE96E010E1200130EDB50F36E76
:10B50A00040E6BEF59F0040EDB50F36E090E6BEF6D
:10B51A0059F0DBCFE6FF47EF59F0E76E050EE7CFAC
:10B52A00DBFF12008BDF6AEF5AF0DBCFE6FF86DF24
:10B53A0073EF5AF0D950F90FE96EFF0E38EF5AF04F
:10B54A00E96E000EDA20EA6E1200256C692C256C71
:10B55A00690A0D00514D2C25692C25692C25692C69
:10B56A0025690A0D00253032580D0A002530346944
:10B57A002C253034690D0A002531690D0A00253061
:10B58A0033690D0A00253031306C750D0A002564C7
:10B59A000A0D004D616A6F72206D616C66756E638B
:10B5AA0074696F6E204178697332205374657043F1
:10B5BA006F756E746572207A65726F0A0D004D613F
:10B5CA006A6F72206D616C66756E6374696F6E2046
:10B5DA0041786973322053746570436F756E746570
:10B5EA007220746F6F2068696768203A20256C752D
:10B5FA000A0D004D616A6F72206D616C66756E632B
:10B60A0074696F6E20417869733120537465704391
:10B61A006F756E746572207A65726F0A0D004D61DE
:10B62A006A6F72206D616C66756E6374696F6E20E5
:10B63A0041786973312053746570436F756E746510
:10B64A007220746F6F2068696768203A20256C75CC
:10B65A000A0D002130204572723A20484D203C6183
:10B66A00786973323E207374657020726174652044
:10B67A003E2032354B2073746570732F7365636F88
:10B68A006E642E0A0D002130204572723A20484D10
:10B69A00203C61786973313E207374657020726151
:10B6AA007465203E2032354B2073746570732F7396
:10B6BA0065636F6E642E0A0D002130204572723A5E
:10B6CA0020737465707320746F20686F6D65206CC9
:10B6DA006172676572207468616E2031362C373763
:10B6EA00372C3231352E0A0D002130204572723A3C
:10B6FA00203C61786973323E2073746570207261F0
:10B70A007465203C20312E3331487A2E0A0D0021EF
:10B71A0030204572723A203C61786973323E207358
:10B72A007465702072617465203E2032354B207337
:10B73A00746570732F7365636F6E642E0A0D002132
:10B74A0030204572723A203C61786973323E206C2F
:10B75A006172676572207468616E203136373737D7
:10B76A003231352073746570732E0A0D0021302032
:10B77A004572723A203C61786973313E2073746570
:10B78A00702072617465203C20312E3331487A2E44
:10B79A000A0D002130204572723A203C61786973A3
:10B7AA00313E20737465702072617465203E2032C8
:10B7BA00354B2073746570732F7365636F6E642ED7
:10B7CA000A0D002130204572723A203C6178697373
:10B7DA00313E206C6172676572207468616E203137
:10B7EA00363737373231352073746570732E0A0D48
:10B7FA00002130204572723A203C6D6F76655F6495
:10B80A0075726174696F6E3E206C61726765722031
:10B81A007468616E203136373737323135206D73AF
:10B82A002E0A0D005374617475733D25690D0A0063
:10B83A002135204572723A204E65656420636F6D2A
:10B84A006D61206E6578742C20666F756E643A207F
:10B85A00272563270D0A0025730D0A0050617261BE
:10B86A006D383D25630D0A00506172616D373D25C3
:10B87A00630D0A00506172616D363D256C750D0AC3
:10B88A0000506172616D353D256C640D0A0050618E
:10B89A0072616D343D25750D0A00506172616D3318
:10B8AA003D25640D0A00506172616D323D25640DBB
:10B8BA000A00506172616D313D25640D0A0025311F
:10B8CA00750D0A0050492C2531750D0A004D522C70
:10B8DA00253033750D0A002C253032753A2530345F
:10B8EA0075004100492C253033692C253033692CE9
:10B8FA00253033692C253033692C253033690D0AFC
:10B90A00002138204572723A20556E6B6E6F776E41
:10B91A0020636F6D6D616E642027256325633A2568
:10B92A003258253258270D0A002138204572723ABA
:10B93A0020556E6B6E6F776E20636F6D6D616E64EE
:10B94A00202725633A253258270D0A00213720453A
:10B95A0072723A204578747261207061726D6174F6
:10B96A0065720D0A002136204572723A20496E76B8
:10B97A00616C696420706172616D746572207661B0
:10B98A006C75650D0A002134204572723A204D69A2
:10B99A007373696E6720706172616D657465722870
:10B9AA0073290D0A002133204572723A2052582019
:10B9BA00427566666572206F76657272756E0D0ADB
:10B9CA00002132204572723A205458204275666628
:10B9DA006572206F76657272756E0D0A00213120CC
:10B9EA004572723A2043616E277420737465702021
:10B9FA007468617420666173740D0A002130200D29
:10BA0A000A002008002573001B5B421B5B314B1B9D
:07BA1A005B3047000D0A003C
:10BA2200040130511F0B010801E012003051600B7C
:10BA3200E842E842E842E842E842010801E0120036
:10BA4200345103E0340501E012003151220A31E0A1
:10BA5200030A24E0010A15E0210A0DE0010A01E0CF
:10BA620012000101A00E866F060E876F080E896F05
:10BA72008A6B888121D00101A00E866F060E876F26
:10BA82001BD036C48EF137C48FF10101800E8B6F4B
:10BA9200060E8C6F906B916B8D8F12000101800EE0
:10BAA200866F060E876F070E896F8A6BC10E886FCD
:10BAB200120032C49BF60101888F12000601806BCE
:10BAC2004B0E816F826B836B846B856B080E866F66
:10BAD2008F6B1A0EE66E010EE66EEFEC4EF0E5523B
:10BAE200E5521E0EE66E020EE66EEFEC4EF0E552E9
:10BAF200E5522FD902E2E16AE5524FD90601996B6C
:10BB02009A6B906B12001CD982D9050E1E1801E1A6
:10BB12001F5002E0000E18D051D9060197510018AB
:10BB220008E19851011805E114D902E2E16AE552EF
:10BB320034D944D906019951001805E19A510118E6
:10BB420002E1906B956B010E0CD1FAD806018F6B56
:10BB52009751981102E1000E05D045D9EF50800BA4
:10BB620001E0010E000931E1FB0EDBCF00F03BD911
:10BB7200EE52EF50D880005405E235D9EE52FB0E5A
:10BB8200EFCFDBFF8F6BFB0EDB508F5D19E28F5126
:10BB9200EA6A400FE96E060EEA22EF50E66E8F5116
:10BBA200E76EFC0EDBCFE9FFFD0EDBCFEAFFE750CD
:10BBB200E926000EEA22E552E750EF6E8F2BE3D71B
:10BBC200C8D802E2E16AE552E8D806018F51C9D02D
:10BBD200B7D80601905107E1E7D8FB0EDBCF95F607
:10BBE200010E966F906FBDD00BD917E1C0D8EDD87A
:10BBF20002E101500BE0010EDBCFE9FFDB2A020E6E
:10BC0200DBCFEAFF01E3DB2AEF50F1E1CDD8DFCF52
:10BC120095F60601010E966F906FE552E552E552D8
:10BC2200A0D0EED818E1A3D8D0D802E101500CE0A0
:10BC3200010EDBCFF6FFDB2A020EDBCFF7FF01E3BB
:10BC4200DB2A0800F550F0E1AFD8DFCF95F6060108
:10BC5200966B010E906FE552E552E55282D070D894
:10BC6200E652E652060199519A1102E1000E08D0FD
:10BC720099C6E9FF9AC6EAFFEF50800B01E0010E78
:10BC820000095BE1030E905D01E1906B905155E07C
:10BC9200020E905D0DE1E66A000EE66EE66A8BD852
:10BCA20002E2E16AE55298D80601030E906F45D090
:10BCB200900543E1400E006E016A9551005C000E52
:10BCC200015803E2400EDF6E02D095C6DFFFDF505F
:10BCD200955D956F000E936F060E946F010EDFCF88
:10BCE200DBFF96510BE1010EDB5012E091C6F6FF2D
:10BCF20092C6F7FF0800F55043D8F5D7010EDB5086
:10BD020007E091C6E9FF92C6EAFFEF5039D8F6D7AD
:10BD12000601955107E1400EDF5C02E1020E01D0FF
:10BD2200030E906FDFCFE6FF000EE66E060EE66EA4
:10BD320042D802E2E16AE5524FD8E552E55211D00B
:10BD4200D9CFE6FFDACFE6FFE1CFD9FFE2CFDAFFC4
:10BD52001200400EE66E400EE66E060EE66EE66AD3
:10BD620047D0E552E5CFDAFFE7CFD9FF1200DF6A0D
:10BD72004ED8DE521EC0DEFF1FC0DDFFDD521200B4
:10BD820093C6E9FF94C6EAFFEF6E932B000E94234D
:10BD9200912B9223010EDB061200E16E0050F3CFCD
:10BDA20097F6F4CF98F61200FC0EDBCF91F6FD0E5B
:10BDB200DBCF92F61200010EE66E1AD0FA0EDBCF3E
:10BDC20000F0FB0EDBCF01F01200DF2ADF50006E25
:10BDD200016AFF0E00181200E16E0050F3CF99F6CF
:10BDE200F4CF9AF6120097C6E9FF98C6EAFF12004E
:10BDF200020EE66E0EEC4FF0006E050EE15C1200D4
:10BE02009FDFE652E652E652060190511200FC0E06
:10BE1200DBCF1EF0FD0EDBCF1FF0120078D9E65209
:10BE22000E01006BA96BDF6A180EDF5C14E291D978
:10BE3200010EE9260E0E93D9DF5085D9EF6A89D912
:10BE4200490EE9260E0E8BD984D9790EE9260E0EFB
:10BE520086D9DF2AE9D70E01C60EAC6F0E0EAD6F82
:10BE62003F0E79140009796ECF0E79140009796EAC
:10BE720079827B6A7A6A79900F0152815293F00E2D
:10BE8200B4140909B46E0E01080EAA6F030EAB6F4B
:10BE9200C60EAE6F3B0EAF6F250EB06F580EB16F70
:10BEA200040EB66F900EB26F010EB36F900EB46FA8
:10BEB200010EB56F000EE66EE66A010EE66E57ECF5
:10BEC20031F0E552E552E5528996E55236D11FD955
:10BED200E652DF6A180EDF5C0AE2DF5034D9EFCF98
:10BEE20000F0FD0EDB50005C0AE0DF2AF3D7DF6AC8
:10BEF200180EDF5C08E2DF5026D9EF5002E1DF289E
:10BF020003D0DF2AF5D7000EE55217D100D9070E6C
:10BF1200E12402E3E168E652E16EDE6ADD6A020EC6
:10BF2200DB6A030EDB6A040EDB6A050EDB6A060EB1
:10BF3200DB6A010EE66ED9CFE6FFDACFE6FF030E2B
:10BF4200EFD8020F10D9010EEBD8030F0CD9030E54
:10BF5200E7D8050F08D9030E0BD90601B45124E125
:10BF6200020EDB50180802E2B48D1ED0050EDBCFA4
:10BF7200E6FF060EDBCFE6FF030EDBCFE6FF040E85
:10BF8200DBCFE6FF020EDBCFE6FFDECFE6FFDDCF43
:10BF9200E6FF11D8006E070EE15C02E2E16AE552AB
:10BFA200E16E0050E7EC41F0070EE15C02E2E16A6B
:10BFB200E552E16EC2D0ABD8E652E652FB0EDBCFC1
:10BFC200E6FF85DFE552E76E010EE7CFDBFFDB50D0
:10BFD20002E1000E99D0D950FC0FE96EFF0EDA2073
:10BFE200EA6EEE50ED101FE1010EDB04ACD8EF500B
:10BFF2000E01EA6AAC25E96EAD51EA22EF6A95D8E4
:10C00200790EE9260E0EABD890D8490EE9260E0E0F
:10C01200A6D8010EDB0497D8EF6A87D8010EE9266D
:10C022000E0E9DD86FD0010EDB04006E0E01AA51D8
:10C03200005C68E2FB0EDB50180864E3FB0EDB5089
:10C04200070802E10401F26B70D8010EE9260E0E18
:10C05200EA22EE50ED1010E1E66AFB0EDBCFE6FFBE
:10C062002EEC4BF0E552E552E66AFB0EDBCFE6FF23
:10C0720000EC4BF0E552E5520401A951FDE0FB0E44
:10C08200DB50040809E189861DC519F51EC51AF59C
:10C092001FC51BF520C51CF50401030EB66FF70E74
:10C0A200DBCFD0F4F80EDBCFD1F4D26BD36B190E09
:10C0B200216E226A236A246AD0C41CF0D1C41DF006
:10C0C200D2C41EF0D3C41FF043EC64F018C0D0F405
:10C0D20019C0D1F41AC0D2F41BC0D3F4010EDBCFC5
:10C0E200D7F4FB0EDBCFD6F4FC0EDBCFD4F4FD0E7F
:10C0F200DBCFD5F4F90EDBCFD8F4FA0EDBCFD9F4CF
:10C102000401A96B010EDB50E552E55216D0D9CFDE
:10C11200E6FFDACFE6FFE1CFD9FFE2CFDAFF120086
:10C1220027D8010EE66ED9501200010EDB04E96E2B
:10C13200EA6AD890E936EA361200E552E5CFDAFF2C
:10C14200E7CFD9FF1200EA6A310FE96E0E0EEA223A
:10C152001200EA6ADF34FE0BEA36E96E1200EA22C6
:10C16200EE6AED6A1200E66E000EDA20E66E12004A
:10C17200E66ED2EC48F0E552E552E552E552120085
:10C18200D9CFE6FFDACFE6FFE1CFD9FFE2CFDAFF80
:10C19200060EE12402E3E168E652E16EDF6A010E77
:10C1A200DB6AD950FA0FE96EFF0EDA20EA6E020E50
:10C1B200EECFDBFF030EEECFDBFF040EEECFDBFF95
:10C1C200050EEECFDBFFD950FA0FE96EFF0EDA2033
:10C1D200EA6E060EE76ED890030EEB32020EEB32D9
:10C1E200010EEB32EF32E706F6E1D950FA0FE96EB3
:10C1F200FF0EDA20EA6E060EE76ED890EF36010ED9
:10C20200EB36020EEB36030EEB36E706F6E1D950BB
:10C21200FA0FE96EFF0EDA20EA6E400EEE26000EED
:10C22200EE22000EEE22000EEE22FA0EDBCF04F01A
:10C23200FB0EDBCF05F0FC0EDBCF06F0FD0EDBCFF5
:10C2420007F0D950020FE96E000EDA20EA6EEE50C6
:10C25200045C006EEE500558016EEE500658026EF8
:10C26200EE500758036E0050DF6ED950F80FE96E9A
:10C27200FF0EDA20EA6EEE50ED1065E0040EDB50A0
:10C28200F86E030EDB50F76E020EDB50F66EDF50D7
:10C29200DF0600091AE0F60EDBCFE9FFDB2AF70E14
:10C2A200DBCFEAFF01E3DB2AEF50F56E0D00F80E5B
:10C2B200DB06DBCF00F0F90E01E2DB06DBCF01F09B
:10C2C2000050011001E101D0E2D7040EDB50F86EFC
:10C2D200030EDB50F76E020EDB50F66EA684F2AE52
:10C2E20004D0F29EDE52010EDD6E550EA76EAA0E2E
:10C2F200A76EA682A694010EDB5003E0F28E010E19
:10C30200DB6A400EDF6E400E006E016A026A036A4B
:10C31200D950020FE96E000EDA20EA6EEE500026C6
:10C32200EE500122EE500222EE500322020E00C015
:10C33200DBFF030E01C0DBFF040E02C0DBFF050EB4
:10C3420003C0DBFF92D7060EE15C02E2E16AE5522E
:10C35200E16EE552E5CFDAFFE7CFD9FF120005D84B
:10C3620031EC4EF055EC3DF0FBD78ED8E652E6525A
:10C372000F0148694969600ED36E9B8C580EDE6EC0
:10C38200020EDD6EDFCF00F0DF06010EDBCF01F023
:10C3920001E2DB0600500110F5E1948E8AEC3CF0DC
:10C3A200C7EC4DF0E552E55278D0120012001200AF
:10C3B200120011EF5DF012005FEF5DF001019405D4
:10C3C2001EE1010195051BE1F1DF65920101956B0B
:10C3D2000201100EFE6F0E0EFF6FFE07000EFF5BD6
:10C3E200FE51FF11FAE16584080EFE6F070EFF6F22
:10C3F200FE07000EFF5BFE51FF11FAE16594120089
:10C4020043D8FC0EDBCF1EF0FD0EDBCF1FF0050E76
:10C412001E1801E11F5036E0E8681E1802E17F0E87
:10C422001F182FE0030E1E1801E11F5028E0020E14
:10C432001E1801E11F5021E0010E1E1801E11F50DC
:10C442001AE0740E1E1801E11F5013E0750E1E183B
:10C4520001E11F500CE0730E1E1801E11F5005E0B0
:10C46200720E1E180FE11F500DD0A1DF0BD09DDF01
:10C4720009D09CDF07D0A0DF05D09DDF03D099DF74
:10C4820001D096DF010E09D0D9CFE6FFDACFE6FF61
:10C49200E1CFD9FFE2CFDAFF1200E552E5CFDAFFB2
:10C4A200E7CFD9FF1200D9CFE6FFDACFE6FFE1CF1F
:10C4B200D9FFE2CFDAFFE652E652E652E652E65200
:10C4C200DF6AD950FA0FE96EFF0EDA20EA6E010E2A
:10C4D200EECFDBFF020EEECFDBFF030EEECFDBFF74
:10C4E200040EEECFDBFFF60EDBCF00F0F70EDBCF54
:10C4F20001F0F80EDBCF02F0F90EDBCF03F048D8E3
:10C502000050EE5C0150EE580250EE580350EE58C7
:10C5120033E2030EDB50F86E020EDB50F76E010EB3
:10C52200DB50F66EA684A688F2AE03D0F29E010E10
:10C53200DF6E550EA76EAA0EA76EA682DF5001E02F
:10C54200F28E006A040E016E026A036A21D8EE506E
:10C552000026EE500122EE500222EE500322010E7E
:10C5620000C0DBFF020E01C0DBFF030E02C0DBFFD7
:10C57200040E03C0DBFFB7D7050EE15C02E2E16AFD
:10C58200E552E16EE552E5CFDAFFE7CFD9FF1200BF
:10C59200D950010FE96E000EDA20EA6E12002A0E5F
:10C5A200F66E100EF76E000EF86E04010900F550DB
:10C5B200F96F0900F550FA6F03E1F96701D03DD038
:10C5C2000900F550F46F0900F550F56F0900F550B8
:10C5D200F66F09000900F550E96E0900F550EA6EA0
:10C5E200090009000900F550F76F0900F550F86FCE
:10C5F20009000900F6CFFBF4F7CFFCF4F8CFFDF405
:10C60200F4C4F6FFF5C4F7FFF6C4F8FF0401F753CC
:10C6120002E1F85307E00900F550EE6EF707F8E281
:10C62200F807F9D7FBC4F6FFFCC4F7FFFDC4F8FF17
:10C632000401F907000EFA5BBFD71200FE0EE3CF2A
:10C64200E9FFFF0EE3CFEAFFE9CFF3FFEACFF4FF02
:10C65200FB0EE35003E1FC0EE35009E0FB0EE306A0
:10C6620002E2FC0EE306FD0EE350EE6EF1D712007D
:10C67200FE0EE3CFE9FFFF0EE3CFEAFFF36AF46AAF
:10C68200EE5203E0F34AF42AFBD71200FF0EE3CF87
:10C69200F8FFE552FF0EE3CFF7FFE552FF0EE3CFBF
:10C6A200F6FFE552E66AE66AE66A0900F55209E033
:10C6B200FD0EE32A05E1FE0EE32A02E1FF0EE32A64
:10C6C200F4D7FD0EE3CF1DF0FE0EE3CF1EF0FF0EFA
:10C6D200E3CF1FF01200D9CFE6FFDACFE6FFE1CFBA
:10C6E200D9FFE2CFDAFFE652E652E652E652D950DD
:10C6F200FB0F006EFF0EDA20016E00C0DEFFDD6E62
:10C70200DECFE6FFDDCFE6FFFB0EDBCFE6FFFC0E62
:10C71200DBCFE6FFFD0EDBCFE6FFFEC4E6FFFFC484
:10C72200E6FFAFEC54F0006E070EE15C02E2E16A54
:10C73200E552E16E0050020EF3CFDBFF030EF4CFA1
:10C74200DBFF020EDBCF00F0030EDBCF01F000C0F7
:10C75200F3FF01C0F4FF040EE15C02E2E16AE5527C
:10C76200E16EE552E5CFDAFFE7CFD9FF1200D9CF6C
:10C77200E6FFDACFE6FFE1CFD9FFE2CFDAFFE652FA
:10C78200E652E652E652D9CFE9FFDACFEAFFFA0ED5
:10C79200DBCFEEFFFB0EDBCFEEFFFC0EDBCFEEFFBF
:10C7A200FD0EDBCFEEFF020EDB50F86E010EDB500A
:10C7B200F76EDF50F66EF80EDBCF00F0DB06F90EF7
:10C7C200DBCF01F001E2DB06005001100DE00900B1
:10C7D200F60EDBCFE9FFDB2AF70EDBCFEAFF01E340
:10C7E200DB2AF5CFEFFFE7D7040EE15C02E2E16A54
:10C7F200E552E16EE552E5CFDAFFE7CFD9FF12004D
:10C80200D9CFE6FFDACFE6FFE1CFD9FFE2CFDAFFF9
:10C81200FB0EDBCF00F0FC0EDBCF01F00001800E3F
:10C8220001141AE1FB0EDBCFE9FFFC0EDBCFEAFFBE
:10C83200EECFF3FFEDCFF4FFEE2A000EEF22F3CF9F
:10C84200E9FFF4CFEAFFFD0EDBCFEFFFEF50016A05
:10C85200F36E01C0F4FF10D0FB0EDB50FE0806E1C0
:10C86200FD0EDBCFE6FF57EC65F005D0FD0EDBCF0A
:10C87200E6FFC9EC3EF0E552E552E5CFDAFFE7CF3D
:10C88200D9FF12001C502102F3CF18F0F4CF19F097
:10C892002202F3501926000EF4201A6E1C502302B5
:10C8A200F3501A26000EF4201B6E1C502402F35083
:10C8B2001B261D502102F3501926F4501A22000E95
:10C8C2001B221D502202F3501A26F4501B221D5027
:10C8D2002302F3501B261E502102F3501A26F45055
:10C8E2001B221E502202F3501B261F502102F3501E
:10C8F2001B2612001FC02BF01EC02AF01E5023025E
:10C90200F4CF1DF0F3CF1CF01F502402F4CF1FF020
:10C91200F3CF1EF02302F3501D26F4501E22E86AC4
:10C922001F222A502402F3501D26F4501E22E86AC8
:10C932001F2224AEA1EF64F02A501E5E2B501F5A14
:10C942002BAE000C23501E5E24501F5A000C120105
:10C95200000202000040D80492FD8201010203019C
:10C9620009024300020100C0320904000001020270
:10C97200010005240010010424020205240600011E
:10C9820005240100010705810308000209040100D2
:10C99200020A0000000705020240000007058202A9
:05C9A20040000062C925
:10C9A800FF0EE124E96EFF0EE220EA6EEDCFF4FF00
:10C9B800EFCFF3FFF46607D0600EF36404D07B0E6C
:10C9C800F36001D0F39A1200F36AF46AFF0EE124CF
:10C9D800E96EFF0EE220EA6EED6607D02F0EEF64D7
:10C9E80004D03A0EEF6001D0F32A12001B6A1A6ACB
:10C9F800196A186A200EE76ED8901C361D361E3646
:10CA08001F36183619361A361B362150185C225034
:10CA1800195823501A5824501B5809E32150185EFE
:10CA28002250195A23501A5A24501B5A1C2AE72EEE
:10CA3800E4D712004F4B0D0A000D0A00454242761A
:10CA480031335F616E645F61626F766520454220B5
:10CA58004669726D776172652056657273696F6E8B
:10CA680020322E372E300D0A0001C00EF36E00EE74
:10CA780000F00E0E01D81200EA6002D0EE6AFCD770
:10CA8800F350E9601200EE6AFCD71DEE00F02DEEBF
:10CA980000F0F86A279CD0EC62F079EC65F0B0EC15
:10CAA80061F0FBD71200FF0EE350ADBA04D0B06AB4
:10CAB800AC8EAD8A949CADA2FED7AE6EF36EF46ACE
:10CAC8001200F36AF46AF32A0F0B05E0D890F336E4
:10CAD800F436E804FBE112003031323334353637AE
:09CAE8003839616263646566007F
:10CAF20012000403090418035300630068006D0068
:10CB020061006C007A004800610075007300380310
:10CB12004500690042006F00740042006F0061002E
:10CB2200720064002C002000200020002000200061
:10CB320020002000200020002000200020002000F3
:10CB420020002000200022032000200020002000DE
:10CB520020002000200020002000200020002000D3
:10CB62002000200020002000800284029C02D402C7
:10CB7200FEFF0000000000000000000000000000B6
:10CB82000000000000000000000000000000006043
:10CB9200EA000000000000000000000000000000A9
:10CBA2000000000000000000000000000000000083
:10CBB2000000000000000000000000000000000073
:10CBC2000000000000000000000000000000000063
:10CBD2000000000000000000000000000000920FB2
:10CBE200920F920F930F930F930F930F930F930F35
:10CBF200930F930F940F940F940F940F940F940F1D
:10CC0200940F940F950F950F950F950F950F950F04
:10CC1200890F890F890F8A0F8A0F8A0F8A0F8A0F4D
:10CC22008A0F8A0F8A0F8B0F8B0F8B0F8B0F8B0F35
:10CC32008B0F8B0F8B0F8C0F8C0F8C0F8C0F8C0F1D
:10CC42008C0F000105000102030405060700010222
:0BCC52000304050607020304050607A3
:08FFF800ACF70AFF63F801F009
:00000001FF
